:100000000C94D0260C9475B10C944AB10C941FB189
:100010000C94F4B00C94C9B00C949EB00C9473B0D2
:100020000C9448B00C9401270C9401270C940127E0
:100030000C9401270C94FD9A0C9401270C94012731
:100040000C9401270C94D9430C9401270C9401279C
:100050000C9401270C9401270C94C1620C9402B3F8
:100060000C9401270C9448F80C94ECF80C9401279C
:100070000C9401270C9401270C9401270C94012760
:100080000C9401270C9401270C9401270C94012750
:100090000C9401270C9401270C9401270C94012740
:1000A0000C9401270C9401270C9401270C94012730
:1000B0000C9401270C9401270C9401270C94012720
:1000C0000C9401270C9401270C9401270C94012710
:1000D0000C9401270C9401270C9401270C94012700
:1000E0000C9401273CA922A925A928A92BA937A945
:1000F0002EA945A931A934A9AFACB2ACA1ACA5AC2D
:10010000ABACE9ACB6ACBAACC0ACC4ACC8ACCEAC71
:10011000D2ACD6ACE9ACDCACE0ACE4AC1EB223B201
:1001200028B232B23CB2B5B246B24EB256B260B2AA
:100130006AB274B283B28DB2B5B297B2A1B2ABB2A9
:1001400077F87DF88EF899F8A1F8B6F8A5F8B6F822
:10015000A9F8ADF8B6F8B3F8ACFCACFCB3FCB3FC52
:10016000B3FCBAFCBAFCBAFCC7FCC1FCC1FCC1FCC4
:10017000084AD73B3BCE016E84BCBFFDC12F3D6C0E
:1001800074319ABD56833DDA3D00C77F11BED9E474
:10019000BB4C3E916BAAAABE000000803F05A84C54
:1001A000CDB2D44EB93836A9020C50B99186880820
:1001B0003CA6AAAA2ABE000000803F004E414E493C
:1001C0004E495459494E46CDCCCC3D0AD7233C1715
:1001D000B7D13877CC2B329595E6241FB14F0A0062
:1001E0000020410000C84200401C4620BCBE4CCA52
:1001F0001B0E5AAEC59D74434F4D4D554E4943415C
:1002000054494F4E0044525952554E004552524F98
:10021000525300494E464F004543484F0020746FEB
:100220006F206C6F6E6720657874727573696F6E7E
:100230002070726576656E7465640A0020636F6C69
:100240006420657874727573696F6E20707265765C
:10025000656E7465640A00536C6565702E2E2E0001
:10026000436C69636B20746F20726573756D652EC6
:100270002E2E004E6F206D6F76652E00456E642029
:1002800066696C65206C6973740A00426567696E03
:100290002066696C65206C6973740A004D313235D3
:1002A00000286E6F2066696C6529005344207072C7
:1002B000696E74696E67206279746520004E6F7490
:1002C000205344207072696E74696E670A0043752A
:1002D0007272656E742066696C653A2000507269AE
:1002E0006E742074696D653A200050726F74656396
:1002F0007465642050696E0A00000125301D0CFFF2
:100300002829FF24311C0BFF4527FF232F1B0AFF41
:100310004443FFFFFF040308060202222B1A414256
:10032000FF033809FF36180213020C020502F70119
:100330006F66660044454255473A006F6B00205790
:100340003A00457874727564657220436F6F6C690A
:100350006E672E2E2E004578747275646572204883
:10036000656174696E672E2E2E0020573A00426533
:100370006420636F6F6C696E672E2E2E0042656479
:100380002068656174696E672E2E2E007A5F6D6934
:100390006E3A2000795F6D696E3A2000785F6D6972
:1003A0006E3A20005265706F7274696E6720656ED8
:1003B0006473746F70207374617475730A002054D1
:1003C00000205200416363656C65726174696F6EF1
:1003D0003A2050004F666673657473206170706CCC
:1003E000696564004572723A20546F6F20666172CD
:1003F0002100546F6F206661722066726F6D2072EB
:1004000065666572656E636520706F696E740A005B
:10041000205A00205900580020204D61783A2000D1
:10042000205A00205900580020204D696E3A2000C3
:100430004F6E20004F666600536F667420656E64D1
:1004400073746F70733A200020466C6F773A200007
:1004500020643A0020693A0020703A00496E7661C3
:100460006C69642065787472756465720A0043294A
:100470000A0061626C656420286D696E2074656D88
:10048000702000436F6C64206578747275646573C6
:100490002061726520004B64200023646566696EEC
:1004A000652044454641554C545F004B692000236C
:1004B000646566696E652044454641554C545F004D
:1004C0004B70200023646566696E65204445464193
:1004D000554C545F00504944204175746F74756EDB
:1004E000652066696E6973686564212050757420A3
:1004F000746865206C617374204B702C204B6920EC
:10050000616E64204B6420636F6E7374616E7473EC
:100510002066726F6D2062656C6F7720696E746FF4
:1005200020436F6E66696775726174696F6E2E68BD
:100530000A00504944204175746F74756E652066D9
:1005400061696C6564212074696D656F75740A005A
:10055000453120544845524D414C2052554E41574B
:1005600041590042454420544845524D414C205287
:10057000554E4157415900546865726D616C205267
:10058000756E617761790045312048656174696EE7
:1005900067206661696C6564004265642068656116
:1005A00074696E67206661696C6564004865617492
:1005B000696E67206661696C65640050494420413A
:1005C00075746F74756E65206661696C6564212051
:1005D00054656D706572617475726520746F6F20FB
:1005E000686967680A00204B643A2000204B693A2A
:1005F0002000204B703A20000A20436C617373691D
:100600006320504944200A002054753A2000204BB2
:10061000753A2000206D61783A2000206D696E3AAD
:10062000200020643A200020626961733A20005063
:100630004944204175746F74756E65206661696CFC
:100640006564212042616420657874727564657206
:10065000206E756D6265720A0050494420417574C0
:100660006F74756E652073746172740A0020643A49
:100670000020693A0020703A004E6F206361736574
:10068000206C696768740A00454550524F4D204FF1
:100690004B0A00496E736572742066696C616D6502
:1006A0006E7420616E64207072657373206275745D
:1006B000746F6E20286F72204D313038290A005037
:1006C0007265737320627574746F6E20286F722068
:1006D0004D3130382920746F2068656174206E6F49
:1006E0007A7A6C650A00496E736572742066696C6B
:1006F000616D656E7420616E642070726573732025
:10070000627574746F6E20286F72204D31303829F5
:100710000A00416374697665204578747275646572
:10072000723A2000496E76616C6964206578747253
:10073000756465720A0024F4D43050C38E20C2A2BE
:100740004017828B7011127A910D816CD90AA861C1
:10075000E108C7586607615143061E4B5D05C14558
:10076000A7041A411104093D980371393103403639
:10077000DB0265339102D4305402802E1D02632CBB
:10078000EE01752AC501B028A001102781018F252F
:1007900064012B244B01E0223401AC211F018D2088
:1007A0000D01801FFC00841EED00971DDF00B81CAA
:1007B000D200E61BC600201BBC00641AB200B219AE
:1007C000A8000A19A0006A189900D11791004017D3
:1007D0008B00B516840031167E00B31579003A15EA
:1007E0007300C7146F0058146A00EE136600881374
:1007F000630025135E00C7125B006C1257001512D0
:100800005400C111510070114F0021114B00D6103E
:1008100049008D1047004610440002104200C00FEE
:100820004000800F3E00420F3C00060F3B00CB0E05
:100830003800930E37005C0E3500270E3400F30DA0
:100840003200C10D3100900D3000600D2E00320DD0
:100850002D00050D2C00D90C2B00AE0C2900850CA9
:1008600029005C0C2700350C27000E0C2600E80B35
:100870002400C40B2400A00B23007D0B23005A0B83
:100880002100390B2100180B2000F80A1F00D90A9B
:100890001E00BB0A1E009D0A1D00800A1D00630A7F
:1008A0001C00470A1B002C0A1B00110A1A00F7093A
:1008B0001A00DD091900C4091900AB0919009209D1
:1008C00017007B091800630917004C091600360948
:1008D0001600200916000A091500F5081500E008A1
:1008E0001400CC081400B8081400A40814009008E0
:1008F00013007D0812006B08130058081200460808
:100900001200340811002308110012081100010818
:100910001100F0071000E0071000D0071000C0071A
:100920001000B0070F00A107100091070E00830709
:100930000F0074070F0065070E0057070E004907E8
:100940000E003B070D002E070E0020070D001307B9
:100950000D0006070D00F9060C00ED060D00E0067F
:100960000C00D4060C00C8060C00BC060C00B00637
:100970000C00A4060B0099060C008D060B008206E5
:100980000B0077060B006C060B0061060A00570689
:100990000B004C060A0042060A0038060A002E0622
:1009A0000A0024060A001A060A00100609000706B3
:1009B0000A00FD050900F4050900EB050900E20540
:1009C0000900D9050900D0050900C7050900BE05C1
:1009D0000900B5050800AD050800A50509009C053E
:1009E0000800940508008C050800840508007C05B3
:1009F0000800740508006C050700650508005D0522
:100A00000700560508004E0507004705070040058A
:100A1000080038050700310507002A0507002305EF
:100A200007001C050600160507000F05070008054E
:100A3000060002050700FB040600F5040700EE04AB
:100A40000600E8040600E2040700DB040600D50403
:100A50000600CF040600C9040600C3040600BD0456
:100A60000600B7040600B1040500AC040600A604A5
:100A70000600A00405009B040600950405009004F0
:100A800006008A04050085040500800406007A0437
:100A9000050075040500700405006B04050066047C
:100AA0000500610405005C040500570405005204BC
:100AB00005004D04050048040500430405003E04FC
:100AC00004003A04050035040500300404002C0439
:100AD000050027040400230405001E0404001A0472
:100AE000040016040500110404000D0404000904A8
:100AF00005000404040000040400FC030400F803DF
:100B00000400F4030400F0030400EC030400E80311
:100B10000400E4030400E0030400DC030400D80341
:100B20000400D4030400D0030400CC030400C80371
:100B30000300C503030024F404D9201BC40C5C0E7D
:100B40009804C4095F0265077101F405F900FB040C
:100B5000B30048048700C10369005803550003032C
:100B60004500BE023A008402310053022A002902E5
:100B7000250004022000E4011C00C8011900AF0197
:100B80001700980114008401130071011000610125
:100B9000100051010E0043010D0036010B002B0126
:100BA0000B0020010B00150109000C0109000301D5
:100BB0000800FB000800F3000800EB000700E40059
:100BC0000600DE000600D8000600D2000600CC00B9
:100BD0000500C7000500C2000500BD000400B90003
:100BE0000400B5000400B1000400AD000400A90039
:100BF0000400A5000300A20003009F0004009B0066
:100C00000300980003009500020093000300900089
:100C100003008D0002008B000300880002008600A4
:100C2000020084000300810002007F0002007D00BA
:100C300002007B00020079000200770001007600CC
:100C400002007400020072000100710002006F00D7
:100C500002006D0001006C0002006A0001006900E2
:100C600002006700010066000100650001006400E9
:100C700002006200010061000100600001005F00ED
:100C800002005D0001005C0001005B0001005A00F1
:100C900001005900010058000100570001005600F2
:100CA00001005500010054000100530000005300F2
:100CB00001005200010051000100500001004F00EE
:100CC00001004E0000004E0001004D0001004C00EC
:100CD00001004B0000004B0001004A0001004900E8
:100CE00001004800000048000100470001004600E4
:100CF00000004600010045000000450001004400DE
:100D000001004300000043000100420000004200D7
:100D100001004100000041000100400001003F00CF
:100D200000003F0001003E0000003E0001003D00C9
:100D300000003D0001003C0000003C0000003C00C1
:100D400001003B0000003B0001003A0000003A00B7
:100D500001003900000039000100380000003800AF
:100D600000003800010037000000370001003600A5
:100D7000000036000000360001003500000035009C
:100D80000000350001003400000034000000340091
:100D90000100330000003300000033000100320086
:100DA000000032000000320001003100000031007C
:100DB0000000310001003000000030000000300071
:100DC00001002F0000002F0000002F0000002F0066
:100DD00001002E0000002E0000002E0001002D005A
:100DE00000002D0000002D0000002D0001002C004F
:100DF00000002C0000002C0000002C0001002B0043
:100E000000002B0000002B0000002B0001002A0036
:100E100000002A0000002A0000002A00010029002A
:100E2000000029000000290000002900000029001E
:100E30000100280000002800000028000000280011
:100E40000000280001002700000027000000270004
:100E500000002700000027000100260000002600F7
:100E600000002600000026000000260001002500EA
:100E700000002500000025000000250000002500DE
:100E800000002500010024000000240000002400D0
:100E900000002400000024000100230000002300C3
:100EA00000002300000023000000230000002300B6
:100EB00000002300010022000000220000002200A8
:100EC000000022000000220000002200010021009A
:100ED000000021000000210000002100000021008E
:100EE000000021000000210001002000000020007F
:100EF0000000200000002000000020000000200072
:100F0000000020000000200001001F0000001F0062
:100F100000001F0000001F0000001F0000001F0055
:100F200000001F0001001E0000001E0000001E0047
:100F300000001E000000043700001E290000511BA5
:100F400000005810000010090000CC0400007802D6
:100F5000000041010000526573656E643A20002074
:100F600042002050006F6B004B494C4C45442E20F2
:100F7000004B494C4C206361757365642062792095
:100F8000746F6F206D75636820696E616374697634
:100F9000652074696D65202D2063757272656E74AD
:100FA00020636F6D6D616E643A2000506C656173F3
:100FB00065207265736574005052494E5445522045
:100FC00048414C544544005072696E746572206803
:100FD000616C7465642E206B696C6C2829206361D8
:100FE0006C6C6564210A00656E7175657565696E66
:100FF0006720220000000000000000000000000048
:10100000000048420000484200004040000000004C
:101010005761726E696E673A20486F6D696E67201E
:1010200042756D702044697669736F72203C20317F
:101030000A000202040000A0400000A040000000DE
:10104000400000904300008A4300007A43FFFFFF06
:10105000496E736572742066696C616D656E74208B
:10106000616E6420707265737320627574746F6E44
:1010700020286F72204D313038290A00002F2F614F
:101080006374696F6E3A726573756D650A004D36EB
:1010900030303A20546F6F20636F6C6400486F7477
:1010A000656E6420746F6F20636F6C640A002F2F6D
:1010B000616374696F6E3A70617573650A002575B6
:1010C0003A2530327500253032753A2530327500B8
:1010D00025756420253032753A25303275000006BA
:1010E0000900FE000000000001090008FE000005E4
:1010F000080806000040F0C888889878100508089D
:10110000060000C0F88888888888F805050506006C
:10111000012030F830200508080600002070F82073
:10112000202020E00509090600FF2070A8A8B88843
:101130008870200509090600FFE080C0B0A82830AB
:1011400028280509090600FFF8A88888888888A843
:10115000F8050A0A0600FE205050505088A8A888BA
:101160007003030306000340A04000060900FE07C9
:1011700001920321207FFF07FF07FF000000060008
:101180000001070706020080808080800080030243
:1011900002060105A0A00507070600005050F85000
:1011A000F850500507070600002078A07028F020AE
:1011B000050707060000C0C810204098180507075B
:1011C0000600006090A040A8906802030306010496
:1011D000C040800307070601002040808080402037
:1011E00003070706010080402020204080050505F8
:1011F00006000120A870A820050505060001202092
:10120000F820200203030602FFC04080050101060A
:101210000003F8020202060200C0C0050505060030
:1012200001081020408005070706000070888888A4
:1012300088887003070706010040C040404040E036
:10124000050707060000708808708080F80507070A
:10125000060000F81020100808F005070706000037
:1012600010305090F81010050707060000F880F0C5
:1012700008088870050707060000708080F08888DD
:1012800070050707060000F8081020202020050739
:1012900007060000708888708888700507070600B8
:1012A0000070888878080870020505060200C0C032
:1012B00000C0C00206060602FFC0C000C040800495
:1012C0000707060000102040804020100503030699
:1012D0000002F800F80407070601008040201020F3
:1012E00040800507070600007088081020002005D0
:1012F000070706000070880868A8A8700507070699
:101300000000708888F8888888050707060000F0C4
:101310008888F08888F005070706000070888080BC
:10132000808870050707060000F08888888888F0A4
:10133000050707060000F88080F08080F8050707A1
:10134000060000F88080F080808005070706000016
:10135000708880B88888700507070600008888882C
:10136000F8888888010707060200808080808080D6
:101370008005070706000038101010109060050760
:10138000070600008890A0C0A09088050707060007
:1013900000808080808080F805070706000088D8DC
:1013A000A8888888880507070600008888C8A89844
:1013B0008888050707060000708888888888700577
:1013C0000707060000F08888F08080800507070680
:1013D000000070888888A89068050707060000F05C
:1013E0008888F0A090880507070600007880807044
:1013F0000808F0050707060000F82020202020201C
:101400000507070600008888888888887005070710
:101410000600008888888888502005070706000095
:101420008888888888A850050707060000888850A3
:1014300020508888050707060000888888502020EB
:1014400020050707060000F80810204080F8030771
:1014500007060100E08080808080E0050505060029
:10146000018040201008030707060100E02020202B
:101470002020E00503030600042050880501010632
:101480000000F8020202060205804005050506007C
:101490000070087888780507070600008080B0C8CB
:1014A0008888F005050506000070808088700507B3
:1014B0000706000008086898888878050505060072
:1014C000007088F880700507070600003048E0408B
:1014D0004040400506060600FF70888878087005C1
:1014E00007070600008080B0C888888801070706C3
:1014F0000200800080808080800308080601FF20B1
:101500000020202020A040040707060000808090D3
:10151000A0C0A090030707060100C0404040404023
:10152000E0050505060000D0A8A8A8A80505050641
:101530000000B0C888888805050506000070888806
:1015400088700506060600FFF08888F08080050692
:10155000060600FF7888887808080505050600005B
:10156000B0C880808005050506000070807008F016
:101570000407070600004040E040404030050505F4
:101580000600008888889868050505060000888898
:101590008850200505050600008888A8A850050584
:1015A0000506000088502050880506060600FF88C2
:1015B0008888780870050505060000F8102040F8B6
:1015C0000307070601002040408040402001070734
:1015D000060200808080808080800307070601006B
:1015E00080404020404080050202060002689000D2
:1015F00000000600005A00590058000920000000B1
:10160000000000000000000000003FFFF0000000AC
:101610000000000000000000003800700000000022
:10162000000000000000000030FC3000000000005E
:101630000000000000000020FC100000000000007E
:1016400000000000000020781000000000000000F2
:10165000000000000020301000000000000000002A
:10166000000000002C00D03FC0000000000000007F
:101670002082002E31D07FE000000000000000102A
:1016800041002F7BD07FE0000000000000001041EF
:10169000002F7BD07FE000000000000000208200CF
:1016A0002E31D03FC0000000000000004104002C9B
:1016B00000D03FC000000000000000820800203081
:1016C000107FE00000000000000082080020781079
:1016D0007FE00000000000000041040020FC107FBB
:1016E000E00000000000000020820030FC301F807D
:1016F000000000000000000000003800700F000033
:10170000000000000000FFFFC03FFFF006000000E7
:101710000000000000FFFFC000000000000000000B
:10172000000000000000003FFFF00000000000008B
:101730000000000000003800700000000000000001
:1017400000000000003186300000000000000000B2
:1017500000000000238710000000000000000000CF
:10176000000000278790000000000000000000003B
:1017700000002F87D00000000000000000000000E3
:10178000002F03D03FC000000000000000208200B6
:101790002030107FE0000000000000001041002019
:1017A00078107FE000000000000000104100207869
:1017B000107FE000000000000000208200203010B8
:1017C0003FC0000000000000004104002F03D03F94
:1017D000C0000000000000008208002F87D07FE0DA
:1017E000000000000000008208002787907FE000D2
:1017F0000000000000004104002387107FE000008B
:1018000000000000002082003186301F80000000B0
:10181000000000000000003800700F000000000011
:10182000000000FFFFC03FFFF006000000000000C6
:101830000000FFFFC00000001000C90210012C01D1
:101840004001220170011801B0010E01F0010401F4
:101850005002FA00B002F0003003E600D003DC00D2
:101860009004D2007005C800A006BE000008B400B5
:10187000B009AA00D00BA000600E960060118C0089
:101880000015820020197800C01D6E00A02264009F
:10189000B0275A00902C500000314600E0343C0044
:1018A00010383200903A2800603C1E00A03D140021
:1018B000803E0A00203F00006265640A002C20730D
:1018C000797374656D2073746F707065642120483E
:1018D00065617465725F49443A200042656420681E
:1018E000656174696E67206661696C65640048654E
:1018F0006174696E67206661696C656400453120BA
:1019000048656174696E67206661696C656400484A
:10191000656174696E67206661696C6564004B4936
:101920004C4C45442E20001000AD0330016A01509C
:10193000022B0170030A019004F500B005E500D008
:1019400006D800F007CE001009C500300ABE0050CE
:101950000BB700700CB100900DAB00B00EA600D01C
:101960000FA200F0109D0010129900301395005046
:1019700014920070158E0090168B00B0178700D05F
:10198000188400F0198100101B7E00301C7B005071
:101990001D7900701E7600901F7300B0207000D07B
:1019A000216E00F0226B0010246900302566005083
:1019B0002663007027610090285E00B0295C00D08B
:1019C0002A5900F02B5600102D5400302E51005093
:1019D0002F4E0070304B0090314800B0324500D09F
:1019E000334200F0343E0010363B003037370050B1
:1019F00038330070392E00903A2900B03B2300D0D4
:101A00003C1B00F03D1100103F0100F03F0000457D
:101A100031204572723A204D415854454D50004591
:101A200072723A204D415854454D50204245440071
:101A30004D415854454D5020747269676765726511
:101A400064004531204572723A204D494E54454D4F
:101A500050004572723A204D494E54454D50204237
:101A60004544004D494E54454D5020747269676796
:101A700065726564004D383420582059205A20453D
:101A800000202F002042403A0020403A004D696378
:101A9000726F737465707320756E617661696C61C5
:101AA000626C650A0045313A200045303A20005A00
:101AB0003A2000593A2000583A20004D53312C4D1D
:101AC00053322050696E730A004572726F7220772C
:101AD000726974696E6720746F20454550524F4D8E
:101AE000210A004E6F20436865636B73756D207724
:101AF000697468206C696E65206E756D6265722C04
:101B0000204C617374204C696E653A200053544F29
:101B1000505045442E20005072696E7465722073D7
:101B2000746F707065642064756520746F206572D1
:101B3000726F72732E204669782074686520657212
:101B4000726F7220616E6420757365204D3939396A
:101B500020746F20726573746172742E202854652E
:101B60006D7065726174757265206973207265733A
:101B700065742E20536574206974206166746572E3
:101B80002072657374617274696E67290A004E6F02
:101B900020436865636B73756D2077697468206C8A
:101BA000696E65206E756D6265722C204C61737470
:101BB000204C696E653A2000636865636B73756DD0
:101BC000206D69736D617463682C204C617374209F
:101BD0004C696E653A20004C696E65204E756D62E9
:101BE0006572206973206E6F74204C617374204C91
:101BF000696E65204E756D6265722B312C204C61CB
:101C00007374204C696E653A20004D313130004DBF
:101C100033310053442072656164206572726F72C3
:101C20000A00446F6E65207072696E74696E672079
:101C300066696C650A0020496E76616C696420658E
:101C40007874727564657220000000000000000066
:101C500000000000000000904300008A4300007A6A
:101C60004347322F47332062616420706172616D97
:101C700065746572730A00486F6D65205859206657
:101C8000697273740A00486F6D652058592066693F
:101C900072737400001FFFFFFFFFFFFF6000000072
:101CA0000001FF400000000000FF80000000000075
:101CB0007F83CF00000C303F87FF80000C301F86F1
:101CC0007980000C000F8C30C7838C30E78C30CFCC
:101CD000C7CC31F38C30DCECEC33B98C30D86C6C85
:101CE00033198C30D06C0C33198C30D86C0C331900
:101CF0008C30DC6C0E3B198C30CF7C079F198C30FC
:101D0000C77C038F19400000000000026000000043
:101D10000000061FFFFFFFFFFFF82020506C616EE0
:101D20006E657242756666657242797465733A20B3
:101D3000002046726565204D656D6F72793A20000E
:101D4000436F6D70696C65643A2053657020313063
:101D500020323031380A00207C20417574686F725F
:101D60003A2028416C657068204F626A656374731D
:101D700020496E632E2C204C756C7A426F7420477C
:101D80006974205265706F7369746F7279290A00E3
:101D9000536570203130203230313831353A3434A7
:101DA0003A353300204C617374205570646174655A
:101DB000643A2000312E312E390A004D61726C696F
:101DC0006E0020536F66747761726520526573658B
:101DD000740A00205761746368646F6720526573EA
:101DE00065740A002042726F776E206F75742052FE
:101DF000657365740A002045787465726E616C20A5
:101E000052657365740A00506F77657255700A00E9
:101E100073746172740A006175746F25692E6700AE
:101E20006572726F722077726974696E6720746F61
:101E30002066696C650A00456E6473746F70732068
:101E4000256320256320256320256300205A3A005E
:101E500020593A0020583A00656E6473746F7073AD
:101E6000206869743A2000446F6E6520736176695A
:101E70006E672066696C652E0A004D323900473066
:101E80002058313730205932393020463330303005
:101E90000A4D313137205072696E742061626F7261
:101EA0007465642E000045787472756465642074EE
:101EB0006F74616C3A2000256C642E25696D0000FA
:101EC0004C6F6E67657374206A6F622074696D650C
:101ED0003A200000546F74616C207072696E742037
:101EE00074696D653A2000436F6D706C657465644C
:101EF0003A20005072696E7420436F756E743A20F8
:101F0000004D36303020423020542564004D3730AB
:101F10003120542564004D373032203B2564004D7C
:101F200037303220542564004368616E676520664F
:101F3000696C616D656E74005072656865617420CE
:101F4000437573746F6D00507265686561742043EA
:101F50007573746F6D0050726568656174204142DD
:101F600053005072656865617420504C41004D61AA
:101F7000696E005052494E5420504155534544001B
:101F8000554E4C4F41442046494C414D454E54001E
:101F90004C4F41442046494C414D454E54005075EC
:101FA000726765206D6F726500456E642066696CAE
:101FB000616D656E74206368616E67650000202046
:101FC0004E6F7A7A6C653A20006368616E676500CF
:101FD0006F66207468652066696C616D656E74005B
:101FE0005761697420666F72207374617274002087
:101FF000204E6F7A7A6C653A2000200066696C6129
:102000006D656E7420756E6C6F61640057616974E4
:1020100020666F720020204E6F7A7A6C653A20003D
:102020002000506C6561736520776169742E2E2ED7
:102030000048656174696E67206E6F7A7A6C65001E
:1020400020204E6F7A7A6C653A2000200068656126
:1020500074206E6F7A7A6C652E00507265737320EF
:10206000627574746F6E20746F0020204E6F7A7AE0
:102070006C653A2000746F20636F6E74696E7565CD
:102080002E2E2E00616E642070726573732062754F
:1020900074746F6E00496E736572742066696C614A
:1020A0006D656E740020204E6F7A7A6C653A200060
:1020B000200066696C616D656E74206C6F616400F0
:1020C0005761697420666F720020204E6F7A7A6CB7
:1020D000653A2000200066696C616D656E74207041
:1020E00075726765005761697420666F7200506C85
:1020F0006561736520776169742E000043617264C5
:102100002072656D6F766564004361726420696E4C
:102110007365727465640000060900FE0601890299
:10212000FE20FFFE07FE06FE000000060007010677
:1021300006060200808080800080030303060103FE
:10214000A0A0A00507070600FF5050F850F8505017
:102150000509090600FE2070A8A07028A8702006B6
:1021600008080600FF40A848102048540805070743
:102170000600FF60909060989068010303060203D8
:102180008080800207070602FF40808080808040B8
:102190000207070602FF80404040404080050505D9
:1021A0000600008850F8508805050506000020202C
:1021B000F820200204040602FEC040408005010110
:1021C000060002F8020202060200C0C0040606066B
:1021D0000100101020408080040606060100609077
:1021E0009090906003060606010040C0404040E029
:1021F0000406060601006090102040F00406060662
:102200000100F020601010E0050606060000103006
:102210005090F810040606060100F080E01010E06F
:102220000406060601006080E09090600406060641
:102230000100F010102040400406060601006090E6
:102240006090906004060606010060909070106037
:10225000020505060200C0C000C0C0020707060252
:10226000FEC0C000C04040800505050600001860A3
:10227000806018050303060001F800F8050505064F
:102280000000C0300830C00407070601006090104D
:10229000604000400506060600007090A8B08070FF
:1022A000050606060000205088F888880506060600
:1022B0000000F088F08888F00406060601006090AF
:1022C00080809060040606060100E090909090E007
:1022D000040606060100F080E08080F00406060691
:1022E0000100F080E0808080040606060100609016
:1022F00080B090600406060601009090F0909090E7
:10230000030606060100E040404040E005060606E0
:10231000000038101010906004060606010090A01E
:10232000C0A090900406060601008080808080F0A6
:1023300005060606000088D8A8A8888804060606B0
:10234000010090D0B09090900506060600007088BD
:1023500088888870040606060100E09090E080807E
:102360000407070601FF609090D0B06010040606D5
:10237000060100E09090E0909004060606010060DF
:102380009040209060050606060000F820202020DE
:1023900020040606060100909090909060040606C6
:1023A000060100909090F060600506060600008827
:1023B00088A8A8D888050606060000885020205066
:1023C000880506060600008888502020200406069E
:1023D000060100F010204080F0030606060100E030
:1023E00080808080E0040606060100808040201086
:1023F00010030606060100E020202020E00503036C
:102400000600032050880501010600FEF8020202C2
:1024100006020480400404040601007090907004D9
:1024200006060601008080E09090E00404040601A6
:1024300000708080700406060601001010709090F5
:102440007004040406010060B0C0700406060601B2
:1024500000205040E040400406060601FE609090D7
:102460007010600406060601008080E090909003E2
:1024700006060601004000C04040E00308080601CF
:10248000FE200060202020A04004060606010080F7
:1024900080A0C0A090030606060100C04040404056
:1024A000E0050404060000D0A8A88804040406017E
:1024B00000E0909090040404060100609090600495
:1024C00006060601FEE09090E08080040606060104
:1024D000FE709090701010040404060100A0D080DB
:1024E0008004040406010070C030E0040606060102
:1024F000004040E040502004040406010090909009
:102500007004040406010090906060050404060055
:102510000088A8A85004040406010090606090049C
:1025200006060601FE909090709060040404060177
:1025300000F02040F00307070601002040408040E3
:1025400040200107070602FF808080808080800392
:102550000707060100804040204040800402020638
:10256000010350A0FFFFFFFFFFFFFFFFFFFFFFFF83
:10257000FFFFFFFFFFFFFFFFFFFFFFFFFFFFFFFF6B
:10258000FFFFFFFFFF00000006000701060606022E
:10259000008000808080800406060601FF2070A075
:1025A000A070200507070600FF304840F04040F8C3
:1025B000050505060000A8508850A8050606060077
:1025C000008850F820F8200107070602FF8080806D
:1025D000008080800407070601FF70806090601013
:1025E000E0030101060105A0060707060000788444
:1025F00094A494847803050506010160A06000E0BE
:102600000505050600002850A05028040303060114
:1026100000F01010040101060102F0060707060091
:10262000007884B4A4A48478040101060105F004B0
:1026300003030601026090600507070600FF2020E3
:10264000F8202000F803050506010140A02040E025
:10265000030505060101C0204020C0020202060257
:102660000440800405050601FF9090B0D080050667
:102670000606000078E8E868282801010106020241
:10268000800202020602FE408003050506010140A9
:10269000C04040E003050506010140A04000E00500
:1026A0000505060000A0502850A00508080600FFF8
:1026B00040C04050703078100508080600FF40C048
:1026C0004050680810380508080600FFC020403058
:1026D000F030781004070706010020002060809089
:1026E0006005070706000040202050708888050715
:1026F0000706000010202050708888050707060094
:1027000000205020507088880507070600002850D8
:102710002050708888050707060000500020507080
:10272000888805070706000020502050708888051B
:10273000060606000078A0F0A0A0B804080806016C
:10274000FE609080809060204004070706010040F2
:1027500020F080E080F00407070601002040F080B0
:10276000E080F00407070601002050F080E080F0D0
:102770000407070601005000F080E080F00307071F
:102780000601008040E0404040E0030707060100EA
:102790002040E0404040E003070706010040A0E081
:1027A000404040E0030707060100A000E040404031
:1027B000E00506060600007048E848487004070770
:1027C00006010050A090D0B09090040707060100C9
:1027D0004020609090906004070706010020406050
:1027E0009090906004070706010020506090909040
:1027F0006004070706010050A060909090600407F5
:1028000007060100500060909090600505050600E5
:102810000088502050880408080601FF1070B0B0EE
:10282000D0D0E080040707060100402090909090EF
:102830006004070706010020409090909060040714
:102840000706010020509090909060040707060151
:10285000005000909090906005070706000010203F
:10286000885020202004060606010080E09090E0B9
:10287000800406060601006090A0A090A00407074F
:1028800006010040200070909070040707060100C8
:10289000204000709090700407070601002050004F
:1028A0007090907004070706010050A0007090908F
:1028B000700406060601005000709090700407072F
:1028C000060100205020709090700504040600005E
:1028D00070A8B0780406060601FE70808070204063
:1028E00004070706010040200060B0C0700407071D
:1028F00006010020400060B0C07004070706010018
:1029000020500060B0C07004060606010050006050
:10291000B0C070030707060100804000C04040E0DF
:10292000030707060100204000C04040E0030707FE
:1029300006010040A000C04040E00306060601007A
:10294000A000C04040E0040707060100306010709E
:1029500090906004070706010050A000E09090905E
:1029600004070706010040200060909060040707FC
:1029700006010020400060909060040707060100F7
:102980002050006090906004070706010050A000EE
:102990006090906004060606010050006090906010
:1029A0000505050600002000F800200404040601C7
:1029B0000070B0D0E00407070601004020009090AE
:1029C000907004070706010020400090909070046A
:1029D000070706010020500090909070040606063C
:1029E00001005000909090700409090601FE2040FB
:1029F000009090907090600408080601FE8080E0CE
:102A00009090E080800408080601FE5000909090AD
:102A1000709060022569730025696D202569730037
:102A20002569682025696D20256973002569642062
:102A30002569682025696D2025697300256979203D
:102A4000256964202569682025696D202569730042
:102A5000486F6D696E67206661696C656400010589
:102A60000800FF060121023520FFFF07FF06FF09CE
:102A70000050221656808080800080153353A0A01D
:102A8000A00257575050F850F85050025757207036
:102A9000A07028702013355580A040A02002475711
:102AA00040A0A040A0A0502513538080801226563D
:102AB0004080808080401226568040404040800206
:102AC00045559060F060900255552020F820201167
:102AD0003353604080044151F011335340E04002D1
:102AE000465610102040808012365640A0A0A0A06C
:102AF0004012365640C0404040E0024656609010BA
:102B00006080F0024656F020601090600246562029
:102B100060A0F02020024656F080E010906002464F
:102B2000566080E0909060024656F01020204040B1
:102B30000246566090609090600246566090907099
:102B40001060122555C0C000C0C01136566060002C
:102B5000604080123656204080804020034353F06E
:102B600000F012365680402020408012365640A099
:102B700020400040015858304898A8A890403002A2
:102B80004656609090F09090024656E090E090900B
:102B9000E0024656609080809060024656E0909039
:102BA0009090E0024656F080E08080F0024656F0B9
:102BB00080E0808080024656609080B0906002463F
:102BC000569090F0909090123656E040404040E091
:102BD00002465670202020A04002465690A0C0A079
:102BE000A0900246568080808080F002465690F089
:102BF000F090909002465690D0F0B0B090024656B9
:102C0000609090909060024656E09090E080800145
:102C10004757609090D0B06010024656E09090E028
:102C20009090024656609040209060123656E040E8
:102C30004040404002465690909090906002465628
:102C4000909090906060024656909090F0F09002C4
:102C5000465690906060909002565688885020208A
:102C600020024656F010204080F0123656E0808058
:102C70008080E0024656808040201010123656E0D8
:102C800020202020E016325240A0014151F01622AF
:102C9000528040024454709090700246568080E00A
:102CA0009090E0123454608080600246561010709C
:102CB00090907002445460B0C0600246562050406C
:102CC000E04040014555609070106002465680809B
:102CD000E09090901236564000C04040E0113757C7
:102CE0002000202020A040024656808090E0909056
:102CF000123656C040404040E0025454D0A8A8A824
:102D0000024454E0909090024454609090600145D9
:102D100055E090E08080014555709070101002449D
:102D200054A0D0808012345460C020C00246564067
:102D300040E040502002445490909070123454A0CF
:102D4000A0A04002545488A8A85002445490606047
:102D5000900145559090709060024454F02040F0EE
:102D6000024757304020C0204030221656808080D5
:102D7000808080024757C02040304020C006425229
:102D800050A0FFFFFFFFFFFFFFFFFFFFFFFFFFFF61
:102D9000FFFFFFFFFFFFFFFFFFFFFFFFFFFFFFFF43
:102DA000FFFFFF09005022165680008080808001BE
:102DB00046562070A0A070200246562050E0405099
:102DC000A002555588705070880256568850F820D9
:102DD000F82022175780808000808080024757703B
:102DE00080E0907010E0173151A002565670A8C8CC
:102DF000C8A87014355560A06000E003435350A08C
:102E000050123353E02020143151E002565670E83E
:102E1000D8E8D870173151E015335340A04012352F
:102E20005540E04000E014355540A02040E0143506
:102E300055C020C020C016225240800145559090B8
:102E400090E08002565678E8E868282824115180DE
:102E5000112252408014355540C04040E014355591
:102E600040A04000E0034353A050A0024757808099
:102E700080A060F0200247578080A0D01020700210
:102E8000475780408060A0F02012365640004080B6
:102E9000A04002475740206090F090900247572092
:102EA000406090F0909002475760906090F0909052
:102EB00002475750A06090F09090024757900060F2
:102EC00090F0909002475760906090F0909002468A
:102ED0005670A0A0F0A0B00147576090808090602D
:102EE000400247574020F080E080F00247572040E2
:102EF000F080E080F00247576090F080E080F002C0
:102F000047579000F080E080F01237578040E04053
:102F10004040E01237572040E0404040E012375731
:102F200040A0E0404040E0123757A000E040404061
:102F3000E00256567048E848487002475750A09043
:102F4000D0B0909002475740206090909060024728
:102F5000572040609090906002475760906090903A
:102F6000906002475750A060909090600247579041
:102F7000006090909060123353A040A002465670BB
:102F8000B0B0D0D0E00247574020909090906002BF
:102F900047572040909090906002475760909090E3
:102FA0009090600247579000909090906002575721
:102FB0001020885020202002465680E09090E0802B
:102FC0000246566090A0A090A00247574020007093
:102FD00090907002475720400070909070024757C1
:102FE0002050007090907002475750A00070909051
:102FF0007002465650007090907002475760906083
:1030000070909070025454F068B07811355560801B
:1030100080604002475740200060B0C060024757C0
:1030200020400060B0C06002475760900060B0C0B0
:1030300060024656500060B0C060123757804000B2
:10304000C04040E0123757204000C04040E01237F7
:103050005740A000C04040E0123656A000C040409B
:10306000E0024757A040A01070906002475750A060
:1030700000E09090900247574020006090906002DE
:103080004757204000609090600247576090006072
:1030900090906002475750A00060909060024656A2
:1030A0009000609090601235554000E0004002446E
:1030B0005470B0D0E00247574020009090907002CA
:1030C00047572040009090907002475760900090C2
:1030D0009090700246569000909090700148582051
:1030E000400090907090600147578080E090E080B1
:1030F000800147579000909070906001050700FE96
:103100000500FB01F220FFFE05FE05FE0200400265
:1031100015258080800080053242A0A002556550B0
:10312000F850F8500146562070C030E02002556536
:103130009010204048025565608068906805122212
:1031400080800225354080808040022535804040C7
:103150004080043343A040A003334340E0400122B9
:10316000324080043141E00211218002556508108F
:103170002040800245556090909060022535C04007
:10318000404040024555E0106080F0024555E01097
:103190006010E00245552060A0F020024555F08007
:1031A000E010E00245556080E09060024555F01067
:1031B0002040400245556090609060024555609007
:1031C000701060031323800080021424800080802C
:1031D0000235452040804020033343E000E00235C3
:1031E000458040204080024555E010600040025577
:1031F000657088B8A870024555609090F0900245BF
:1032000055E090E090E002354560808080600245A6
:1032100055E0909090E0023545E080E080E0023596
:1032200045E080E080800245557080B09070024596
:10323000559090F09090023545E0404040E00245C6
:1032400055301010906002455590A0C0A0900235F6
:103250004580808080E002556588D8A8888802452E
:103260005590D0B090900245556090909060024586
:1032700055E09090E080014656609090906010027A
:103280004555E09090E09002455570806010E00256
:103290003545E04040404002455590909090600296
:1032A00045559090A0A04002556588A8A8A8500256
:1032B0004555909060909002455590907010600236
:1032C0003545E0204080E0022535C0808080C00286
:1032D00055658040201008022535C0404040C0059B
:1032E000324240A0024151F0052232804002445453
:1032F0007090907002455580E09090E002344460F8
:10330000808060024555107090907002445460B007
:10331000C0600235452040E0404000465670909025
:1033200070106002455580E0909090021525800055
:103330008080800027374000404040408002455553
:103340008090A0E0900215258080808080025464E7
:10335000F0A8A8A8024454E09090900244546090D1
:103360009060004656E09090E08080004656709055
:1033700090701010023444A0C0808002445470C089
:1033800030E002354540E0404020024454909090A7
:10339000700244549090A040025464A8A850500277
:1033A0003444A04040A000465690909070106002B7
:1033B0004454F02040F002354560408040600215E2
:1033C000258080808080023545C0402040C0054275
:1033D0005250A0FFFFFFFFFFFFFFFFFFFFFFFFFFB8
:1033E000FFFFFFFFFFFFFFFFFFFFFFFFFFFFFFFFED
:1033F000FFFFFFFF020040FFFFFFFFFFFFFFFFFF98
:10340000FFFFFFFFFFFFFFFFFFFFFFFFFFFFFFFFCC
:10341000FFFFFFFFFFFFFFFFFFFFFFFFFFFFFFFFBC
:10342000FFFFFFFFFFFFFFFFFFFFFFFFFFFFFFFFAC
:10343000FFFFFFFFFFFFFFFFFFFFFFFFFFFFFFFF9C
:10344000FFFFFFFFFFFFFFFFFFFFFFFFFFFFFFFF8C
:10345000FFFFFFFFFFFF01060D00FE09016602D618
:1034600020FFFE0BFE0AFE0D00602219698080809D
:10347000808080800080183363A0A0A0035767502D
:1034800050F850F850500259692078A0A0702828B0
:10349000F02002596948A85010204050A8900258C6
:1034A0006840A0A040A09890682813638080801195
:1034B0003B6B2040408080808080404020113B6BEF
:1034C000804040202020202040408006556520A8D4
:1034D00070A8200455652020F82020113363604037
:1034E00080065161F811336340E0400259690808D1
:1034F00010102040408080025969205088888888B8
:103500008850200259692060A02020202020F80245
:1035100059697088880810204080F8025969F808B5
:1035200010207008088870025969101030505090AF
:10353000F81010025969F88080B0C8080888700235
:10354000596970888080F088888870025969F80805
:103550001010202040404002596970888888708887
:10356000888870025969708888887808088870117E
:10357000386840E040000040E04011386840E040DA
:1035800000006040800259690810204080402010EF
:1035900008045464F80000F80259698040201008BB
:1035A000102040800259697088880810202000206F
:1035B00002596970888898A8A8B080780259692053
:1035C00050888888F8888888025969F04848487087
:1035D000484848F0025969708880808080808870EF
:1035E000025969F048484848484848F0025969F883
:1035F000808080F0808080F8025969F8808080F0B7
:103600008080808002596970888080809888887066
:1036100002596988888888F888888888123969E01A
:1036200040404040404040E00259693810101010BE
:1036300010109060025969888890A0C0A090888876
:103640000259698080808080808080F80259698872
:1036500088D8A8A88888888802596988C8C8A8A86E
:1036600098988888025969708888888888888870BE
:10367000025969F0888888F080808080015A6A70D9
:10368000888888888888A87008025969F08888889E
:10369000F0A0908888025969708880807008088836
:1036A00070025969F820202020202020200259692A
:1036B0008888888888888888700259698888888876
:1036C000505050202002596988888888A8A8A8A846
:1036D0005002596988885050205050888802596992
:1036E000888850502020202020025969F8081010A6
:1036F00020404080F8113B6BE0808080808080809B
:103700008080E00259698080404020101008081134
:103710003B6BE0202020202020202020E008536365
:10372000205088015161F82A22628040025666705A
:103730000878889868025969808080F0888888882D
:10374000F0025666708880808870025969080808FF
:103750007888888888780256667088F88088700231
:10376000596930484040F0404040400058687088F7
:10377000888878088870025969808080B0C88888F5
:1037800088881238684000C040404040E0004A6AE3
:1037900010003010101010909060025969808080E5
:1037A00090A0C0A09088123969C04040404040407D
:1037B00040E0025666D0A8A8A8A888025666B0C8FD
:1037C000888888880256667088888888700058685B
:1037D000F0888888F08080800058687888888878A9
:1037E000080808025666B0C880808080025666705D
:1037F00088601088700258684040F040404048306F
:103800000256668888888898680256668888885034
:1038100050200256668888A8A8A85002566688508C
:103820002020508800586888888898680888700226
:103830005666F810204080F8015B6B18202020208D
:10384000C0202020201822196980808080808080FC
:103850008080015B6BC0202020201820202020C009
:1038600008536348A890FFFFFFFFFFFFFFFFFFFF24
:10387000FFFFFFFFFFFFFFFFFFFFFFFFFFFFFFFF58
:10388000FFFFFFFFFFFFFF0D00602219698000802E
:103890008080808080800358682070A8A0A0A870D5
:1038A0002002596930484040E0404048B003566625
:1038B00088705050708802596988885050F820F8F4
:1038C0002020221969808080800080808080124AB8
:1038D0006A609080609090601090601A3262A0A040
:1038E0000359697088A8D8C8D8A888700457677029
:1038F0000878887800F80356662850A0A05028045D
:103900005363F80808163161E00359697088E8D8F4
:10391000D8E8D888700A5161F817446460909060C4
:103920000357672020F8202000F807356540A020C5
:1039300040E007356540A04020C02A226240800058
:1039400058688888888898E8808002596978E8E80B
:10395000E8E868282828262161C0202262408007E4
:10396000356540C04040E004576770888888700023
:10397000F8035666A050282850A0025A6A40C0405A
:1039800040E00818283808025A6A40C04040E01059
:1039900028081038025A6A40A04020A04818283849
:1039A00008025969200020204080888870025A6AE5
:1039B00040200020508888F88888025A6A10200029
:1039C00020508888F88888025A6A30480020508839
:1039D00088F88888025A6A28500020508888F88819
:1039E00088025A6A50500020508888F88888025A05
:1039F0006A20502020508888F8888802596958A089
:103A0000A0A0B0E0A0A0B8005B6B70888080808030
:103A10008088702040025A6A402000F88080F08040
:103A200080F8025A6A102000F88080F08080F80246
:103A30005A6A304800F88080F08080F8025A6A5054
:103A40005000F88080F08080F8123A6A804000E0F0
:103A50004040404040E0123A6A204000E040404090
:103A60004040E0124A6A609000E04040404040E040
:103A7000123A6AA0A000E04040404040E00259698C
:103A8000F0484848E8484848F0025A6A28500088F8
:103A900088C8A8988888025A6A4020007088888858
:103AA000888870025A6A1020007088888888887018
:103AB000025A6A30480070888888888870025A6A7A
:103AC00028500070888888888870025A6A50500090
:103AD00070888888888870035565885020508801D0
:103AE0005B6B08709898A8A8A8C8C87080025A6A2A
:103AF00040200088888888888870025A6A102000D0
:103B000088888888888870025A6A3048008888883F
:103B100088888870025A6A50500088888888888807
:103B200070025A6A102000888850202020200259F4
:103B30006980F0888888F080808002596960909060
:103B4000A0A0908888B00259694020007008788849
:103B5000986802596910200070087888986802599E
:103B600069304800700878889868025969285000C0
:103B700070087888986802596950500070087888F1
:103B80009868025A6A30483000700878889868024D
:103B90005666702870A0A850005868708880808889
:103BA0007020400259694020007088F880887002B7
:103BB00059691020007088F880887002596930486F
:103BC000007088F88088700259695050007088F839
:103BD000808870123969804000C040404040E01247
:103BE0003969204000C040404040E012496960907F
:103BF00000C040404040E0123969A0A000C04040F1
:103C00004040E0025A6A50206010708888888870AE
:103C1000025969285000B0C88888888802596940CC
:103C20002000708888888870025969102000708888
:103C30008888887002596930480070888888887040
:103C40000259692850007088888888700259695024
:103C50005000708888888870035767202000F8001B
:103C60002020015868087098A8A8C8708002596977
:103C70004020008888888898680259691020008848
:103C800088888898680259693048008888888898A8
:103C900068025969505000888888889868005B6B72
:103CA0001020008888889868088870005A6A808088
:103CB000B0C88888C8B08080005B6B50500088888E
:103CC000889868088870000000000000000000006C
:103CD00000000000000000000000000000000000E4
:103CE0000000000000000000000C000000000000C8
:103CF000000C0000000000000012000000000000A6
:103D0000002300000000000000210000000000006F
:103D1000004C800000000000005E800000000000F9
:103D2000009240000000000000A1400000000000E0
:103D30000121200000000000027F90000000000030
:103D4000020010000000000007FFF8000000000063
:103D5000040008000000000008000400000000004B
:103D60000800060000000000100002000000000033
:103D7000301E010000000000207F810000000000D4
:103D800041FFE0800000000043FCF08000000000E4
:103D9000873B7840000000018EDBFC6000000001E2
:103DA0000FEBCC20000000021FEDB6100000000257
:103DB0001FDEB6100000000439CD7F0800000004AB
:103DC00036E0FF08000000087EC0BB840000001839
:103DD0007F005D86000000107FC0ED8200000020A3
:103DE0003CC07301000000203B337F0100000070E5
:103DF0001BE77E03800000C81DEEDE04C0000088C3
:103E00000FDEDC04400001240FDF3C092000012606
:103E100007DBF8192000027203E7F013900002514B
:103E200001FFE02290000489007F802448000904FB
:103E3000801E004824000BFE400000DFF40010004C
:103E40004000008002001FFFFFFFFFFFFE00000098
:103E50000000000000000000000000000000000062
:103E60000000000000001022103C3C0E1F00102239
:103E70001004221104001022100822110400102244
:103E800010083C110400102210102211040010220E
:103E90001020221104001E1C1E3C3C0E04000000D9
:103EA0000000000000000000000000000000000012
:103EB0000000000000000000000000000000000002
:103EC00000000000000000000000000000000000F2
:103ED00000000000000000000000000000000000E2
:103EE00000000000000000000000000000000000D2
:103EF00000000000000000000000000000000000C2
:103F0000000000004D3234004D3233202573002074
:103F1000746F6F206C6F6E6720657874727573694B
:103F20006F6E2070726576656E7465640A0020633A
:103F30006F6C6420657874727573696F6E2070722F
:103F40006576656E7465640A000000200023002613
:103F50000029002C002F00320000010000030106A0
:103F600001090146696C652064656C657465643A95
:103F70000044656C6574696F6E206661696C656488
:103F80002C2046696C653A200046696C616D656E4F
:103F90007420757365643A200053746174733A2019
:103FA000002C204C6F6E67657374206A6F623A2034
:103FB00000546F74616C2074696D653A200053740D
:103FC0006174733A20002C204661696C65643A2064
:103FD000002C2046696E69736865643A200050724F
:103FE000696E74733A200053746174733A20004D03
:103FF00031343520533C696E6465783E206F7574AA
:10400000206F662072616E67652028302D31290A85
:10401000004C756C7A426F742054415A2035204F01
:1040200066662E00205A3A0020593A0020436F75E8
:104030006E7420583A0020453A00205A3A00205920
:104040003A00583A003A004361703A0054484552E9
:104050004D414C5F50524F54454354494F4E0041DF
:1040600055544F5245504F52545F53445F5354413F
:1040700054555300454D455247454E43595F5041B5
:104080005253455200434153455F4C494748545FA2
:104090004252494748544E45535300544F47474CAA
:1040A000455F4C494748545300534F46545741527B
:1040B000455F504F574552004255494C445F50456B
:1040C0005243454E54004C4556454C494E475F447B
:1040D000415441005A5F50524F4245004155544FA0
:1040E0004C4556454C005052494E545F4A4F420091
:1040F00050524F4752455353004155544F5245502B
:104100004F52545F54454D5000564F4C554D4554F9
:1041100052494300454550524F4D00534552494185
:104120004C5F584F4E5F584F4646004649524D57D8
:104130004152455F4E414D453A4D61726C696E206A
:10414000204649524D574152455F56455253494FBB
:104150004E3A312E312E392E313620455854525593
:104160004445525F545950453A4D4F415273747211
:104170007564657220534F555243455F434F444524
:104180005F55524C3A68747470733A2F2F636F64A2
:10419000652E616C6570686F626A656374732E6307
:1041A0006F6D2F646966667573696F6E2F4D41522E
:1041B0004C494E2050524F544F434F4C5F5645523E
:1041C00053494F4E3A312E30204D414348494E45D8
:1041D0005F545950453A4C756C7A426F7420544183
:1041E0005A20352045585452554445525F434F5547
:1041F0004E543A3120555549443A6333323535638C
:1042000039362D343039372D343838342D3865640B
:10421000302D6465643266663962616536310A0044
:104220002F2F20006F70656E206661696C65642CAD
:104230002046696C653A200043616E6E6F74206F92
:1042400070656E2073756264697220006563686FC3
:104250003A00453120544845524D414C2052554E6C
:10426000415741590042454420544845524D414C24
:104270002052554E4157415900546865726D616C2A
:104280002052756E617761790000002200250028B8
:10429000002B002E0031003400020100000501084F
:1042A000010B0100002100240027002A002D00300E
:1042B00000330001010000040107010A01050505A2
:1042C00005070508080808020202020A0A0808048D
:1042D00004040401010101010101010303030303BB
:1042E000030303040707070C0C0C0C0C0C0C0C024A
:1042F00002020206060606060606060B0B0B0B0B51
:104300000B0B0B0102102020080810204010204049
:104310008002010201080402010102040810204089
:1043200080804020100804020180040201804020A7
:1043300010080402010804020101020408102040D0
:10434000800102040810204080454550524F4D2006
:104350006461746173697A65206572726F722E0A86
:1043600000290A002062797465733B206372632020
:104370000053657474696E67732053746F7265645B
:10438000202800290A002062797465733B2063723B
:104390006320002073746F726564207365747469A0
:1043A0006E67732072657472696576656420280093
:1043B000202863616C63756C6174656429210A004F
:1043C00020213D2000454550524F4D20435243206F
:1043D0006D69736D61746368202D202873746F722A
:1043E00065642920002053697A653A2000496E648B
:1043F00065783A2000204D61726C696E3D56353506
:10440000290A0028454550524F4D3D004545505220
:104410004F4D2076657273696F6E206D69736D61A3
:1044200074636820007C3C3E5E2B3D3F2F5B5D3B10
:104430002C2A225C00457874727564657220004DE8
:104440006F7665205A004D6F76652059004D6F7666
:10445000652058004D6F76656D656E7400436F6F13
:104460006C646F776E0046616E20737065656420C2
:10447000310046616E2073706565642031004265CD
:104480006400426564004E6F7A7A6C65004E6F7A04
:104490007A6C65004D61696E005654726176206DCC
:1044A000696E005654726176206D696E00565472C2
:1044B0006176206D696E00566D696E00566D696E8D
:1044C00000566D696E00566D6178204500566D612D
:1044D00078204500566D6178204500566D61782042
:1044E0005A00566D6178205A00566D6178205A0046
:1044F000566D6178205900566D6178205900566DCF
:104500006178205900566D6178205800566D6178A9
:10451000205800566D61782058004D6F74696F6E99
:1045200000416D6178204500416D61782045004172
:104530006D6178205A00416D6178205A00416D61AB
:1045400078205900416D6178205900416D617820D3
:104550005800416D6178205800412D747261766574
:104560006C00412D74726176656C00412D7265742A
:104570007261637400412D726574726163740041ED
:104580006363656C00416363656C004D6F74696FB4
:104590006E004D6F766520617869730044697361C0
:1045A000626C65207374657070657273004D383489
:1045B000004175746F20686F6D6500473238004D9B
:1045C00061696E004D3530320A4D353030004C6F28
:1045D00061642073657474696E67730052657374E7
:1045E0006F7265206661696C736166650053746FF4
:1045F00072652073657474696E67730041647661D7
:104600006E6365642053657474696E6773004D61F1
:10461000696E005072696E746572205374617473B0
:10462000004669726D776172652056657273696FB5
:104630006E004D61696E00466C6F7700466C6F7757
:104640000046616E20737065656420310046616EBE
:1046500020737065656420310042656400426564C2
:10466000004E6F7A7A6C65004E6F7A7A6C650053F3
:1046700070656564005370656564004D61696E0026
:104680004D6F76652058004D6F76652059004D6F4F
:104690007665205A00457874727564657220004D05
:1046A0006F766520302E316D6D004D6F766520314F
:1046B0006D6D004D6F76652031306D6D004D6F76FC
:1046C000652061786973004578747275646572203D
:1046D000004D6F7665205A004D6F76652059004D6C
:1046E0006F766520580056652D6A65726B005665B9
:1046F0002D6A65726B0056652D6A65726B00567A7D
:104700002D6A65726B00567A2D6A65726B00567958
:104710002D6A65726B0056792D6A65726B00567949
:104720002D6A65726B0056782D6A65726B0056783B
:104730002D6A65726B0056782D6A65726B004D6F3D
:1047400074696F6E004573746570732F6D6D0045ED
:1047500073746570732F6D6D005A73746570732F69
:104760006D6D005A73746570732F6D6D005973749D
:104770006570732F6D6D005973746570732F6D6D57
:10478000005873746570732F6D6D00587374657085
:10479000732F6D6D004D6F74696F6E004F6666000C
:1047A0004F6E2000456E6473746F702061626F728B
:1047B000740053746570732F6D6D004A65726B00E1
:1047C000416363656C65726174696F6E0056656CF8
:1047D0006F6369747900416476616E636564205328
:1047E000657474696E67730043616E6E6F742065E3
:1047F0006E746572207375626469723A2000022ECD
:104800002E004D61696E0053442063617264206F15
:104810006B0A006F70656E526F6F74206661696C11
:1048200065640A00766F6C756D652E696E6974201B
:104830006661696C65640A00534420696E6974207E
:104840006661696C0A0057726974696E6720746FDB
:104850002066696C653A20006F70656E206661693C
:104860006C65642C2046696C653A20006F70656E3B
:10487000206661696C65642C2046696C653A20008D
:1048800046696C652073656C65637465640A002015
:1048900053697A653A200046696C65206F70656ED1
:1048A00065643A20002066696C653A2000646F698F
:1048B0006E67006672657368004E6F772000454E24
:1048C0004420535542524F5554494E450A00222028
:1048D000706F73002220706172656E743A2200530B
:1048E0005542524F5554494E452043414C4C20743B
:1048F00061726765743A22004B494C4C45442E2046
:1049000000747279696E6720746F2063616C6C202B
:104910007375622D67636F64652066696C657320CB
:104920007769746820746F6F206D616E79206C6593
:1049300076656C732E204D4158206C6576656C2031
:1049400069733A004572726F723A0048617264632B
:104950006F6465642044656661756C74205365748A
:1049600074696E6773204C6F616465640A00282364
:104970000000282300006400000010270000000051
:10498000964300009643000040400000C8410000EC
:10499000C9420000C9420000C84400804F4420289A
:1049A0006D6D290020204D36303320002055004CFD
:1049B0000046696C616D656E74206C6F61642F7563
:1049C0006E6C6F6164206C656E677468733A0A0080
:1049D00020440020490020204D3330342050002056
:1049E000440020490020204D3330312050005049F0
:1049F000442073657474696E67733A0A0020460038
:104A000020420020480020204D3134352053004DF5
:104A10006174657269616C2068656174757020707D
:104A20006172616D65746572733A0A00205A0020E4
:104A3000590020204D323036205800486F6D6520D7
:104A40006F66667365743A0A00204500205A00209C
:104A5000590020580020540020530020204D3230AF
:104A60003520420020453C6D61785F655F6A657264
:104A70006B3E0020583C6D61785F785F6A65726BB1
:104A80003E20593C6D61785F795F6A65726B3E20AC
:104A90005A3C6D61785F7A5F6A65726B3E00416473
:104AA00076616E6365643A20423C6D696E5F736542
:104AB000676D656E745F74696D655F75733E2053D5
:104AC0003C6D696E5F66656564726174653E205415
:104AD0003C6D696E5F74726176656C5F6665656476
:104AE000726174653E0020540020520020204D3237
:104AF0003034205000416363656C65726174696F86
:104B00006E2028756E6974732F7332293A20503CD9
:104B10007072696E745F616363656C3E20523C72B3
:104B20006574726163745F616363656C3E20543CBD
:104B300074726176656C5F616363656C3E0A002028
:104B40004500205A0020590020204D323031205895
:104B5000004D6178696D756D20416363656C6572A8
:104B60006174696F6E2028756E6974732F733229B2
:104B70003A0A00204500205A0020590020204D32DA
:104B800030332058004D6178696D756D206665651C
:104B90006472617465732028756E6974732F73294C
:104BA0003A0A00204500205A0020590020204D39A3
:104BB0003220580053746570732070657220756ED2
:104BC00069743A0A0020204D3230302044300A0007
:104BD00020204D3230302044002044697361626CE3
:104BE00065640A0046696C616D656E742073657456
:104BF00074696E67733A0020204D313439204320A8
:104C00003B20556E69747320696E2043656C73692F
:104C100075730A002020473231202020203B004CB1
:104C2000756C7A626F742054415A20352072656128
:104C300064792E005072696E74696E672E2E2E0094
:104C40005072696E7420706175736564004D313205
:104C500035004D3234005072696E742061626F729B
:104C6000746564005072696E742066726F6D2053B3
:104C7000440053746F70207072696E7400526573D3
:104C8000756D65207072696E74004E6F20534420FC
:104C900063617264005061757365207072696E742F
:104CA0000041626F7574205072696E7465720043C2
:104CB00068616E67652066696C616D656E7400433E
:104CC00068616E67652066696C616D656E74004D24
:104CD00036303020423000436F6E6669677572610E
:104CE00074696F6E0054656D70657261747572657C
:104CF000004D6F76656D656E740054756E65004984
:104D00006E666F2073637265656E00556E6B6E6FB5
:104D1000776E20636F6D6D616E643A202200486F7C
:104D200074656E6420746F6F20636F6C640A00009A
:104D3000000A0B02090C0D0E080703040100000015
:104D40000000000000000000000000000000000063
:104D50000000000000000000000000121110000020
:104D60000000000000000000000000000000000043
:104D70000000000000486F6D6520257325732573C2
:104D8000206669727374002066697273740A005A2F
:104D90000059005800486F6D65200000D1BA0F50CF
:104DA00011241FBECFEFD1E2DEBFCDBF00E00CBFAC
:104DB00013E0A0E0B2E0E4EFF3E102E00BBF02C0D9
:104DC00007900D92A438B107D9F725E1A4E8B3E024
:104DD00001C01D92AB32B207E1F716E2CFECD6E28A
:104DE00000E006C021970109802FFE010F946B0996
:104DF000CE3CD10780E00807A9F70E949B7E0D9466
:104E0000E9090C9400002F923F924F925F926F92AB
:104E10007F928F929F92AF92BF92CF92DF92EF924A
:104E2000FF920F931F93CF93DF93CDB7DEB7C65991
:104E3000D1090FB6F894DEBF0FBECDBFC257DF4F0A
:104E40008883CE58D04080912A058D3409F425C13D
:104E5000843511F40C942D3C873411F00C94713C82
:104E600020912805309129052A31310509F477C0B0
:104E70006CF42430310534F422303105C4F537FFA9
:104E80002FC007C124303105D9F103C12A353105BE
:104E900009F49CC06CF42B31310509F467C02C3146
:104EA000310509F0F6C080E00E9450790C94733C03
:104EB0002B35310509F48EC02C35310509F0E9C0D8
:104EC0000DEE12E01DAB0CAB34EDE32E35E0F32E0E
:104ED00045E8C42E43E0D42E312C00E010E0B4C0ED
:104EE00080911E0281110C947E3C0C94733C81E0F5
:104EF0002230310509F080E00E943A730C94733C33
:104F000080E50E948190882329F00E94C78F6B0161
:104F10007C0103C0C12CD12C760183E50E948190D5
:104F2000882361F00E94079020E030E04AE754E4D3
:104F30000F947B020F94C9076B017C010E94D54B33
:104F40008091C10E811105C060E087E592E00E946A
:104F50005391C701B6010E9468720C94733C81E0C2
:104F600080931E02109220090C94733C0E94B8FB9F
:104F700081110C94733C80E090E0A8ECB2E489834A
:104F80009A83AB83BC8380E090E8A9E8B3E48D8387
:104F90009E83AF83B88780E090E0A0EAB1E4898780
:104FA0009A87AB87BC8780E50E948190882319F09F
:104FB0000E94D78F01C060E068A3BE016F5F7F4F82
:104FC000CE0180960E945AF60C94733C1092A10375
:104FD0000C94733C81E08093A1030C94733C0E9479
:104FE00007902B013C01133049F0F60120813181FB
:104FF000428153810F947F062B013C01D7012D91F3
:105000003D914D915C91C301B2010F947F064B011C
:105010005C012DEB37E346E855EB0F94A60887FDBE
:105020001DC02DEB37E346E855E3C501B4010F94ED
:10503000160218169CF01F5FF4E0EF0EF11C24E03E
:10504000C20ED11C1430B1F0ACA9BDA98D91BDAB7D
:10505000ACAB0E948190882371F3C1CF133011F063
:1050600001E002C033243394F7014082518262820E
:105070007382E1CF002319F00E94BD8F06C0332058
:1050800021F080EE95E00E9454FC0E9452B50C94F1
:10509000733C0E9445FD0C94733C809128059091CF
:1050A00029058637910509F4A3C50CF0ADC08B34F2
:1050B000910509F445C40CF04DC08931910509F4FE
:1050C000B4C21CF58431910509F426C27CF4813107
:1050D000910509F416C22CF4029708F49BC10C94B4
:1050E0002A3C429709F461C50C942A3C863191050B
:1050F00009F459C20CF453C28731910509F459C21D
:10510000489709F46CC20C942A3C8E31910509F43D
:105110004CC384F48B31910509F4A3C20CF493C2FF
:105120008C31910509F437C34D9711F40C94733CFD
:105130000C942A3C8032910509F43BC30CF485C3DE
:105140008A32910509F4ABC38934910509F4EBC3A4
:105150000C942A3C8836910509F402C45CF582352A
:10516000910509F419C59CF48D34910509F4F0C337
:105170000CF4EAC38E34910509F4EEC38135910530
:1051800011F00C942A3C0E944EB70C94733C843569
:10519000910509F40AC50CF403C58535910509F498
:1051A00008C58C35910511F00C942A3C0E943FB63D
:1051B0000C94733C8E36910509F4F3C384F48A365B
:1051C000910509F4E1C40CF44DC48B36910509F442
:1051D000DFC48D36910509F486C40C942A3C8237CD
:1051E000910509F4EAC434F48F36910509F4ECC34F
:1051F0000C942A3C8337910509F4E5C48537910561
:1052000009F4E5C40C942A3C8D3231E0930711F483
:105210000C9490320CF07AC0893C910509F4A5C534
:1052200084F58C38910509F47AC49CF4883791058B
:1052300009F446C50CF4E0C48937910509F447C563
:105240008D37910511F00C942A3C0E940DB40C94FA
:10525000733C8B39910509F41FC44CF481399105D5
:1052600011F00C942A3C0E9463B70C94733C8E3B63
:10527000910509F472C4883C910509F42EC50C947B
:105280002A3C833D910509F485C73CF58C3C91058A
:1052900009F4A3C57CF48B3C910511F00C942A3CD5
:1052A000E5E5EE2EE9E0FE2E0DEE12E0F4E0DF2E55
:1052B000D00E84C58D3C910509F407C68E3C91053E
:1052C00011F00C942A3C6DEEC62E62E0D62E78ECDE
:1052D000E72E75E0F72E10E06CC68D3D910511F4B8
:1052E0000C94AE313CF48C3D910511F40C949F313B
:1052F0000C942A3C823E910511F40C941F328C329E
:10530000914011F40C9466320C942A3C853FA1E044
:105310009A0711F40C943B39DCF58F35E1E09E07D8
:1053200011F40C94CD38B4F48F3201E0900711F4ED
:105330000C948A3314F40C943333803321E09207B5
:1053400011F40C941B388E35914011F40C9498385C
:105350000C942A3C803941E0940711F40C943839BC
:105360004CF48336914011F00C942A3CE4E4F9E4C7
:105370000C9421398C3AB1E09B0709F42CC6843F88
:10538000914011F00C942A3C0E94AEC70C94733CDF
:105390008835F2E09F0711F40C947B39B4F4873F11
:1053A00011E0910711F40C94413914F40C943E3936
:1053B000883F31E0930711F40C944D398C319240C1
:1053C00011F40C9470390C942A3C8C3853E09507F6
:1053D00011F40C94FC3B94F48B35B2E09B0711F470
:1053E0000C944C3B8B38934011F00C942A3C9DEE6E
:1053F000E92E92E0F92E10E00C94D83B803AF3E0CD
:105400009F0709F415C2873E934011F40C94153C94
:105410000C942A3CA0902605B090270580E50E94B8
:105420008190882359F00E94C78F6B017C0111E0A5
:10543000672B682B692B31F410E004C010E0C12CFD
:10544000D12C760183E50E948190882311F40C947D
:10545000653D0E94079020E030E04AE754E40F9455
:105460007B020F94C9076B017C0111110BC0672BE4
:10547000682B692B39F4A114B10421F0D5018C916A
:10548000811102C010E001C011E00E94D54B112330
:1054900029F061E0C5010E948D9105C060E080E6C1
:1054A00092E00E94539181E080936914C114D10469
:1054B000E104F104F1F00E94F6B2C60ED71EE81E18
:1054C000F91E0E94F6B2DC01CB018C199D09AE09D0
:1054D000BF09B7FD06C00E9439F9109269140C94F7
:1054E000733C809169148823B1F380E00E94A85036
:1054F000E8CF80916914882371F380E00E94A8505E
:10550000F8CF60E083E792E00E94539117981698D5
:10551000159814980C94733CEBE8F2E084918F0199
:105520000F5F1F4F882321F00E94F0F6F801F6CF9D
:105530001092C51140E050E0BA0188E79FE00E9458
:10554000A4CE8BE1E8E7FFE0DE01159601900D9215
:105550008A95E1F78091760F9091770F9C838B83EA
:1055600082E793E09A83898340E050E0BE016F5F59
:105570007F4F80E090E00E94EBBECE0101960E943A
:105580002C50ECE7F2E084918F010F5F1F4F8823CE
:1055900011F40C94733C0E94F0F6F801F4CF0E94D1
:1055A00066EE0C94733C1092210F1092220F0C9413
:1055B000733CE0912605F09127058081882329F02E
:1055C000803209F410823196F8CF40E061E080919A
:1055D0002605909127050E9475EC0C94733C198266
:1055E0001A821B821C8218A219A21AA21BA21CA238
:1055F0001DA21EA21FA28091AC0E882359F020E0AC
:10560000AE014F5F5F4FBE01605E7F4FCE0184965B
:105610000E946B538091220F882319F081E08093C0
:10562000210F0E9463990C94733C1092210F0E94E9
:105630004E998CE992E090930809809307090E94A3
:105640005E8F0C94733C8091220F882311F40C948C
:10565000733C83E50E94819081110C946A3D0C9407
:10566000733C83E40E943A90882309F454C0EEEC22
:10567000F2E084918F010F5F1F4F882321F00E9479
:10568000F0F6F801F6CF80911311882391F0BE0156
:105690006F5F7F4F80E191E10E9494D48E010F5F94
:1056A0001F4FF80181918F01882381F10E94F0F64C
:1056B000F8CFE1EAF2E084918F010F5F1F4F88235A
:1056C00029F10E94F0F6F801F6CF80917F0E882331
:1056D00009F4BBC126E2C22E23E0D22EE12CF12C2C
:1056E00020E080917F0E90E00E2C02C0959587956A
:1056F0000A94E2F780FD91C1FFEFEF1AFF0A02E082
:10570000C00ED11C15E0E116F10459F78AE00E94A1
:10571000F0F60C94733C8091220F882371F18091F4
:10572000210F882351F1EBEAF2E084918F010F5FA2
:105730001F4F882321F00E94F0F6F801F6CF609108
:10574000C1117091C2118091C3119091C4114AE0AE
:105750000E9443F78FE20E94F0F66091BD117091B4
:10576000BE118091BF119091C0114AE00E9443F791
:105770008AE00E94F0F60C94733CEDEBF2E0849129
:105780008F010F5F1F4F882311F40C94733C0E940C
:10579000F0F6F801F4CF40E060E0809126059091AA
:1057A00027050E9475EC0C94733C0E942EB90C9452
:1057B000733C8091210F81110E94D54B8091220F63
:1057C000882311F40C94733C80E50E948190882317
:1057D00019F00E94F88F03C080E50E943A90182FBC
:1057E000482F61E080912605909127050E9475EC75
:1057F00083E50E948190882381F00E94D78FAB01BE
:10580000BC014093C1115093C2116093C3117093B6
:10581000C41180E191E10E94A4CE8091220F8823DF
:1058200019F081E08093210F11110C94733CF9CE93
:10583000809126059091270521E02093200F40E0DC
:1058400060E00E9475EC0C94733C0E941A9968A366
:1058500079A38AA39BA3BE016F5F7F4FCE01809681
:105860000E943D9A60E0CE0101960E948D91ECE489
:10587000F2E484918F010F5F1F4F882321F00E9473
:10588000F0F6F801F6CFBE016F5F7F4F8DED92E02D
:105890000E94E8688AE00E94F0F60C94733C83E56D
:1058A0000E948190882311F40C94733C0E94E78F2E
:1058B000E82E80E50E948190882311F40C94733CBB
:1058C00080E50E948190882339F00E94E78F182F8D
:1058D00087FF03C00C94733C1DE0E9EFF2E08DE21A
:1058E0008E0F9491191729F031968E13FACF0C94DC
:1058F0007B3DE4E4F9E484918F010F5F1F4F88231F
:1059000021F00E94F0F6F801F6CFEAEEF2E0849181
:105910008F010F5F1F4F882311F40C94733C0E947A
:10592000F0F6F801F4CF8091210F81110C94733CB3
:1059300080E50E943A9081110C94963D0C94733C42
:105940000E9463990C94733C0E944E990C94733C92
:105950000E94C0990C94733C0E9415B80C94733C3F
:1059600088E690E00E94CC7B81110C94733C80917E
:105970007F0E83FF02C00C94733C83E50E948190EC
:10598000882311F40C94733C0E9407900F94C40771
:10599000709313156093121580E00E9443630C947A
:1059A000733C8EE40E948190882311F40C94733C24
:1059B0000E94D78F60932214709323148093241431
:1059C000909325140C94733C83E50E943A908823AD
:1059D00059F083E50E948190882319F00E94E78F97
:1059E00001C080E080937F0EECE4F2E484918F01AB
:1059F0000F5F1F4F882321F00E94F0F6F801F6CFC9
:105A0000E4E3F3E084918F010F5F1F4F882309F4D3
:105A10005CCE0E94F0F6F801F5CFBB24B394B20E31
:105A2000222319F08CE20E94F0F6F60125913491C0
:105A3000F901849189010F5F1F4F882321F00E9493
:105A4000F0F69801F5CF2B2D57CEE0E3F3E08491EB
:105A50008F010F5F1F4F882309F458CE0E94F0F684
:105A6000F801F5CF89E690E00E94CC7B81110C947F
:105A70006E42EBE3F3E084918F010F5F1F4F8823A9
:105A800021F00E94F0F6F801F6CF0E9425688AE026
:105A90000E94F0F60C946E4283E50E948190882368
:105AA00011F40C94733C0E94E78F182F8D3308F08B
:105AB0001CE310933B040E94F6B26B017C01212F82
:105AC00030E0A8EEB3E00F947006C60ED71EE81EB5
:105AD000F91EC0923704D0923804E0923904F09253
:105AE0003A040C94733C8DE690E00E94CC7B8111CB
:105AF0000C94733C80917F0E83FF02C00C94733C26
:105B000083E50E9481908CAB81110C94A13D82E5CC
:105B10000E94819081110C94A13D0C94733C809162
:105B20007F0E83FF02C00C94733C83E50E9481903A
:105B3000882311F40C94733C0E9407900F94C407BF
:105B40006639710514F066E970E07093070560939B
:105B500006050E94F8620C94733C80917F0E83FFCF
:105B600002C00C94733C83E50E94819028968FAF0D
:105B7000289781110C942E3F82E50E94819081111B
:105B80000C942E3F0C94733C0E94EFB70C94733C22
:105B90000E94DAB70C94733C1092A0030C94733CEF
:105BA00081E08093A0030C94733C0E94F5B60C94A2
:105BB000733C0E94DDB60C94733C0E94D54B0E944E
:105BC00052B50C94733C0E9403B50C94733C8091C5
:105BD000260590912705DC012C91211104C00E941B
:105BE00039F90C94733C60E00E948D910C94733CE5
:105BF0000E94B1B40C94733CE4EAF3E084918F0109
:105C00000F5F1F4F882321F00E94F0F6F801F6CFB6
:105C1000ECE9F3E084918F010F5F1F4F882321F09F
:105C20000E94F0F6F801F6CF1E9B03C006ED12E0CD
:105C300002C00BED12E0F80181918F01882319F069
:105C40000E94F0F6F8CF8AE00E94F0F6E4E9F3E073
:105C500084918F010F5F1F4F882321F00E94F0F67F
:105C6000F801F6CF1D9B03C006ED12E002C00BED5C
:105C700012E0D8018D918D01882319F00E94F0F671
:105C8000F8CF8AE00E94F0F6ECE8F3E084918F010F
:105C90000F5F1F4F882321F00E94F0F6F801F6CF26
:105CA0001C9B03C006ED12E002C00BED12E0F801F0
:105CB00081918F01882309F429CD0E94F0F6F7CF56
:105CC00081E08093C7058093C5050C94733C1092C6
:105CD000C7051092C5050C94733C88EC90E00E94B7
:105CE000CC7B81110C94733C84E40E943A9088230D
:105CF000C1F10E94079011E020E030E0A9010F946B
:105D00001602811101C010E010936714112349F1AC
:105D10000E940790E091010504E0E09FF00111244A
:105D2000ED59FB4E608371838283938320E030E0E2
:105D3000A90160916314709164148091651490912D
:105D400066140F94160281110CC080E090E0A0E46C
:105D5000B0E48093631490936414A0936514B0939B
:105D600066140E94204D0C94733CA3E5EA2EA4E136
:105D7000FA2E0DEE12E0B4E0DB2ED00ED8018D919C
:105D80008D010E943A90882349F00E9407900F9459
:105D9000C907F7016083718382839383F4E0EF0E78
:105DA000F11CD012EBCF0E940D4B0C94733CF4E02D
:105DB000EF0EF11CD01611F40C94733CD8018D91A8
:105DC0008D010E943A90882391F30E940790F70179
:105DD0006083718382839383EACF83E50E948190FD
:105DE0008823A1F00E94079060934D0970934E099B
:105DF00080934F09909350096093490970934A0921
:105E000080934B0990934C0910E001C011E080E5AC
:105E10000E948190882359F00E94079060934D0959
:105E200070934E0980934F099093500910E082E5DA
:105E30000E948190882359F00E9407906093510935
:105E400070935209809353099093540910E084E5AC
:105E50000E948190882361F00E9407906093490915
:105E600070934A0980934B0990934C090C94733CAE
:105E7000112311F40C94733C40914D0950914E093B
:105E800060914F097091500984EC93E00E94D167B2
:105E900040915109509152096091530970915409F0
:105EA00081EC93E00E94D1674091490950914A09E1
:105EB00060914B0970914C098EEB93E00E94D16781
:105EC0008AE00E94F0F60C94733C82E40E943A90BF
:105ED000882351F00E94C78F6093690970936A0903
:105EE00080936B0990936C0983E50E943A90882314
:105EF00051F00E940790609381097093820980930A
:105F000083099093840984E50E943A90882351F094
:105F10000E94079060937D0970937E0980937F09AA
:105F20009093800988E50E943A90882351F00E945E
:105F30000790609325097093260980932709909311
:105F4000280989E50E943A90882351F00E94079021
:105F50006093290970932A0980932B0990932C0947
:105F60008AE50E943A90882351F00E94079060933E
:105F70002D0970932E0980932F099093300985E4A1
:105F80000E943A90882311F40C94733C0E9407906D
:105F900060933109709332098093330990933409E7
:105FA0000C94733C1F5FF4E0EF0EF11C133009F406
:105FB0006CC8D6018D916D010E943A90882391F3AF
:105FC0000E940790F7016083718382839383812FFE
:105FD0000E948C7BE7CF0E94B8FB81110C94733C2C
:105FE00054EF852E5FE0952E04ED15E01DAB0CAB54
:105FF0009E012F5F3F4F59010DE410E1190133E07D
:10600000300F3EABF4016591759185919491ACA9E7
:10601000BDA9CD90DD90ED90FD90BDABACABA701DF
:1060200096010F947F062B013C0120E030E040EA0E
:1060300051EC0F94A60887FD10C020E030E040EA44
:1060400051E4C301B2010F941602181634F0F101A5
:1060500040825182628273820DC0F80184911816C9
:10606000B4F7F7FAF094F7F8F094F101C082D18216
:10607000E282F382D101CD90DD90ED90FD901D0183
:1060800020E030E040EA51ECC701B6010F94A608C9
:1060900087FF03C0E4E4F9E40BC020E030E040EA0D
:1060A00051E4C701B6010F94160218167CF5F2CF21
:1060B00084918F010F5F1F4F882321F00E94F0F61B
:1060C000F801F6CFE2EFF3E084918F010F5F1F4FED
:1060D000882321F00E94F0F6F801F6CF61E084EE0B
:1060E00093E00E9453910E94C95B88E290E099A3DB
:1060F00088A388EC90E09DA38CA3BE01605E7F4FD7
:10610000CE0184960E949FEF0C94733CB4E08B0EFA
:10611000911C0F5F1F4FEEA9E01374CF48ECE42EE3
:1061200045E0F42E10E0F50181919191A191B1919A
:106130005F01F70181939193A193B1937F01812F27
:106140000E948C7B1F5F133071F70E9452B560E094
:1061500084ED93E00E94539183E992E09DA38CA388
:1061600004E610E019A308A3BE016C5D7F4FCE01C9
:1061700080960E949FEF8AEB92E09DA38CA319A3C7
:1061800008A3BE016C5D7F4FCE0180960E949FEFF9
:106190000C94733CECE4F2E484918F010F5F1F4F89
:1061A000882321F00E94F0F6F801F6CF83E50E94E3
:1061B0003A90882321F00E94F88F80931902E8E337
:1061C000F4E084918F010F5F1F4F882321F00E941C
:1061D000F0F6F801F6CF80911902811103C0E4E3D3
:1061E000F4E002C0E0E3F4E084918F010F5F1F4F01
:1061F000882321F00E94F0F6F801F6CFE8E2F4E0FF
:1062000084918F010F5F1F4F882321F00E94F0F6C9
:10621000F801F6CF40908503509086036090870385
:1062200070908803209191033091920340919303E1
:1062300050919403C301B2010F948006AB01BC01DD
:1062400086E294E00E94D1678090890390908A034F
:10625000A0908B03B0908C0320919503309196030E
:106260004091970350919803C501B4010F948006A3
:10627000AB01BC0183E294E00E94D167C0908D0322
:10628000D0908E03E0908F03F090900320919903BB
:1062900030919A0340919B0350919C03C701B60132
:1062A0000F948006AB01BC0180E294E00E94D167AC
:1062B000E8E1F4E084918F010F5F1F4F882321F004
:1062C0000E94F0F6F801F6CF20910D0230910E02F7
:1062D00040910F0250911002C301B2010F94800649
:1062E000AB01BC0186E194E00E94D16720911102CC
:1062F000309112024091130250911402C501B40171
:106300000F948006AB01BC0183E194E00E94D16749
:1063100020911502309116024091170250911802F7
:10632000C701B6010F948006AB01BC0180E194E087
:106330000E94D1678AE00E94F0F60C94733C83E5DA
:106340000E948190882311F40C94733C0E94D78F93
:1063500070930502609304020C94733C8DED90E001
:106360000E94CC7B81110C94733C83E50E94819048
:106370008823E1F10091010510E00E94D78F000F02
:10638000111FF801EA5FFD4F718360838091010561
:1063900090E08C01000F111F000F111F9801255C68
:1063A0003D4F7901880F991FFC01EA5FFD4F608125
:1063B0007181072E000C880B990B0F941C022AE0A8
:1063C00037ED43E25CE30F947B02F801EE55FC4F9E
:1063D00020813181428153810F947B02D7016D93DB
:1063E0007D938D939C9313970C94733CECE4F2E4AF
:1063F00084918F010F5F1F4F882321F00E94F0F6D8
:10640000F801F6CF85E40E94F0F680910105805DE9
:106410000E94F0F6E0910105F0E0EE0FFF1FEA5F49
:10642000FD4F6081718188E494E00E94CF6885E22D
:106430000E94F0F68AE00E94F0F60C94733C80E52E
:106440000E943A90882311F40C94733C0E94D78FD9
:106450006B017C0183E50E948190882321F00E94DA
:10646000D78F8B0102C00FEF1FEF98012F5F3F4FB7
:106470002330310510F00C94733CD7FE02C00C940D
:10648000733C0E94D54B0F3FBFEF1B0731F001302B
:10649000110571F401E010E00DC08C2D0E94A0B137
:1064A00031E020E0892B09F030E0032F122F02C0E9
:1064B00000E010E08C2D0E94A0B18017910711F42C
:1064C0000C94733C80E00E94A850F4CF83E50E94B6
:1064D0008190882319F00E94D78F02C064E071E098
:1064E00079A368A380E50E948190882339F00E94F7
:1064F000D78F6938E3E17E0730F402C068EE73E0BD
:106500007A83698304C088E893E19A838983BE0112
:10651000605E7F4FCE0101960E949FEF0C94733C0A
:1065200085E40E948190811110C080E50E943A901C
:10653000882391F00E940790609343147093441451
:10654000809345149093461407C00E94E78F8823D8
:1065500061F3E4E4F9E46FC089E40E943A9088238F
:1065600081F00E9407902CEA35EC47E25EE30F943D
:106570007B0260933F147093401480934114909376
:10658000421484E40E943A90882381F00E9407908C
:106590002CEA35EC47E25EE30F945C0760933B1412
:1065A00070933C1480933D1490933E14ECE4F2E419
:1065B00084918F010F5F1F4F882321F00E94F0F616
:1065C000F801F6CF40914314509144146091451462
:1065D0007091461488E594E00E94D1672CEA35EC6E
:1065E00047E25EE360913F14709140148091411442
:1065F000909142140F945C07AB01BC0184E594E0D8
:106600000E94D1672CEA35EC47E25EE360913B14CF
:1066100070913C1480913D1490913E140F947B0234
:10662000AB01BC0180E594E00E94D1678AE00E9442
:10663000F0F60C94733C84918F010F5F1F4F8823F9
:1066400021F00E94F0F6F801F6CFECE5F4E0849139
:106650008F010F5F1F4F882311F40C94733C0E942D
:10666000F0F6F801F4CF83E50E943A90182F8823C2
:1066700071F00E9407900F94C407709340026093DA
:106680003F0221E0672B09F020E020938A0980E592
:106690000E943A90882361F020913F02309140029D
:1066A000232B11F00E94F88F80938A090C94733C7D
:1066B00011110C94733CECE4F2E484918F010F5FB0
:1066C0001F4F882321F00E94F0F6F801F6CF809149
:1066D0008A09811103C065EE72E002C068ED72E0C4
:1066E00083E894E00E94E86860913F027091400264
:1066F00082E794E00E94CF68EEE6F4E084918F0197
:106700000F5F1F4F882311F40C94733C0E94F0F626
:10671000F801F4CF85E40E948190882321F00E9443
:10672000D78F7B0102C0E12CF12C83E40E94819081
:10673000882321F00E94D78F6EAF02C005E00EAF14
:1067400085E50E948190882319F00E94F88F03C08C
:1067500085E50E943A90AC968FAFAC97F7FC07C0E6
:10676000812C912C06E1A02E03E4B02E06C0812CD2
:10677000912C1CE8A12E12E4B12E83E50E94819099
:10678000882321F00E9407904B015C01E114F10481
:1067900011F410920105ECAA0E94F6B22B013C0103
:1067A0001CA917FD08C0A8E2CA2ED12C0AE0BAE045
:1067B0002B2E312C07C0ECE3CE2ED12C02E0F5E0DD
:1067C0002F2E312C61E06E0D623070F0EFE2F6E0BA
:1067D00084918F010F5F1F4F882311F40C94733C39
:1067E0000E94F0F6F801F4CFE9E5F6E084917F012C
:1067F0002FEFE21AF20A882321F00E94F0F6F70147
:10680000F5CF0E948E631CA917FF08C087E680930E
:10681000000527E630E040E050E00CC01CA9E12F65
:10682000110FFF0BE150FB4F8FE780832FE730E024
:1068300040E050E026962CAF3DAF4EAF5FAF2697BD
:10684000C501B4010F94C407072E000C880B990BE7
:106850000F941C0227966FAF279728967FAF289733
:1068600029968FAF29972D969FAF2D97402F50E0F7
:106870009601A8EEB3E00F947006E0966CAF7DAF82
:106880008EAF9FAFE097DC01CB01840D951DA61D57
:10689000B71DEC968CAF9DAFAEAFBFAFEC9781E06C
:1068A000809354020CA907FF05C08EEC90E0A0E095
:1068B000B0E004C08FEF90E0A0E0B0E08C019D015B
:1068C0000351110921093109C258DF4F0883198387
:1068D0002A833B83CE57D0408C019D01045111097E
:1068E00021093109CE57DF4F088319832A833B835F
:1068F000C258D0408C019D01359527951795079575
:10690000CA57DF4F088319832A833B83C658D04078
:106910008C019D010150110921093109C657DF4F32
:10692000088319832A833B83CA58D04026968CACAF
:106930009DACAEACBFAC2697A7964CAE5DAE6EAE2E
:106940007FAEA797E4964CAE5DAE6EAE7FAEE49799
:10695000A3961FAEA397E8961CAE1DAE1EAE1FAE4B
:10696000E89768961FAE689710E469961FAF69971D
:106970000CE16A960FAF6A9716E46B961FAF6B97A0
:106980006C961FAE6C976D961FAE6D976E961FAE90
:106990006E976F961FAE6F9767961CAE1DAE1EAEBC
:1069A0001FAE679763961CAE1DAE1EAE1FAE6397FB
:1069B000C12CD12C7601AB961CAE1DAE1EAE1FAE07
:1069C000AB9701E0A2960FAFA2972F961FAE1EAE17
:1069D0002F9710E01EAA1AAE00E02CA9822F220FDA
:1069E000990BDC01A150BB4FEE96BFAFAEAFEE9757
:1069F000880F991F880F991FFC01E557F64FA19644
:106A0000FFAFEEAFA197CA01052E000CAA0BBB0B7E
:106A1000C157DF4F88839983AA83BB83CF58D04067
:106A2000240E351E9FEF291A390A9101330C440BAD
:106A3000550BCD56DF4F288339834A835B83C35977
:106A4000D0404EAD242E440F330880915402882349
:106A500009F428C10E94F6B222966CAF7DAF8EAFCA
:106A60009FAF22978091EE04882309F4F7C00E941B
:106A70004C640CA907FF0BC010910205009103059F
:106A80000EAB009104050AAF009105050FC0A19659
:106A9000AEADBFADA1971C9111960C9111970EABA5
:106AA00012960C9112970AAF13960C91212F3EA9C2
:106AB0004AAD502F6C966FAD6C976D967FAD6D970C
:106AC0006E968FAD6E976F969FAD6F970F9416026F
:106AD00087FF0EC06C961FAF6C972EA96D962FAFD7
:106AE0006D973AAD6E963FAF6E976F960FAF6F97FB
:106AF000212F3EA94AAD502F68966FAD68976996D1
:106B00007FAD69976A968FAD6A976B969FAD6B97CD
:106B10000F94A608181674F468961FAF68974EA9CC
:106B200069964FAF69975AAD6A965FAF6A976B9651
:106B30000FAF6B97A2968FADA29727962FAD279791
:106B400028963FAD289729964FAD29972D965FAD92
:106B50002D97612F7EA9882309F460C08AAD902FFC
:106B60000F94A60818160CF079C022964CAD5DADB6
:106B70006EAD7FAD22974419550966097709DB018F
:106B8000CA0188589341A109B109B7FD67C026968B
:106B90008CAD9DADAEADBFAD269788199909AA09F8
:106BA000BB09ECA9B595A79597958795E7FF03C015
:106BB0008093000505C0EE96EEADFFADEE978083A5
:106BC000AB964CAF5DAF6EAF7FAFAB972796FFAD87
:106BD00027976C96FFAF6C9728962FAD28976D96E8
:106BE0002FAF6D9729963FAD29976E963FAF6E9761
:106BF0002D964FAD2D976F964FAF6F9722968CAD18
:106C00009DADAEADBFAD2297A7968CAF9DAFAEAF99
:106C1000BFAFA797A2961FAEA29720C08AAD902FB4
:106C20000F94160287FF1AC022968CAD9DADAEADB3
:106C3000BFAD2297A7962CAD3DAD4EAD5FADA797EA
:106C4000821B930BA40BB50BAC01BD0148585341FB
:106C50006109710977FD02C00C94C54020E030E065
:106C600040EA51E427966FAD279728967FAD289785
:106C700029968FAD29972D969FAD2D970F9480065D
:106C80009B01AC01612F7EA98AAD902F0F94A608BD
:106C900018167CF4EBEBF5E084918F010F5F1F4F2A
:106CA000811103C00E948E631EC60E94F0F6F80197
:106CB000F3CF22968CAD9DADAEADBFAD2297E496DD
:106CC0002CAD3DAD4EAD5FADE497821B930BA40B95
:106CD000B50BB7FDCAC00E9425688AE00E94F0F695
:106CE00022968CAD9DADAEADBFAD22978053984F2F
:106CF000AF4FBF4FE4968CAF9DAFAEAFBFAFE49741
:106D0000A3969FADA397911187C0E8962CAD3DAD9A
:106D10004EAD5FADE897612F7EA98AAD902F0F949D
:106D2000A60818160CF05BC0C157DF4F6881798147
:106D30008A819B81CF58D0400F941C029B01AC01EB
:106D4000612F7EA98AAD902F0F948006E8966CAFD4
:106D50007DAF8EAF9FAFE89722962CAD3DAD4EAD87
:106D60005FAD2297E0968CAD9DADAEADBFADE09727
:106D7000280F391F4A1F5B1FEC962CAF3DAF4EAF5B
:106D80005FAFEC97CD56DF4F688179818A819B8117
:106D9000C359D0400F941C029B01AC0127966FADE4
:106DA000279728967FAD289729968FAD29972D96FE
:106DB0009FAD2D970F947F069B01AC0191E0A396A8
:106DC0009FAFA397612F7EA98AAD902F0F94A6083D
:106DD00018160CF44AC0A3961FAEA39746C022967D
:106DE0008CAD9DADAEADBFAD2297EC962CAD3DAD5B
:106DF0004EAD5FADEC97821B930BA40BB50BB7FDAB
:106E000034C03CA93F3F19F047E855E002C049E9CA
:106E100055E06CEA75E026C020E030E040EA51E43D
:106E200027966FAD279728967FAD289729968FAD27
:106E300029972D969FAD2D970F947F069B01AC014E
:106E4000612F7EA98AAD902F0F94160287FF0DC087
:106E50004CA94F3F19F040E555E002C043E655E02C
:106E600067E775E08CA90E946B6422968CAD9DAD9E
:106E7000AEADBFAD2297880F991FAA1FBB1FA79663
:106E80002CAD3DAD4EAD5FADA797821B930BA40B10
:106E9000B50B84199509A609B70981389F44A24109
:106EA000B10568F0E2E3F5E084918F010F5F1F4FB9
:106EB000882309F4F7CE0E94F0F6F801F5CF2F965B
:106EC0004EAD5FAD2F97241635060CF0B1C0E5ED41
:106ED000F4E084918F010F5F1F4F882321F00E94FF
:106EE000F0F6F801F6CF0CA907FD03C007E613E0A2
:106EF00002C009EE12E0B80184EC94E00E94E86858
:106F0000B701A60180EC94E00E94D1678AE00E945C
:106F1000F0F6B8018FEA94E00E94E86863964CAD01
:106F20005DAD6EAD7FAD63978BEA94E00E94D16753
:106F30008AE00E94F0F6B8018AE994E00E94E868CD
:106F400067964CAD5DAD6EAD7FAD679786E994E019
:106F50000E94D1678AE00E94F0F6AC961FADAC9714
:106F6000112309F4C0C40CA907FF31C0C092371423
:106F7000D0923814E0923914F0923A142CEA35EC9D
:106F800047E25EE363966CAD7DAD8EAD9FAD6397DA
:106F90000F947B02609333147093341480933514F0
:106FA000909336142CEA35EC47E25EE367966CADBD
:106FB0007DAD8EAD9FAD67970F945C0760932F14E6
:106FC0007093301480933114909332148CC4C09217
:106FD0004314D0924414E0924514F09246142CEAE3
:106FE00035EC47E25EE363966CAD7DAD8EAD9FAD53
:106FF00063970F947B0260933F14709340148093C7
:107000004114909342142CEA35EC47E25EE3679614
:107010006CAD7DAD8EAD9FAD67970F945C076093AF
:107020003B1470933C1480933D1490933E145BC4C6
:107030000E94B4910ACD80E50E943A90882351F0D5
:107040000E9407906093371470933814809339141A
:1070500090933A1489E40E943A90882381F00E9428
:1070600007902CEA35EC47E25EE30F947B026093D5
:10707000331470933414809335149093361484E44D
:107080000E943A90882381F00E9407902CEA35EC08
:1070900047E25EE30F945C0760932F147093301403
:1070A0008093311490933214ECE4F2E484918F01D4
:1070B0000F5F1F4F882321F00E94F0F6F801F6CFF2
:1070C00040913714509138146091391470913A14EA
:1070D00085E796E00E94D1672CEA35EC47E25EE353
:1070E000609133147091341480913514909136145A
:1070F0000F945C07AB01BC0181E796E00E94D16769
:107100002CEA35EC47E25EE360912F147091301465
:1071100080913114909132140F947B02AB01BC0129
:107120008DE696E00E94D1678AE00E94F0F6DBC30C
:1071300083E50E943A90811106C07DEEE72E72E051
:10714000F72E10E00EC010E00E94E78F682F812F0D
:107150000E942D711F5F1530B9F7EFCF1F5F1430FC
:1071600071F0D7018D917D010E943A908823B1F38F
:107170000E94E78F682F812F0E942D71EFCF82E44C
:107180000E943A90882331F00E94E78F682F84E0B4
:107190000E942D710E947570A6C383E50E948190A4
:1071A000882309F44BC00E94E78F813049F0823078
:1071B00009F044C05DEEE52E52E0F52E10E023C04C
:1071C0006DEEE62E62E0F62E10E0F70181917F0170
:1071D0000E948190882339F00E94E78F4FEF682F3B
:1071E000812F0E94E0421F5F143079F782E40E94F1
:1071F0008190882319F10E94E78F4FEF682F1BC001
:107200001F5F143079F0D7018D917D010E9481902C
:107210008823B1F30E94E78F482F6FEF812F0E94E0
:10722000E042EECF82E40E948190882339F00E94F0
:10723000E78F482F6FEF84E00E94E0420E94757054
:1072400052C384918F010F5F1F4F882321F00E944A
:10725000F0F6F801F6CFE9E7F6E084918F010F5FD1
:107260001F4F882309F43FC30E94F0F6F801F5CFC1
:107270000E94D54B38C30E9436F535C30E94EBF30C
:1072800032C383E50E943A90882321F00E94F88F50
:1072900091E089270E94D3EF26C381E080932614D2
:1072A0000E94F9C110922614882309F41CC3ECE44F
:1072B000F2E484918F010F5F1F4F882321F00E9419
:1072C000F0F6F801F6CFE8E8F6E084918F010F5F61
:1072D0001F4F882309F407C30E94F0F6F801F5CF89
:1072E00083E50E943A90882309F4FDC20E94F88F3A
:1072F0008093EA05F8C280E090E0A8ECB2E48983CC
:107300009A83AB83BC8380E090E8A9E8B3E48D83E3
:107310009E83AF83B88780E090E0A0EAB1E48987DC
:107320009A87AB87BC8788E592E00E94CC7B81116D
:10733000DAC2609101050E9413A90E94B8FB88235C
:1073400019F081E00E94507985E40E943A908823E8
:1073500081F00E9407906B017C0120E030E0A901E0
:107360000F94A60887FF0AC0F7FAF094F7F8F09494
:1073700005C0C12CD12CE12C40E4F42EF7FAF09496
:10738000F7F8F094C8AAD9AAEAAAFBAA8AE50E944B
:107390008190882379F08AE50E948190882319F0F2
:1073A0000E94079003C060E070E0CB0169877A8794
:1073B0008B879C8788E50E948190882379F088E5F7
:1073C0000E948190882319F00E94079003C060E01A
:1073D00070E0CB0169837A838B839C8389E50E946B
:1073E0008190882379F089E50E948190882319F0A3
:1073F0000E94079003C060E070E0CB016D837E8344
:107400008F83988785E50E943A90882329F00E940F
:1074100007906B017C010CC0E0911115B4E0EB9F6B
:10742000F0011124E95DFB4EC080D180E280F38041
:1074300020E030E0A901C701B6010F94A60887FF3C
:1074400004C0F7FAF094F7F8F094F7FAF094F7F82C
:10745000F094CCA6DDA6EEA6FFA618A619A61AA63D
:107460001BA68CE40E943A90882329F00E94079082
:107470006B017C010CC0E091111504E0E09FF0016C
:107480001124E55DFB4EC080D180E280F38020E0D6
:1074900030E0A901C701B6010F94A60887FF04C018
:1074A000F7FAF094F7F8F094CCA2DDA2EEA2FFA2D6
:1074B00082E40E948190882321F00E94D78F162FAA
:1074C00001C01AE00091B3058091AC0E8111DEC0BD
:1074D00021E0AE01445D5F4FBE016F5F7F4FCE0183
:1074E000C0960E94CB4D882309F4D0C0609111153D
:1074F00082E00E9413A9ECE4F2E484917F012FEF73
:10750000E21AF20A882321F00E94F0F6F701F5CF83
:10751000E6EEF6E084917F013FEFE31AF30A882359
:1075200021F00E94F0F6F701F5CF61E0812F0E9473
:10753000DCB90E94F6B2DC01CB0180529C46AB4F15
:10754000BF4F8093DA049093DB04A093DC04B093E4
:10755000DD041092B80E81E080936914DD24D39489
:1075600080916914882309F47AC060E0812F0E9419
:10757000DCB98091B80E882309F46DC060911115B3
:1075800088E00E9413A9ECE4F2E484917F014FEFBC
:10759000E41AF40A882321F00E94F0F6F701F5CFEF
:1075A000EFEBF6E084917F015FEFE51AF50A88239F
:1075B00021F00E94F0F6F701F5CF8091691488233D
:1075C00021F081E00E94A850F8CF1092DA041092C6
:1075D000DB041092DC041092DD041092B80E0E94BD
:1075E00043630E94C8FC6091111582E00E9413A9B8
:1075F000ECE4F2E484917F019FEFE91AF90A882311
:1076000021F00E94F0F6F701F5CFE3E9F6E084916E
:107610007F01AFEFEA1AFA0A811119C00E94F6B28F
:10762000DC01CB0180529C46AB4FBF4F8093DA0404
:107630009093DB04A093DC04B093DD041092B80EA9
:10764000D092691461E0812F0E94DCB904C00E94CD
:10765000F0F6F701DCCF81E00E94A85081CF80E0F6
:1076600090E0A0EAB1E488A399A3AAA3BBA3809168
:10767000AC0E882359F0212FAE01405E5F4FBE0152
:107680006C5D7F4FCE0188960E946B53013009F0EC
:107690002AC10E94639927C18BE592E00E94CC7BAE
:1076A000811121C185E50E943A908823D9F100918A
:1076B000010510E00E9407906B017C0120E030E0A2
:1076C000A9010F94A60887FF04C0F7FAF094F7F811
:1076D000F094000F111F000F111FF801E95DFB4E20
:1076E000C082D182E282F38200910105B4E00B9F57
:1076F00080011124095D1B4E20E030E048E453E492
:10770000F80160817181828193810F94A608181617
:107710004CF480E090E0A8E4B3E4F8018083918326
:10772000A283B3838CE40E943A90882309F4DBC0DF
:107730000091010510E00E9407906B017C0120E0A0
:1077400030E0A9010F94A60887FF04C0F7FAF0946F
:10775000F7F8F094000F111F000F111FF801E55DFD
:10776000FB4EC082D182E282F38200910105F4E0F7
:107770000F9F80011124055D1B4E20E030E048E49E
:1077800053E4D8016D917D918D919C910F94A60841
:1077900018160CF0A8C080E090E0A8E4B3E4F8016B
:1077A00080839183A283B3839EC01F5F143061F0F6
:1077B000D7018D917D010E943A908823B1F30E94F8
:1077C000D78F812F7BD7F1CF82E40E943A90882314
:1077D00021F00E94D78F84E071D783E50E943A9010
:1077E000882309F480C010E00E94D78F812F66D7CC
:1077F0001F5F1530C9F777C083E50E948190882309
:1078000021F00E94D78F8B0102C000E010E080E5DC
:107810000E948190882321F00E94D78FCB0102C063
:1078200080E090E0B8013BD75EC081E080931E020B
:107830001092200983E50E948190882339F00E94EC
:10784000F88F811150C00E94D0554DC083E50E9431
:107850003A90F7CF0E9445FD46C0F09028050E945F
:10786000D54BFF2029F1ECE4F2E484918F010F5F06
:107870001F4F882321F00E94F0F6F801F6CF84E52F
:107880000E94F0F66F2D70E080E090E04AE00E94E8
:1078900043F780E20E94F0F6E4E2F7E084918F0182
:1078A0000F5F1F4F8823F9F00E94F0F6F801F6CF22
:1078B00010921115ECE4F2E484918F010F5F1F4FD9
:1078C000882321F00E94F0F6F801F6CF609111159F
:1078D00070E082E197E00E94CF688AE00E94F0F6B3
:1078E00002C00E9445FDC257DF4FB881CE58D0403C
:1078F000BB2309F4F3C50E946455F0C50E9487724A
:1079000089E494E00E940F5580917F0E83FDA5C00D
:10791000C0905504D0905604E0905704F09058045D
:107920002091E0053091E1054091E2055091E30599
:10793000C701B6010F941602882309F48EC0609126
:107940008B0970918C0980918D0990918E092091FD
:107950008A09211129C00F94C40720913F02309158
:1079600040026217730704F5C092E005D092E1056A
:10797000E092E205F092E305ECE4F2E484918F01F9
:107980000F5F1F4F882321F00E94F0F6F801F6CF19
:10799000ECE3F2E084918F010F5F1F4F882321F009
:1079A0000E94F0F6F801F6CF8090550490905604AE
:1079B000A0905704B09058042091E0053091E10563
:1079C0004091E2055091E305C501B4010F947F0693
:1079D0006B017C0120E030E0A9010F94A60887FF2D
:1079E00004C0F7FAF094F7F8F094E091111504E070
:1079F000E09FF0011124E55CFD4F2081318142813F
:107A00005381C701B6010F947B0220E030E048E4C7
:107A100053E40F94A608181604F58092E00590929E
:107A2000E105A092E205B092E305ECE4F2E4849172
:107A30008F010F5F1F4F882321F00E94F0F6F8019D
:107A4000F6CFEDE1F2E084918F010F5F1F4F8823A5
:107A500021F00E94F0F6F801F6CF609104027091D7
:107A60000502072E000C880B990B0F941C02209125
:107A700000023091010240910202509103020F94E2
:107A80007B022AE037ED43E25CE30F947B026983DB
:107A90007A838B839C83E090111518A219A21AA2F5
:107AA0001BA29E01205E3F4F69018E010F5F1F4F99
:107AB00025E534E041E554E06DE474E089E494E0C8
:107AC0000E949C9B0E949D900ECF11110C94422A03
:107AD0000C943B2A0E94D78FAB01BC014093C1118B
:107AE0005093C2116093C3117093C41180E191E16E
:107AF0000E94A4CEF8CE812F0E9487BB6E2D812FCD
:107B00000E94C8B1F12CB701812F0E94F7B1163045
:107B100029F4F0928909E0928809E5CE183009F03D
:107B2000E2CEF0928709E0928609DDCE0E94E78FCF
:107B3000853620F084E680938403D5CE8093840339
:107B4000D2CE0E9407900F94C407709313156093D0
:107B5000121580E00E944363609112157091131515
:107B6000072E000C880B990B0F941C0220918B0997
:107B700030918C0940918D0950918E090F94A6087F
:107B8000181634F00CA9011108C082E493E002C079
:107B900086E593E060E00E94539181E08093540277
:107BA0001AAE1BAE1CAE1DAE2C961CAE1DAE1EAE8C
:107BB0001FAE2C971EAA2D961FAE2D971CE32E9656
:107BC0001FAF2E970CE160960FAF609716E4649696
:107BD0001FAF6497C12CD12C80E8E82E9FEBF92EC3
:107BE000412C512C32016091121570911315072E02
:107BF000000C880B990B0F941C021B01182F092FE6
:107C00009B01482F592FB601C7010F9416028823F4
:107C1000B9F020918B0930918C0940918D095091D8
:107C20008E09B101812F902F0F941602881F88278B
:107C3000881F8EAB2CA9222331F0882321F090C11C
:107C400016011E2D0F2D0E94F6B26B017C01DC0186
:107C5000CB012C962CAD3DAD4EAD5FAD2C97821B6C
:107C6000930BA40BB50BB7FD3DC0D701C6018851DE
:107C70009C4FAF4FBF4F2C968CAF9DAFAEAFBFAFF9
:107C80002C970E942568EEE3F3E084915F019FEF5B
:107C9000A91AB90A882321F00E94F0F6F501F5CF60
:107CA0004114510461047104B9F0D301C201885137
:107CB0009C4FAF4FBF4FBC01CD016C197D098E09A0
:107CC0009F0928EE33E040E050E00F942206CA01FD
:107CD000B9010E94A9F703C08FE30E94F0F68AE081
:107CE0000E94F0F680E00E94A8500E94F6B26093D5
:107CF0001304709314048093150490931604A091B8
:107D00008B09AEAFB0918C092396BFAF2397E0915A
:107D10008D092796EFAF2797F0918E092896FFAF30
:107D200028979D01AF01B101812F902F0F947F06FD
:107D30004B015C0120E030E0A9010F94A60887FF09
:107D400004C0B7FAB094B7F8B09420E030E040E255
:107D500051E4C501B401411451046104710429F4D2
:107D60000F94160287FF07C004C00F94A6081816C8
:107D700014F4260137012EA9222309F454C08AAD38
:107D80009BADACADBDAD892B8A2B8B2B61F0D701A0
:107D9000C6012AAD3BAD4CAD5DAD821B930BA40B70
:107DA000B50BB7FD40C02EAD23963FAD2397279668
:107DB0004FAD279728965FAD28972D966FAD2D97DD
:107DC0002E967FAD2E9760968FAD609764969FAD8F
:107DD00064970F947F0620E030E040EC5FE30F945F
:107DE000160287FDBDC0D701C601805A9541AF4F2D
:107DF000BF4F8AAF9BAFACAFBDAF9EAD2D969FAFCF
:107E00002D972396AFAD23972E96AFAF2E9727963B
:107E1000BFAD27976096BFAF60972896EFAD2897C4
:107E20006496EFAF649780915402882309F498C058
:107E3000411451046104710421F46101E12EF02E1A
:107E4000D2CEF8EECF1AF3E0DF0AE108F108C41849
:107E5000D508E608F708F7FE83C0EFCF0E94079029
:107E60000F94C407663971050CF08CC17093070537
:107E7000609306050E94F8626091060570910705FF
:107E8000072E000C880B990B0F941C022091020501
:107E90003091030540910405509105050F94A60803
:107EA00018160CF464C08EE693E060E00E945391D3
:107EB00081E08093540280911115809301051EAAE0
:107EC0001FAA18AE19AE2C961CAE1DAE1EAE1FAE6C
:107ED0002C971CAA2D961FAE2D970CE32E960FAF54
:107EE0002E971CE160961FAF609706E464960FAF73
:107EF0006497C12CD12C10E8E12E0FEBF02E412C11
:107F0000512C32016091060570910705072E000C77
:107F1000880B990B0F941C021B01182F092F9B0132
:107F2000482F592FB601C7010F941602882311F16B
:107F300020910205309103054091040550910505FB
:107F4000B101812F902F0F941602881F8827881F58
:107F50008CAB28962FAD2897222379F0882369F0DF
:107F600080915402882309F4BECC0C94EF2D8DE748
:107F700093E09BCF16011E2D0F2D0E94F6B26B01D0
:107F80007C01DC01CB012C962CAD3DAD4EAD5FAD3F
:107F90002C97821B930BA40BB50BB7FD3DC0D701EB
:107FA000C60188519C4FAF4FBF4F2C968CAF9DAFF1
:107FB000AEAFBFAF2C970E942568EAE6F3E084914C
:107FC0005F019FEFA91AB90A882321F00E94F0F6F9
:107FD000F501F5CF4114510461047104B9F0D301E6
:107FE000C20188519C4FAF4FBF4FBC01CD016C19EE
:107FF0007D098E099F0928EE33E040E050E00F94A0
:108000002206CA01B9010E94A9F703C08FE30E94AA
:10801000F0F68AE00E94F0F680E00E94A8500E94EC
:10802000F6B2609313047093140480931504909334
:108030001604A0910205AAAFB0910305BEAFE0916E
:1080400004052396EFAF2397F09105052796FFAF20
:1080500027979D01AF01B101812F902F0F947F06CB
:108060004B015C0120E030E0A9010F94A60887FFD6
:1080700004C0B7FAB094B7F8B09420E030E040EA1A
:1080800050E4C501B401411451046104710429F4A0
:108090000F94160287FF07C004C00F94A608181695
:1080A00014F4260137012CA9222309F450C08EA90B
:1080B0009FA9A8ADB9AD892B8A2B8B2B61F0D70175
:1080C000C6012EA93FA948AD59AD821B930BA40B45
:1080D000B50BB7FD3CC02AAD3EAD23964FAD2397FF
:1080E00027965FAD27972D966FAD2D972E967FAD76
:1080F0002E9760968FAD609764969FAD64970F94AE
:108100007F0620E030E040EC5FE30F94160287FD2D
:1081100027CFD701C601805A9541AF4FBF4F8EABD5
:108120009FABA8AFB9AF9AAD2D969FAF2D97AEADCF
:108130002E96AFAF2E972396BFAD23976096BFAF15
:1081400060972796EFAD27976496EFAF649780917D
:108150005402882309F404CF4114510461047104CA
:1081600021F46101E12EF02ECDCEF8EECF1AF3E02E
:10817000DF0AE108F108C418D508E608F708F7FE99
:10818000EFCEEFCF66E970E071CE2F964EAD5FADCA
:108190002F97452B09F442C1AB964CAC5DAC6EAC4D
:1081A0007FACAB97480E591E6A1E7B1EAB962CAD5A
:1081B0003DAD4EAD5FADAB97281B390B4A0B5B0B4A
:1081C000CA01B901A50194010F941306A3019201FC
:1081D0000F94440626968CAC9DACAEACBFAC2697F3
:1081E000820E931EA41EB51E34E183169104A104D1
:1081F000B1040CF45AC1C258DF4F88819981AA8119
:10820000BB81CE57D04088169906AA06BB060CF053
:108210005CC1CA57DF4F288139814A815B81C658CA
:10822000D040281539054A055B05ACF426968CAE7E
:108230009DAEAEAEBFAE2697C657DF4F88819981FF
:10824000AA81BB81CA58D04088199909AA09BB09DB
:108250004C015D0106C026968CAE9DAEAEAEBFAEA3
:10826000269726964CAD5DAD6EAD7FAD269787E225
:1082700096E00E94A868B501A40182E296E00E94FF
:10828000A86868964FAD689769965FAD69976A96DA
:108290006FAD6A976B967FAD6B978BE196E00E940E
:1082A000D1676C964FAD6C976D965FAD6D976E967E
:1082B0006FAD6E976F967FAD6F9784E196E00E94E9
:1082C000D1672F96AEADBFAD2F9713970CF4A6C014
:1082D000C501B4010F941C0220E030E040E850E4F6
:1082E0000F947B026B017C0168962FAD68976996AD
:1082F0003FAD69976A964FAD6A976B965FAD6B9786
:108300006C966FAD6C976D967FAD6D976E968FADD9
:108310006E976F969FAD6F970F947F062BED3FE0A2
:1083200049E450E40F947B0220E030E040E05FE35A
:108330000F947B029B01AC01C701B6010F945C074F
:108340006B017C01C301B2010F941C022FE632E1E4
:1083500043E85AE30F947B022B013C01B701A601CD
:108360008EE096E00E94D167B301A20188E096E01A
:108370000E94D1672AE939E949E15FE3C701B60103
:108380000F947B026B017C019B01AC010F94800672
:10839000A30192010F945C0763966CAF7DAF8EAF23
:1083A0009FAF6397A3019201C701B6010F947B02AF
:1083B00020E030E040E05EE30F947B0267966CAF14
:1083C0007DAF8EAF9FAF6797E8EFF5E084913F01F7
:1083D000BFEF6B1A7B0A882321F00E94F0F6F301AD
:1083E000F5CFB701A60182EF95E00E94D1676396B1
:1083F0004CAD5DAD6EAD7FAD63978CEE95E00E94A8
:10840000D16767964CAD5DAD6EAD7FAD679786EE7B
:1084100095E00E94D1678AE00E94F0F626968CAD26
:108420009DADAEADBFAD2697880D991DAA1DBB1D94
:10843000ECA9B595A79597958795E7FF03C080931D
:10844000000505C0EE96EEADFFADEE9780832F964A
:108450002EAD3FAD2F972F5F3F4F2F963FAF2EAFE3
:108460002F9727963FAD279768963FAF6897289636
:108470004FAD289769964FAF699729965FAD2997B9
:108480006A965FAF6A972D968FAD2D976B968FAFDB
:108490006B9722964CAC5DAC6EAC7FAC229791E0B2
:1084A000A2969FAFA2970C942E3684E1882E912C31
:1084B000A12CB12C24E130E040E050E026962CAF16
:1084C0003DAF4EAF5FAF2697CCCECE57DF4F888003
:1084D0009980AA80BB80C258D040A8CECA56DF4F30
:1084E0000FB6F894DEBF0FBECDBFDF91CF911F91C5
:1084F0000F91FF90EF90DF90CF90BF90AF909F9043
:108500008F907F906F905F904F903F902F90089545
:10851000CF93DF938091DB0E9091DC0E891B8F70DF
:1085200009F445C09091D80E992351F0833030F46E
:108530008FEF890F19F08093D80E3BC01092D80EA0
:10854000E091DC0E8FE4E89FF0011124E157F64F33
:10855000808180FD2EC08091650990916609A0916F
:108560006709B0916809EF01C55BDF4F4881598108
:108570006A817B81841B950BA60BB70B80936509E1
:1085800090936609A0936709B09368098091DC0E07
:108590008F5F8F708093D90E9091DC0E8091DA0EF0
:1085A00098130AC08091D90E8093DA0E05C00E94FC
:1085B000096280E090E001C0CF01DF91CF91089582
:1085C00067FD3BC08230D9F028F4882341F0813028
:1085D00061F033C08330E9F0843029F12EC0662386
:1085E00011F0A19A39C0A19837C08091080161119A
:1085F000809580788093060147FF36C0089580916A
:1086000008016111809580748093060147FF32C094
:10861000089580910801611180958870809306010A
:1086200047FF2EC0089580910801611180958270E6
:108630008093060147FF2AC0089547FD2FC082306E
:10864000C9F028F4882351F0813071F00895833007
:10865000B9F08430D9F0089547FD20C0442311F0CB
:10866000A09A0895A0980895442311F0A29A08951D
:10867000A2980895809108014111809580720BC0E5
:108680008091080141118095807105C08091080199
:1086900041118095847080930601089508955F9834
:1086A0008EBD00000DB407FEFDCF8EB56EBD00007F
:1086B0000DB407FEFDCF8EB55F9A0895CF93DF937B
:1086C00000D01F921F92CDB7DEB795E0E5E5F2E04E
:1086D000DE01119601900D929A95E1F7E1E0F0E04C
:1086E000EC0FFD1FE80FF11D808190E00F900F90BF
:1086F0000F900F900F90DF91CF91D1CF90916F009D
:1087000091FB222720F991FF05C090916F009D7F7A
:1087100090936F0034E0839FC0011124FC01EC5E54
:10872000FA4E4081518162817381FC01EB50FC4F14
:10873000408351836283738381E08093F403222317
:1087400029F080916F00826080936F00089590916E
:108750006F0091FB222720F991FF05C090916F00D7
:108760009D7F90936F0094E0899FF0011124EC5E4F
:10877000FA4E6081718182819381222329F02091B8
:108780006F00226020936F000895BC012091F203D6
:108790003091F3034091F2035091F303241735070E
:1087A00011F09A01F7CF81E06217730709F080E0BA
:1087B00008950F930FB70F9300916E000F930B7FE7
:1087C00000936E0000916F000D7F00936F000F9378
:1087D0000BB70F930CB70F921F922F933F934F93AA
:1087E0005F936F937F938F939F93AF93BF93EF9319
:1087F000FF93112471D0FF91EF91BF91AF919F91A1
:108800008F917F916F915F914F913F912F911F9029
:108810000F900CBF0F910BBF0F910260F894009363
:108820006F000F9100936E000F910FBF0F9118957D
:108830008091AA0380FF07C080910B018270809312
:1088400009018FEF07C080910B01809582708093A2
:10885000090181E08093A6038091AA0381FF08C0EB
:1088600080910B0180958170809309018FEF06C084
:1088700080910B0181708093090181E08093A703AF
:108880008091AA0382FF07C080910B0184708093BE
:1088900009018FEF07C080910B0180958470809350
:1088A000090181E08093A8038091AA0383FF08C097
:1088B00080910B0180958074809309018FEF06C031
:1088C00080910B0180748093090181E08093A9035A
:1088D00000000000000008953F924F925F926F9257
:1088E0007F928F929F92AF92BF92CF92DF92EF9240
:1088F000FF920F931F93CF93DF93F8948FEF9FEF27
:108900009093890080938800EAE03E2E00E010E01A
:1089100078948091EE039091EF03A091F003B091D1
:10892000F103892B8A2B8B2B09F0CDC18091F403A5
:108930008823D1F01092F4038091F2039091F30315
:10894000892B91F01092E5031092F3031092F20339
:108950009091DB0E8091DC0E981731F08091DC0E47
:108960008F5F8F708093DC0E8091F2039091F30300
:10897000892B09F4A8C14091EA035091EB0360915F
:10898000EC037091ED039091D803C090E603D09072
:10899000E703E090E803F090E903C41AD50AE60A79
:1089A000F70A892F90E0A0E0B0E0C816D906EA06E1
:1089B000FB0610F4D701C601282F840F951FA61FB0
:1089C000B71F8093EA039093EB03A093EC03B0935B
:1089D000ED0380918400909185004E96C090C00375
:1089E000D090C103E090C203F090C3034091B00364
:1089F0005091B1036091B2037091B3034C0D5D1DB2
:108A00006E1D7F1D4093C0035093C1036093C2034A
:108A10007093C30377FD1CC0409AC0901415D0908A
:108A20001515E0901615F09017154091A603042E29
:108A3000000C550B660B770B4C0D5D1D6E1D7F1DDD
:108A400040931415509315156093161570931715D0
:108A5000C090C403D090C503E090C603F090C70354
:108A60004091B4035091B5036091B6037091B70380
:108A70004C0D5D1D6E1D7F1D4093C4035093C503B7
:108A80006093C6037093C70377FD1CC0419AC090E2
:108A90001815D0901915E0901A15F0901B154091FB
:108AA000A703042E000C550B660B770B4C0D5D1DB8
:108AB0006E1D7F1D409318155093191560931A155C
:108AC00070931B15C090C803D090C903E090CA03EF
:108AD000F090CB034091B8035091B9036091BA0371
:108AE0007091BB034C0D5D1D6E1D7F1D4093C8032F
:108AF0005093C9036093CA037093CB0377FD1CC0E6
:108B0000429AC0901C15D0901D15E0901E15F09053
:108B10001F154091A803042E000C550B660B770B14
:108B20004C0D5D1D6E1D7F1D40931C1550931D1532
:108B300060931E1570931F15C090CC03D090CD0389
:108B4000E090CE03F090CF034091BC035091BD0361
:108B50006091BE037091BF034C0D5D1D6E1D7F1DA6
:108B60004093CC035093CD036093CE037093CF0317
:108B700077FD1CC0439AC0902015D0902115E0903D
:108B80002215F09023154091A903042E000C550BDB
:108B9000660B770B4C0D5D1D6E1D7F1D40932015E0
:108BA00050932115609322157093231540918400F2
:108BB0005091850048175907C8F34091C003509160
:108BC000C1036091C2037091C30377FD15C0C090CB
:108BD000AC03D090AD03E090AE03F090AF034C191E
:108BE0005D096E097F094093C0035093C1036093F0
:108BF000C2037093C30340984091C4035091C503CE
:108C00006091C6037091C70377FD15C0C090AC0397
:108C1000D090AD03E090AE03F090AF034C195D0926
:108C20006E097F094093C4035093C5036093C60344
:108C30007093C70341984091C8035091C903609154
:108C4000CA037091CB0377FD15C0C090AC03D090E0
:108C5000AD03E090AE03F090AF034C195D096E09CF
:108C60007F094093C8035093C9036093CA0370936C
:108C7000CB0342984091CC035091CD036091CE0339
:108C80007091CF0377FD15C0C090AC03D090AD03B9
:108C9000E090AE03F090AF034C195D096E097F09B7
:108CA0004093CC035093CD036093CE037093CF03D6
:108CB0004398215041F0409184005091850048171D
:108CC0005907C8F38ACE8091EE039091EF03A091EB
:108CD000F003B091F103892B8A2B8B2B09F01AC377
:108CE000E091F203F091F303309739F18091EA03B8
:108CF0009091EB03A091EC03B091ED034091E6035A
:108D00005091E7036091E8037091E9038417950798
:108D1000A607B707C8F01092E5031092F30310926C
:108D2000F2039091DB0E8091DC0E981731F0809168
:108D3000DC0E8F5F8F708093DC0E70EDC72E77E0B6
:108D4000D72EE12CF12C4FC14091E1035091E20369
:108D50006091E3037091E403481759076A077B07A2
:108D600008F467C08091DD039091DE03A091DF03DA
:108D7000B091E00342A953A964A975A9CC27859FA6
:108D8000D12D969F9001A69F300DA59F200D311DDE
:108D9000869FD00D211D3C1F959FD00D211D3C1F8E
:108DA000A49FD00D211D3C1F949FD10D2C1F3C1F53
:108DB000D6952C1F3C1F789F200D311D799F300DBB
:108DC000112443AD54AD65AD76AD420F531F611D07
:108DD000711D4093D9035093DA036093DB037093C2
:108DE000DC03C7A8D0ACE1ACF2ACC416D506E606ED
:108DF000F70640F4C092D903D092DA03E092DB0385
:108E0000F092DC03C090D903D090DA03E090DB034A
:108E1000F090DC0326E33FE041E0F9018590959076
:108E2000A590B4908C149D04AE04BF0408F4B9C29C
:108E3000C4C24091D4035091D5036091D603709180
:108E4000D703481759076A077B0708F063C080916A
:108E5000D0039091D103A091D203B091D30342A942
:108E600053A964A975A9CC27859FD12D969F900100
:108E7000A69F300DA59F200D311D869FD00D211D71
:108E80003C1F959FD00D211D3C1FA49FD00D211D7F
:108E90003C1F949FD10D2C1F3C1FD6952C1F3C1FAF
:108EA000789F200D311D799F300D11244901A12C8F
:108EB000B12CC090D903D090DA03E090DB03F0909E
:108EC000DC03FF968C149D04AE04BF0480F4408143
:108ED000518162817381C818D908EA08FB08C41659
:108EE000D506E606F70638F46A017B0104C0C080A7
:108EF000D180E280F38026E33FE041E0F9018590F4
:108F00009590A590B4908C149D04AE04BF0408F411
:108F1000BDC2C8C28091090290910A02A0910B02C1
:108F2000B0910C02B7FF57C087A990ADA1ADB2AD0B
:108F300026E33FE041E0F901C590D590E590F4903B
:108F4000C816D906EA06FB0658F4B695A795979574
:108F50008795440F2C5F3F4FFFE022353F0759F7BD
:108F60004093D80380329105A105B10508F428C3C8
:108F70008097A109B109811528E09207A105B105E3
:108F800008F4F9C244E0949FF00111249F012A5C87
:108F9000344FF901329645915491EE27859FB001E7
:108FA000849F610D7E1F06946E1F7E1F1124AB01EE
:108FB00060E070E0F90185919491A0E0B0E0841B3D
:108FC000950BA60BB70B8093090290930A02A0930E
:108FD0000B02B0930C02C0900902D0900A02E090FC
:108FE0000B02F0900C028091F2039091F303892B15
:108FF00009F088C18DDA9093F3038093F203892BF3
:1090000009F480C1C091F203D091F303888183FFFA
:109010003EC08D899E89AF89B88D80931415909339
:109020001515A0931615B0931715898D9A8DAB8DD4
:10903000BC8D8093181590931915A0931A15B093B1
:109040001B158D8D9E8DAF8DB8A180931C159093AF
:109050001D15A0931E15B0931F1589A19AA1ABA150
:10906000BCA18093201590932115A0932215B09355
:1090700023159091DB0E8091DC0E981709F4BACF7E
:109080008091DC0E8F5F8F708093DC0EB3CF8D8864
:109090009E88AF88B88C81E081149104A104B1044A
:1090A00009F480E0C98CDA8CEB8CFC8CC114D104FF
:1090B000E104F10409F082604D8D5E8D6F8D78A121
:1090C000411551056105710509F084608093E50340
:1090D0001092D0031092D1031092D2031092D303B6
:1090E0001092DD031092DE031092DF031092E00372
:1090F0008DA19EA1AFA1B8A58093E6039093E7034D
:10910000A093E803B093E903442455243201481A9C
:10911000590A6A0A7B0A4092CC035092CD036092AE
:10912000CE037092CF034092C8035092C90360925D
:10913000CA037092CB034092C4035092C50360925D
:10914000C6037092C7034092C0035092C10360925D
:10915000C2037092C303880C991CAA1CBB1C80928A
:10916000B0039092B103A092B203B092B303CC0CBF
:10917000DD1CEE1CFF1CC092B403D092B503E0923C
:10918000B603F092B703440F551F661F771F409335
:10919000B8035093B9036093BA037093BB0349A11A
:1091A0005AA16BA17CA1440F551F661F771F4093E6
:1091B000BC035093BD036093BE037093BF03880F3D
:1091C000991FAA1FBB1F8093AC039093AD03A0937C
:1091D000AE03B093AF031092EA031092EB03109228
:1091E000EC031092ED038AA59BA5ACA5BDA58093C9
:1091F000E1039093E203A093E303B093E4038EA50D
:109200009FA5A8A9B9A98093D4039093D503A0934F
:10921000D603B093D70389A58093AB039EA9209171
:10922000AA0392130AC02091080230E0482F082EAA
:10923000000C550B4217530729F09093AA03809313
:109240000802F6DA0E9499988FEF9FEFDC01809375
:10925000090290930A02A0930B02B0930C028BAD0B
:109260009CADADADBEAD8093D9039093DA03A093CE
:10927000DB03B093DC0326E33FE041E0F901C59056
:10928000D590E590F490C816D906EA06FB0658F486
:10929000B695A79597958795440F2C5F3F4F5FE054
:1092A0002235350759F74093D80380329105A1053F
:1092B000B10508F4ADC18097A109B1098115F8E0A5
:1092C0009F07A105B10508F480C144E0949F900177
:1092D00011242A5C344FF901329645915491EE27BE
:1092E000859FB001849F610D7E1F06946E1F7E1FB7
:1092F0001124F901C590D490E12CF12CC61AD70A9B
:10930000E108F108C092EE03D092EF03E092F0037F
:10931000F092F1038091EE039091EF03A091F0039E
:10932000B091F103AC01BD010097F1E0AF07B105C9
:1093300020F04FEF5FEF60E070E0841B950BA60B11
:10934000B70B8093EE039093EF03A093F003B093D9
:10935000F103F894809184009091850040963A94AE
:10936000332039F0040F151F0817190708F4D0CA65
:1093700001C08C0110938900009388007894DF91DC
:10938000CF911F910F91FF90EF90DF90CF90BF9002
:10939000AF909F908F907F906F905F904F903F9095
:1093A0000895F694E794D794C794440F2C5F3F4FE9
:1093B0005FE02235350709F030CD4093D80320E235
:1093C000C216D104E104F10408F45AC020E2C21A22
:1093D000D108E108F108C11448E0D406E104F10421
:1093E000F8F054E0D59E900111242A5C344FF90125
:1093F000329645915491FC2DEE27F59FB001F49FD4
:10940000610D7E1F06946E1F7E1F1124F901C59009
:10941000D490E12CF12CC61AD70AE108F10823C038
:10942000B701A6017695679557954795FA01EC7FA8
:10943000AF014A5C584FFA0125913491FA013296F6
:1094400065917491EC2DE770E69FA001E79F500DA8
:10945000112463E0569547956A95E1F7241B350B77
:109460006901E12CF12C8C0D9D1DAE1DBF1D80935B
:10947000DD039093DE03A093DF03B093E003B3CD4D
:10948000C0E2CC2ED12CE12CF12CA0CFF694E794A5
:10949000D794C794440F2C5F3F4F5FE022353507C8
:1094A00009F02CCD4093D803F0E2CF16D104E104AB
:1094B000F10408F45AC020E2C21AD108E108F10808
:1094C000C11448E0D406E104F104F8F054E0D59E5C
:1094D000900111242A5C344FF90132964591549140
:1094E000FC2DEE27F59FB001F49F610D7E1F0694C1
:1094F0006E1F7E1F1124F901C590D490E12CF12C30
:10950000C61AD70AE108F10823C0B701A60176956B
:10951000679557954795FA01EC7FAF014A5C584F24
:10952000FA0125913491FA01329665917491EC2DEE
:10953000E770E69FA001E79F500D1124D3E05695F8
:109540004795DA95E1F7241B350B6901E12CF12CE5
:109550008C0D9D1DAE1DBF1D8093D0039093D10334
:10956000A093D203B093D3033ECDE0E2CE2ED12C14
:10957000E12CF12CA0CFAC01BD01769567955795F4
:109580004795FA01EC7FAF014A5C584FFA012591EB
:109590003491FA013296459154918770849FB001BD
:1095A000859F700D1124CB01F3E096958795FA9570
:1095B000E1F7D901A81BB90BCD01A0E0B0E003CDC4
:1095C00080E290E0A0E0B0E0D3CCAC01BD017695A4
:1095D000679557954795FA01EC7F9F012A5C384FB4
:1095E000F901C590D490F901329625913491877094
:1095F000829FA001839F500D1124CA0123E09695FC
:1096000087952A95E1F7C81AD90AE12CF12C7ACE70
:1096100080E290E0A0E0B0E04ECE8F929F92AF92B9
:10962000BF92CF92DF92EF92FF920F931F93CF934F
:10963000DF9300D01F92CDB7DEB783E5882E84E19B
:10964000982E90E8A92E9EE0B92E05E319E0C12CD2
:10965000D12C7601C394F401619171918191919122
:109660004F01F50121913191419151915F01298380
:109670003A834B835C830F941A0229813A814B8190
:109680005C810F947B020F94C907F8016193719379
:10969000819391938F01C616D706E806F90610F458
:1096A0006B017C01F3E68F16F4E19F06A1F66FEFE4
:1096B0007FEFCB01A70196010F9422062093450965
:1096C0003093460940934709509348090F900F90F3
:1096D0000F900F90DF91CF911F910F91FF90EF901E
:1096E000DF90CF90BF90AF909F908F900895809122
:1096F000DB0E9091DC0E891B8F708F3019F480E0A7
:1097000027D5F5CF8091DB0E8F5F8F70E091DB0E58
:109710009FE49E9FF0011124E157F64FDF011D9257
:109720009A95E9F798E090834091F10E5091F20EEE
:109730006091F30E7091F40E458B568B678B708F92
:109740004091F50E5091F60E6091F70E7091F80E63
:10975000418F528F638F748F4091F90E5091FA0EA2
:109760006091FB0E7091FC0E458F568F678F70A332
:109770004091FD0E5091FE0E6091FF0E7091000F12
:1097800041A352A363A374A32091DB0E9091DC0E3E
:10979000291303C094E69093D80E8093DB0E80913A
:1097A0006F00826080936F0008959091DB0E80912E
:1097B000DC0E981719F080E0CBD4F7CF8091900E93
:1097C0009091910E892BB9F70895EF92FF920F9324
:1097D0001F93CF93DF937B018A01E9012091800ED3
:1097E0003091810E4091820E5091830EFC01608178
:1097F0007181828193810F947B020F94B1086093F1
:10980000F10E7093F20E8093F30E9093F40E20916C
:10981000840E3091850E4091860E5091870EF7018F
:1098200060817181828193810F947B020F94B108D2
:109830006093F50E7093F60E8093F70E9093F80EEA
:109840002091880E3091890E40918A0E50918B0E96
:10985000F80160817181828193810F947B020F9462
:10986000B1086093F90E7093FA0E8093FB0E9093FB
:10987000FC0E20918C0E30918D0E40918E0E5091E9
:109880008F0E688179818A819B810F947B020F946E
:10989000B1086093FD0E7093FE0E8093FF0E9093BF
:1098A000000F9091DB0E8091DC0E981739F0DF915C
:1098B000CF911F910F91FF90EF9019CF76DF80919C
:1098C0006F0081FB992790F981FF05C080916F009F
:1098D0008D7F80936F004091F10E5091F20E609158
:1098E000F30E7091F40E4093141550931515609378
:1098F0001615709317154091F50E5091F60E609164
:10990000F70E7091F80E4093181550931915609347
:109910001A1570931B154091F90E5091FA0E609133
:10992000FB0E7091FC0E40931C1550931D15609317
:109930001E1570931F154091FD0E5091FE0E609103
:10994000FF0E7091000F40932015509321156093E6
:10995000221570932315992329F080916F0082605E
:1099600080936F00DF91CF911F910F91FF90EF9047
:1099700008950F931F93CF93DF93C0E8DEE00DE6C9
:1099800019E0299139914991599160E070E080E89E
:109990009FE30F945C07F801619371938193919316
:1099A0008F01FEE0C039DF0761F720EE35E04CEDB6
:1099B00055E068ED75E084ED95E007DFDF91CF912C
:1099C0001F910F912ACE9091DB0E8091DC0E98179B
:1099D00019F080E0BDD3F7CF8091900E9091910E59
:1099E000892BB9F741C3CF93DF9390916F0091FB1F
:1099F000222720F991FF05C090916F009D7F9093E1
:109A00006F0094E0899FE0011124FE01EB50FC4FB0
:109A10006081718182819381222329F020916F00DE
:109A2000226020936F000F941C02C359D64F2881E7
:109A300039814A815B810F947B02DF91CF91089538
:109A4000CF92DF92EF92FF9280916714882371F199
:109A5000C0906314D0906414E0906514F090661484
:109A600020E030E0A901C701B6010F941602882357
:109A7000E9F020E030E040E05FE3C701B6010F9479
:109A80007B029B01AC010F947B022BED3FE049E48C
:109A900050E40F947B029B01AC0160E070E080E831
:109AA0009FE30F945C076B017C0106C0C12CD12C95
:109AB00080E8E82E8FE3F82EC092A203D092A30391
:109AC000E092A403F092A503609106027091070250
:109AD000072E000C880B990B0F941C022AE037ED1F
:109AE00043E25CE30F947B02A70196010F947B0293
:109AF00060933B0270933C0280933D0290933E0240
:109B0000FF90EF90DF90CF9008950F931F93CF9326
:109B1000DF938B01EA01DB016D917C9104960E9439
:109B200094D4D801ED91FC919081888191110EC05F
:109B30008D38B0F48FE28083F801808191810196A5
:109B40009183808388818F5F88830AC08D3880F7F6
:109B50003196D801ED93FC9388818F5F8883E1CFA4
:109B6000DF91CF911F910F910895FC0120E03EE21B
:109B7000DB014C91403241F0283011F430833196B2
:109B8000DB014C91408331962F5F6F5F7F4F2B300D
:109B900079F7108208958F929F92AF92BF92CF92E1
:109BA000DF92EF92FF920F931F93CF93DF93CDB786
:109BB000DEB728970FB6F894DEBF0FBECDBF6C019D
:109BC0005B017A01022FEEEAF0E184914F019FEFF1
:109BD000891A990A882321F00E94F0F6F401F5CF42
:109BE00080917F0E83FD42C020E030E0A901F701A3
:109BF00060817181828193810F9416028823B1F173
:109C0000209112153091131510918A0911112EC04F
:109C100080913F0290914002281739073CF5E4E417
:109C2000F9E484917F019FEFE91AF90A882321F072
:109C30000E94F0F6F701F5CFEDE9F0E184917F01A4
:109C40009FEFE91AF90A882321F00E94F0F6F70144
:109C5000F5CF002329F06091111587E00E9413A928
:109C600060E08EE890E10E945391C2C08091AC0EFA
:109C700091E0980F9093AC0E9091210F992329F0C9
:109C80001092210F8E5F8093AC0E0E944E9980E15E
:109C9000E4EDF5E0A9E5B4E001900D928A95E1F7D5
:109CA00084DD20E030E0A901F601608171818281CC
:109CB00093810F941602882319F160918B0970919A
:109CC0008C0980918D0990918E0920918A0921112A
:109CD00009C00F94C40720913F02309140026217DF
:109CE000730774F080E090E0A0E2B1E489839A8386
:109CF000AB83BC83BE016F5F7F4FC6010E9467BA12
:109D00000E94B8FB811107C082E08983B501CE01B2
:109D100001960E945AF620E030E0A901F701608127
:109D20007181828193810F941602882361F00E94D1
:109D3000C8FC182F811109C0002329F0609111156A
:109D400087E00E9413A911E053C0002329F060911D
:109D5000111581E00E9413A980E090E0A0E8BFE324
:109D60008D839E83AF83B88780E090E0A0ECB0E461
:109D700089839A83AB83BC83BE016B5F7F4FCE0127
:109D800001960E9467BA8090510990905209A09064
:109D90005309B090540980E090E0A8ECB1E48093BE
:109DA000510990935209A0935309B093540980E04C
:109DB00090E0A0EAB0E489839A83AB83BC83BE01C0
:109DC0006F5F7F4FC7010E9467BA809251099092DE
:109DD0005209A0925309B092540980911115811132
:109DE00001C0149A64E670E080E090E00E94DE6EAC
:109DF000812F28960FB6F894DEBF0FBECDBFDF913E
:109E0000CF911F910F91FF90EF90DF90CF90BF9077
:109E1000AF909F908F9008954F925F926F927F9234
:109E20008F929F92AF92BF92DF92EF92FF920F9329
:109E30001F93CF93DF93D82EC82FD0E0FE01E35BB2
:109E4000FF4E64917E01EE0CFF1CEE0CFF1CF7012F
:109E5000EF5BFF4E4590559065907490062E000C78
:109E6000770B880B990B0F941C024B015C0120E0CF
:109E700030E040EC5FE3C301B2010F947B02A50127
:109E800094010F947B02AB01BC0100E010E098014B
:109E90008D2D0E947C78F701EB5CFF4E259135916A
:109EA00045915491C501B4010F947B024B015C01B3
:109EB00020E030E0A9010F941602882309F448C07D
:109EC00000E010E09801B501A40170588D2D0E94AA
:109ED0007C78FE01EE5CFF4E4491411117C0ECE42A
:109EE000F2E48491EF012196882321F00E94F0F69C
:109EF000FE01F7CFE0E1F0E18491EF0121968823A4
:109F000021F00E94F0F6FE01F7CF4AE0F701E050A1
:109F1000F04F4590559065907490642F70E080E00C
:109F200090E00F941C029B01AC01C301B2010F949D
:109F30005C072B013C01A5019401C501B4010F94FC
:109F40008006AB01BC01930182018D2D0E947C78BB
:109F500081E090E00D2C01C0880F0A94EAF79091FF
:109F60002415982B9093241590914804892B809365
:109F70004804F701E45CFB4F1082118212821382C5
:109F80008D2D0E948C7BF701EC50F04F85919591BF
:109F9000A591B491E701CC52DA4F88839983AA83C3
:109FA000BB830E94BD8FF701E75BFB4F88819981DE
:109FB000AA81BB8180839183A283B383DF91CF91F8
:109FC0001F910F91FF90EF90DF90BF90AF909F9007
:109FD0008F907F906F905F904F9008950F931F9395
:109FE000CF93DF938C01ECE4F2E48491EF012196AE
:109FF000882321F00E94F0F6FE01F7CFB80187EE2A
:10A000009FE00E94E86882E20E94F0F68AE00E94E7
:10A01000F0F681E0DF91CF911F910F910895CF93DA
:10A02000DF938CE091E118D082EB9FE0892B41F423
:10A0300083E99FE011D084E79FE0DF91CF910CC0CE
:10A04000C0E0D0E0CE0187539F4E06D06F97CA3C48
:10A050008EEFD807B9F7ECCF22E733E0FC0131836C
:10A06000208304960C948D90179A809124158E7FEE
:10A0700080932415169A809124158D7F8093241542
:10A08000159A809124158B7F80932415149A089536
:10A090008C01E4E4F9E48491EF012196882321F016
:10A0A0000E94F0F6FE01F7CFE7ECFFE08491EF01AC
:10A0B0002196882321F00E94F0F6FE01F7CF0E943E
:10A0C0008E63D2DF0E94149561E0C8010E94539113
:10A0D0000E94C95BC091D111C695C6950E9412BD60
:10A0E000DC2FDD0F1D2F1C0F84E00E94E5971092DE
:10A0F0000712C09308120E9403BD10920712D0935A
:10A10000081288EB9FE00E94EDBC1092071210939A
:10A1100008128BEA9FE00E94EDBC0E94A6BB811151
:10A12000E3CF2FEF8BE49DE1215080409040E1F799
:10A1300000C00000F8942FEF84E39CE021508040A1
:10A140009040E1F700C000000E948E63A895FECF0A
:10A150008F929F92AF92BF92CF92DF92EF92FF9237
:10A160000F931F93CF93DF93C82F0E94B4918091D8
:10A17000CE07853010F40E940E7C0E94F6B2C0908B
:10A180001704D0901804E0901904F0901A04C11438
:10A19000D104E104F10469F1009113041091140455
:10A1A00020911504309116040C0D1D1D2E1D3F1D10
:10A1B0006B017C01C01AD10AE20AF30AF7FC19C04C
:10A1C000E4E4F9E48491EF012196882321F00E94D0
:10A1D000F0F6FE01F7CF60910F157091101581E731
:10A1E0009FE00E94E8688AE00E94F0F688E69FE01F
:10A1F0004FDFC0901A02D0901B02E0901C02F0903A
:10A200001D02C114D104E104F104E1F13091DB0E2F
:10A210002091DC0E321749F06093130470931404FC
:10A2200080931504909316042DC02091AC0E21113B
:10A2300029C0C11127C0009113041091140420916A
:10A240001504309116040C0D1D1D2E1D3F1DDC0143
:10A25000CB01801B910BA20BB30BB7FD13C0179A58
:10A26000809124158E7F80932415169A8091241551
:10A270008D7F80932415159A809124158B7F809370
:10A280002415149A0E94F6B2009107041091080454
:10A290002091090430910A046B017C01C01AD10A93
:10A2A000E20AF30AF7FC4AC08B019C010C53164FDB
:10A2B0002F4F3F4F00930704109308042093090485
:10A2C00030930A04079BB6C0069BB4C0059BB2C07E
:10A2D000209100052111AEC0049BACC00091030485
:10A2E0001091040420910504309106040115110514
:10A2F0002105310599F0DC01CB01801B910BA20BEC
:10A30000B30B80569A4EA109B1098827B7FD8395F2
:10A310009927AA27BB27682F619501C060E0862F87
:10A3200090E09093020480930104662311F0749AE4
:10A3300001C07498BC0182E00E94F7B19091DB0EDD
:10A340008091DC0E981305C0D0918609C0918809D0
:10A350001AC0E091DC0E8FE48E9FF0011124EA52C6
:10A36000F64FD081E091DC0E8E9FF0011124E8526F
:10A37000F64FC0818091DC0E9091DB0E891719F0A9
:10A380008F5F8F70F9CFDD2329F10E94F6B2009123
:10A390000B0410910C0420910D0430910E04DC018B
:10A3A000CB01011511052105310569F48C599F4F29
:10A3B000AF4FBF4F80930B0490930C04A0930D04F8
:10A3C000B0930E046FC1801B910BA20BB30BB7FFB0
:10A3D0006AC168C110920B0410920C0410920D0413
:10A3E00010920E04CC2309F46DC00E94F6B20091C5
:10A3F0000F04109110042091110430911204DC011B
:10A40000CB01011511052105310569F48C599F4FC8
:10A41000AF4FBF4F80930F0490931004A09311048B
:10A42000B093120410C0801B910BA20BB30BB7FFAB
:10A430000BC009C060930304709304048093050467
:10A44000909306044BCFCFEFDD2309F425C18D2F68
:10A4500090E0A0E0B0E09C01AD012150310941093C
:10A460005109A9EBB0E00F9460062EEF30E040E018
:10A4700050E00F944406CA01B9016A5B7F4F8F4FC9
:10A480009F4F88E00E94F7B1CC2349F18C2F90E0D8
:10A49000A0E0B0E09C01AD01215031094109510912
:10A4A000A9EBB0E00F9460062EEF30E040E050E002
:10A4B0000F944406DA01C9018A5B9F4FAF4FBF4F2B
:10A4C000BC010FC010920F041092100410921104DE
:10A4D0001092120460E070E088E00E94F7B160E042
:10A4E00070E086E00E94F7B10E942E66C091B3052D
:10A4F000C13009F08DC080912F0481110CC00E94E1
:10A50000F6B260932B0470932C0480932D049093E7
:10A510002E04C0932F048091230481110DC00E944A
:10A52000F6B260931F0470932004809321049093EB
:10A53000220481E0809323040E94F6B26B017C0127
:10A5400080912B0490912C04A0912D04B0912E04A5
:10A55000A7019601281B390B4A0B5B0BDA01C901D5
:10A5600080319742A105B105A0F180901B04909025
:10A570001C04A0901D04B0901E040E941A996093C0
:10A580001B0470931C0480931D0490931E0400917F
:10A59000B9051091BA052091BB053091BC05081989
:10A5A00019092A093B09DC01CB01800F911FA21F69
:10A5B000B31F8093B9059093BA05A093BB05B093E0
:10A5C000BC05C0922B04D0922C04E0922D04F09292
:10A5D0002E0480911F0490912004A0912104B09139
:10A5E0002204A7019601281B390B4A0B5B0BDA01E9
:10A5F000C90180389E4EA105B10550F0C0921F04DC
:10A60000D0922004E0922104F09222040E94B39997
:10A6100081E09FE00E943197C0913B04CC2309F474
:10A620004DC00E94F6B20091370410913804209179
:10A63000390430913A04DC01CB01801B910BA20B51
:10A64000B30BB7FD3BC00E94F6B26B017C012C2F0F
:10A6500030E0A8EEB3E00F947006DC01CB018C0D66
:10A660009D1DAE1DBF1D8093370490933804A093A9
:10A670003904B0933A040E9425688AE0DF91CF91B3
:10A680001F910F91FF90EF90DF90CF90BF90AF9010
:10A690009F908F900C94F0F660E070E088E00E944C
:10A6A000F7B1F4CEDFEFC111A0CE10920F041092DB
:10A6B00010041092110410921204C9CEDF91CF91B0
:10A6C0001F910F91FF90EF90DF90CF90BF90AF90D0
:10A6D0009F908F9008958F929F92AF92BF92CF924A
:10A6E000DF92EF92FF920F931F93CF93DF9300D0EF
:10A6F0001F92CDB7DEB75C016B017A01922E1091EB
:10A70000B80E1092DA041092DB041092DC0410925E
:10A71000DD041092B80E80E00E94436320E030E038
:10A72000A901F70160817181828193810F941602E2
:10A73000882309F4DCC0111116C060918B09709157
:10A740008C0980918D0990918E0920918A0921119F
:10A750000AC00F94C40720913F0230914002621753
:10A7600073070CF4C4C00E94C8FC811106C060913C
:10A77000111587E00E9413A9BAC0111121C0609180
:10A78000111583E00E9413A920E030E0A901F50132
:10A7900060817181828193810F941602882309F46C
:10A7A0003FC080E090E0A0ECB0E489839A83AB8363
:10A7B000BC83BE016F5F7F4FC5010E9467BA30C086
:10A7C0006091111582E00E9413A9ECE4F2E48491F7
:10A7D0008F010F5F1F4F882321F00E94F0F6F801D0
:10A7E000F6CFE0E5F0E184918F010F5F1F4F8823E2
:10A7F00021F00E94F0F6F801F6CF61E0892D0E9469
:10A80000DCB981E08093691480916914882309F48C
:10A81000B6CF60E0892D0E94DCB981E099DCF4CFED
:10A8200020E030E0A901F60160817181828193818D
:10A830000F941602882351F180905109909052098B
:10A84000A0905309B090540980E090E0A8ECB1E4E6
:10A850008093510990935209A0935309B0935409DE
:10A8600080E090E0A0E8BFE389839A83AB83BC8358
:10A87000BE016F5F7F4FC6010E9467BA8092510987
:10A8800090925209A0925309B0925409812C912CB4
:10A8900080E8A82E8FE3B82E20E030E0A901F70170
:10A8A00060817181828193810F94A60818167CF4CF
:10A8B0006091111584E00E9413A989829A82AB826B
:10A8C000BC82BE016F5F7F4FC7010E9467BA1092C2
:10A8D00069146091111585E00E9413A980911D09EA
:10A8E000811103C081E034DCF9CF8130A9F260919D
:10A8F000111586E00E9413A920E030E0A9016091C3
:10A9000065047091660480916704909168040F94C7
:10A91000160287FF0FC080E090E0A0E2B1E48983D7
:10A920009A83AB83BC83BE016F5F7F4F85E694E063
:10A930000E9467BA80E090E0A8ECB2E489839A8331
:10A94000AB83BC83AE014F5F5F4F6DE574E089E57B
:10A9500094E00E94117980E090E0A0EAB0E489835D
:10A960009A83AB83BC83BE016F5F7F4F81E694E027
:10A970000E9432798091650490916604A0916704E9
:10A98000B09168048093E0059093E105A093E205FF
:10A99000B093E3058093550490935604A093570415
:10A9A000B093580485E594E00E9454FC6091111521
:10A9B00087E00E9413A9EDE7F0E184918F010F5F1A
:10A9C0001F4F882321F00E94F0F6F801F6CF809106
:10A9D000AC0E9FEF980F9093AC0E992351F090918D
:10A9E000220F992319F091E09093210F82508093C8
:10A9F000AC0E60E08CE790E10E9453910F900F90B5
:10AA00000F900F90DF91CF911F910F91FF90EF90DA
:10AA1000DF90CF90BF90AF909F908F900895CF928E
:10AA2000DF92EF92FF92CF93DF93209119022223BE
:10AA300009F443C0EC01C0900D02D0900E02E090EA
:10AA40000F02F0901002A7019601688179818A8136
:10AA50009B810F94A608181624F4C882D982EA8232
:10AA6000FB82C0901102D0901202E0901302F0908D
:10AA70001402A70196016C817D818E819F810F94C4
:10AA8000A608181624F4CC82DD82EE82FF82C090E4
:10AA90001502D0901602E0901702F0901802A7015C
:10AAA0009601688579858A859B850F94A608181676
:10AAB00024F4C886D986EA86FB86DF91CF91FF9081
:10AAC000EF90DF90CF900895CF93DF93E091CD0783
:10AAD000F0E0EC51FA4F8081882309F45EC0E5E68E
:10AAE000FFE08491EF012196882321F00E94F0F687
:10AAF000FE01F7CFC091CD0780E6C89FE001112489
:10AB0000C351DA4F88818E3419F0E2E6FFE010C0BD
:10AB100080E20E94F0F689910E94F0F6899190ED12
:10AB2000980F9A30C8F38D32B9F38B32A9F3EDCF79
:10AB30008491EF012196882321F00E94F0F6FE0116
:10AB4000F7CF8091DB0E9091DC0E891B8F706FE048
:10AB500070E0681B7109072E000C880B990B0E948E
:10AB6000A9F7EFE5FFE08491EF012196882321F01A
:10AB70000E94F0F6FE01F7CF8091CE0765E070E00D
:10AB8000681B7109072E000C880B990B0E94A9F70E
:10AB90008AE0DF91CF910C94F0F6DF91CF91089588
:10ABA000CF93DF938091EB148093EC14E6E5FFE004
:10ABB0008491EF012196882321F00E94F0F6FE0196
:10ABC000F7CF8091221490912314A0912414B09176
:10ABD0002514BC01CD016F5F7F4F8F4F9F4F0E94A7
:10ABE000A9F78AE00E94F0F6DF91CF916DCF4F92E6
:10ABF0005F926F927F92BF92CF92DF92EF92FF921D
:10AC00000F931F93CF93DF93CDB7DEB72A970FB67D
:10AC1000F894DEBF0FBECDBF1092E9078091210FDF
:10AC2000882351F120911311222321F18091BD112C
:10AC30009091BE11A091BF11B091C0110097A105D4
:10AC4000B105B9F0BC01CD016D597F4F8F4F9F4FBA
:10AC500024E630E040E050E00F9422066091C111FC
:10AC60007091C2118091C3119091C4110F9422066A
:10AC700001C020E0209384038091EF071092EF073A
:10AC8000882339F00E947E978AE599EF0E9447BD9C
:10AC9000EBC420910402309105024091BD0E509109
:10ACA000BE0E6091BF0E7091C00EC901840F951F3A
:10ACB0002436310524F4853691053CF416C024363B
:10ACC000310531F08436910584F484E690E00DC0BE
:10ACD000473051056105710514F0069706C04A3FDB
:10ACE0005F4F6F4F7F4F6CF40696909305028093F1
:10ACF00004021092BD0E1092BE0E1092BF0E109262
:10AD0000C00E80910402909105028A3091053CF0BA
:10AD1000883E43E094072CF087EE93E002C08AE07F
:10AD200090E090930502809304020E94C094B82E94
:10AD30000E94F49080910412853198F4BB2049F070
:10AD40008091860990918709892B19F00BE117E111
:10AD500002C00EEF15E123E14FE061E088E00E94C0
:10AD6000E0BB809104128D3108F008C18830A0F555
:10AD70008091B80EB11002C081112EC060911215E1
:10AD800070911315072E000C880B990B0F941C0261
:10AD900020E030E040E05FE30F9480060F94C407AA
:10ADA000CB010E94A86EFC012081203229F4218170
:10ADB000203221F436E003C030E001C033E025E06A
:10ADC000231B2093071227E0209308120E94369835
:10ADD0008BEF95E10E942998809104128D31A0F5A6
:10ADE00080910612853180F120E030E040E05FE3A1
:10ADF00060918B0970918C0980918D0990918E09D9
:10AE00000F9480060F94C407CB010E94A86EFC012A
:10AE10008081803209F0B7C28181803209F0ACC2F2
:10AE200096E085E0891B809307128CE180930812DD
:10AE3000CF010E9436988BEF95E10E94299880916E
:10AE40000412853108F49AC2809104128830A0F56A
:10AE50008091B70EB11002C081112EC0609106051D
:10AE600070910705072E000C880B990B0F941C029C
:10AE700020E030E040E05FE30F9480060F94C407C9
:10AE8000CB010E94A86EFC012081203229F421818F
:10AE9000203221F436E003C030E001C033E021E588
:10AEA000231B2093071227E0209308120E94369854
:10AEB0008BEF95E10E942998809104128D31A0F5C5
:10AEC00080910612853180F120E030E040E05FE3C0
:10AED000609102057091030580910405909105052C
:10AEE0000F9480060F94C407CB010E94A86EFC014A
:10AEF0008081803209F07DC28181803209F072C286
:10AF000096E081E5891B809307128CE180930812FB
:10AF1000CF010E9436988BEF95E10E94299880918D
:10AF20000412853108F460C2809104128C3130F52E
:10AF300080910612843110F18091860990918709E1
:10AF4000019644E6489F9001499F300D112437FF38
:10AF500002C021503F4F832F932F990F990B0097D9
:10AF600069F028E6209307122BE1209308120E9433
:10AF7000A86E0E94369885E20E94E2BC809113116F
:10AF8000882349F080910412843328F480910612BA
:10AF90008A3208F05DC280910412853328F48091D2
:10AFA0000612813308F07AC260918403623048F05F
:10AFB00080910412843328F480910612823308F0C1
:10AFC00072C280910412813308F060C08091061231
:10AFD000893208F45BC00E941A992B013C018CE372
:10AFE000C82ED12CE12CF12CC301B201A70196018E
:10AFF0000F942206CA01B901A70196010F942206F7
:10B00000CA01F62EE72E69018E010F5F1F4F40E83F
:10B01000441641E5540641E06406710408F45EC23A
:10B02000B90128E130E040E050E00F942206290108
:10B030003A01EF92FF92C60168E170E00F94440973
:10B040009F938F935F924F9280ED90E19F938F93A8
:10B050001F930F930F94AF010FB6F894DEBF0FBE8E
:10B06000CDBF9AE0491651046104710408F060C232
:10B0700098E0892F880F980F9195955A9093071211
:10B0800080E380930812C8010E943698E091CA11AB
:10B09000F091CB11848181112FC1209185033091D2
:10B0A000860340918703509188036091D405709185
:10B0B000D5058091D6059091D7050F9480066B0138
:10B0C0007C0120E030E0A9010F94160287FD05C045
:10B0D00020E030E040E05FE304C020E030E040E00A
:10B0E0005FEBC701B6010F9480060F94C407CB0134
:10B0F0000E94156EBC0189E994E00F94BA09209171
:10B10000890330918A0340918B0350918C036091A5
:10B11000D8057091D9058091DA059091DB050F94DF
:10B1200080066B017C0120E030E0A9010F9416023B
:10B1300087FD05C020E030E040E05FE304C020E090
:10B1400030E040E05FEBC701B6010F9480060F943A
:10B15000C407CB010E94156EBC0184E994E00F94F2
:10B16000BA0920918D0330918E0340918F03509145
:10B1700090036091DC057091DD058091DE05909172
:10B18000DF050F9480066B017C0120E030E04AE788
:10B1900054E40F947B022B013C0120E030E0A90134
:10B1A000C701B6010F94160287FD05C020E030E00C
:10B1B00040EA50E404C020E030E040EA50ECC30133
:10B1C000B2010F94800620E030E040E251E40F9499
:10B1D0005C070F94C4076B017C0197FD16C06031BA
:10B1E000F7E27F0781059105D4F020E137E240E0E6
:10B1F00050E00F944406CA01B9012AE030E040E073
:10B2000050E00F944406605D0BC0F094E094D0943D
:10B21000C094C11CD11CE11CF11C6DE201C060E2B4
:10B2200060932C0528EEC21623E0D206E104F10457
:10B2300094F0C701B60128EE33E040E050E00F94EF
:10B240004406CA01B9012AE030E040E050E00F9422
:10B250004406605D01C060E260932D05C701B60140
:10B2600024E630E040E050E00F9444069AE0492E96
:10B27000512C612C712CCA01B901A30192010F94C8
:10B280004406605D60932E05C701B601A3019201DB
:10B290000F9444066B017C01672B682B692B79F0B6
:10B2A0008EE280932F05CA01B901A30192010F9488
:10B2B0004406605D6093300580E38C0D15C0CA01C3
:10B2C000B901A30192010F944406662339F08EE27E
:10B2D00080932F05605D6093300505C080E2809308
:10B2E000300580932F0580E2809331056CE275E094
:10B2F0008DE894E00F94BA09809104128632A8F484
:10B30000809106128E3188F008E020E84EE160E07E
:10B3100080ED91E10E94C8AF80910412863228F43A
:10B32000809106128F3108F005C18091041282339A
:10B3300028F4809106128C3208F077C180910412B3
:10B340008F3308F091C180910612883308F48CC1C4
:10B35000109207128EE38093081281EC9EE00E9407
:10B360000695182F0E9403BD163108F07DC180E2BA
:10B370000E94E2BC1F5FF8CF93E053CD809106128C
:10B38000813118F461CD90E04CCD6091121570912F
:10B390001315072E000C880B990B0F941C0220919B
:10B3A0008B0930918C0940918D0950918E090F9431
:10B3B000A608181674F41092F01102E022E041E1A0
:10B3C0006DE080ED91E10E94C8AF81E08093F011C3
:10B3D0003BCD02E022E041E16DE080ED91E10E9491
:10B3E000C8AF32CD93E08DCD80910612813118F433
:10B3F0009BCD90E086CD6091060570910705072EE4
:10B40000000C880B990B0F941C02209102053091BF
:10B41000030540910405509105050F94A6081816E0
:10B4200074F41092F01102E022E042E168E580ED50
:10B4300091E10E94C8AF81E08093F01175CD02E0E8
:10B4400022E042E168E580ED91E10E94C8AF6CCD59
:10B4500007E028E04AE26AE280ED91E10E94C8AF8D
:10B4600005E022E04CE262E380ED91E10E94C8AF8A
:10B470006AE08AE20E9436BC6091D2117091D311C9
:10B4800082E38093EC118BE28093ED112CEE31E19D
:10B4900042E380ED91E10E9406AE7DCD6AE486E351
:10B4A0000E9436BC81CDF8E46F9FB0011124072EB5
:10B4B000000C880B990B0F941C022AE037ED43E235
:10B4C0005CE30F947B020F94C907262F02E042E34E
:10B4D00067E380ED91E10E94C8AF73CDE4E6CE163C
:10B4E000D10498F4EF92FF923F932F9386EC90E172
:10B4F0009F938F931F930F930F94AF010FB6F89400
:10B50000DEBF0FBECDBF95E0B4CDEF92FF923F936B
:10B510002F938EEB90E19F938F931F930F930F9434
:10B52000AF010FB6F894DEBF0FBECDBF96E0A1CD40
:10B5300099E09FCD1092F01183E08093071215E2FD
:10B540001093081289EF95E10E9429988BE080936F
:10B55000071210930812BB2029F089E994E00E9499
:10B56000369811C08091480480FDF7CF09E914E0B6
:10B57000F80181918F01882331F08F3208F08FE339
:10B580000E941598F5CF8BE28093071215E2109375
:10B59000081287EF95E10E94299883E380930712B0
:10B5A00010930812BB2029F084E994E00E94369899
:10B5B00011C08091480481FDF7CF04E914E0F8013F
:10B5C00081918F01882331F08F3208F08FE30E9440
:10B5D0001598F5CF83E58093071215E210930812B2
:10B5E00085EF95E10E9429988BE5809307121093CF
:10B5F0000812BB2029F08DE894E00E94369811C013
:10B600008091480482FDF7CF0DE814E0F8018191A4
:10B610008F01882331F08F3208F08FE30E94159854
:10B62000F5CF81E08093F01180CE84E00E94E59711
:10B6300083E08093071212E31093081286E00E94C1
:10B6400015980E94F4908CE08093071210930812D2
:10B6500080910402909105020E94A86E0E94369883
:10B6600085E20E94E2BC6ACE2A960FB6F894DEBF4D
:10B670000FBECDBFDF91CF911F910F91FF90EF9043
:10B68000DF90CF90BF907F906F905F904F90089524
:10B69000282F1092E9078091BD0E9091BE0EA091C7
:10B6A000BF0EB091C00E81309048A105B10540F0A9
:10B6B0001092BD0E1092BE0E1092BF0E1092C00ED0
:10B6C0008091DE07882331F08091BD0E8093D207F0
:10B6D0001092BA0E8091D3071816FCF4082E000CB5
:10B6E000990B821B91092091D207022E000C330B7B
:10B6F0002817390794F097FF02C080E090E080930C
:10B70000D207092E000CAA0BBB0B8093BD0E9093A1
:10B71000BE0EA093BF0EB093C00E8091D2076623D9
:10B72000A9F09091D407891714F48093D40720913D
:10B73000D407022E000C330B2C5F3F4F482F082EEE
:10B74000000C550B241735071CF484508093D40744
:10B7500008958091BB0E8630D8F496E0899FF00161
:10B760001124E759FB4F209152023091530231834B
:10B7700020834091BD0E5091BE0E6091BF0E70911E
:10B78000C00E42835383648375838F5F8093BB0EA7
:10B79000089587EF95E50C9447BDE091BB0EEE232D
:10B7A00069F0E150E093BB0E86E0E89FF0011124C0
:10B7B000E759FB4F808191810C9447BDEACFAF924E
:10B7C000BF92CF92DF92EF92FF920F931F93CF938E
:10B7D000DF935C016B010E94F894EC01C6010E94AA
:10B7E000069504E110E0081B1109DD270C171D0761
:10B7F0001CF0FF24F39402C082E0F82E8091D11156
:10B8000090E06F2D70E06F5F7F4F0F945809E62E28
:10B81000C6E0C60F80910412C81750F0409106127E
:10B8200050E02C2F30E02B503109421753079CF584
:10B83000D0E0C114D104C1F18AE30E94E2BC82E0ED
:10B84000F8120FC0CE0D80910412C81768F1209134
:10B85000061230E08C2F90E00B97281739071CF464
:10B8600023C0DD2309F1902F990F090F000F0093DA
:10B870000712C093081280E20E94E2BCC601DF9169
:10B88000CF911F910F91FF90EF90DF90CF90BF90DD
:10B89000AF900C94369810920712C0930812C5010D
:10B8A0000E94EDBCD1E0C5CFDF91CF911F910F91E8
:10B8B000FF90EF90DF90CF90BF90AF9008950F93DF
:10B8C0004CE0849F402D112421E0240F20930C098B
:10B8D0008CE0840F80930D09E0910412F0E090E079
:10B8E00002968E179F070CF1822F90E0209106128E
:10B8F00030E082179307CCF4662371F081E08093E7
:10B90000F0114D5F0BE020E860E080ED91E10E94D6
:10B91000C8AF1092F01103C081E08093F0118091C4
:10B920000D0910920712809308120F910895CF927B
:10B93000DF92EF92FF920F93CF93DF93982F862F92
:10B940006A017901692FBBDF9091041280910D0982
:10B95000891708F448C09091061280910C09981735
:10B9600008F441C0002321F0C7010E94F89403C0ED
:10B97000C7010E940695D82FC4E1C81BF601849127
:10B98000882339F00E94FE97C81BFFEFCF1ADF0A09
:10B99000F5CF8AE30E94E2BCCC2329F080E20E942A
:10B9A000E2BCC150F9CF80910D099AEFD99FD02DFB
:10B9B0001124D058D093071280930812C701002396
:10B9C00049F0DF91CF910F91FF90EF90DF90CF90F2
:10B9D0000C942998DF91CF910F91FF90EF90DF9019
:10B9E000CF900C943698DF91CF910F91FF90EF900C
:10B9F000DF90CF900895CF92DF92EF92FF920F9356
:10BA0000CF93DF93CDB7DEB7E989FA89C080D180C3
:10BA1000E280F38020E030E0A901C701B6010F9475
:10BA2000160287FD05C020E030E040E05FE304C07F
:10BA300020E030E040E05FEBC701B6010F948006E4
:10BA40000F94C407CB010E94A86E00E09C014D85B5
:10BA50005E856C858B856BDFDF91CF910F91FF90B9
:10BA6000EF90DF90CF900895DF92EF92FF920F93C7
:10BA70001F93CF93DF931F92CDB7DEB77B01622F69
:10BA800049831DDF9091041280910D094981891726
:10BA900008F44CC09091061280910C09981708F494
:10BAA00045C0442359F10115110541F5C7010E9414
:10BAB000F89426E130E0281B390B37FF02C02F5FD6
:10BAC0003F4F3595279536E1D32E2751822F8D0D87
:10BAD00087FD11C080E229830E94E2BCDA942981AB
:10BAE000F5CFF7018491882361F00E94FE97D81A60
:10BAF0008FEFE81AF80A1D14A4F303C086E1D82ECC
:10BB0000FACF0115110559F01D144CF4F80181917B
:10BB10008F01882321F00E94FE97D81AF5CF1D14BB
:10BB20002CF480E20E94E2BCDA94F9CF0F90DF910E
:10BB3000CF911F910F91FF90EF90DF9008954F925A
:10BB40005F926F927F928F929F92AF92BF92CF92AD
:10BB5000DF92EF92FF92CF93DF93CDB7DEB72C97B2
:10BB60000FB6F894DEBF0FBECDBF80910205909155
:10BB70000305A0910405B091050589839A83AB83E1
:10BB8000BC836091060570910705072E000C880B99
:10BB9000990B0F941C0229813A814B815C810F948F
:10BBA0007F066B017C016093CC047093CD0480937D
:10BBB000CE049093CF0420913714309138144091E3
:10BBC000391450913A140F947B026D837E838F83D6
:10BBD00098876093C8047093C9048093CA049093B3
:10BBE000CB042091C4043091C5044091C604509107
:10BBF000C704C701B6010F9480064B015C01609336
:10BC0000C4047093C5048093C6049093C704209124
:10BC100033143091341440913514509136140F94EC
:10BC20007B0269877A878B879C876093C0047093B7
:10BC3000C1048093C2049093C30420ED3CEC4CE417
:10BC40005DE360912F1470913014809131149091C4
:10BC500032140F947B022B013C012091BC043091E3
:10BC6000BD044091BE045091BF0469817A818B81EB
:10BC70009C810F947F069B01AC01C301B2010F941C
:10BC80007B022B013C0123E333E343E75FE3609155
:10BC9000B8047091B9048091BA049091BB040F94D8
:10BCA0007B029B01AC01C301B2010F9480062B0102
:10BCB0003C016093B8047093B9048093BA049093E4
:10BCC000BB0489819A81AB81BC818093BC04909331
:10BCD000BD04A093BE04B093BF0429853A854B856B
:10BCE0005C856D817E818F8198850F948006A3018C
:10BCF00092010F947F062B013C0120E030E04EE4DE
:10BD000053E40F94A60820E030E0A9011816ACF423
:10BD1000C701B6010F94A60818166CF5A701960185
:10BD2000C501B4010F947F066093C4047093C504E9
:10BD30008093C6049093C7041EC0C301B2010F9440
:10BD4000160287FF22C020E030E0A901C701B6013A
:10BD50000F94160287FF16C0A7019601C501B40112
:10BD60000F947F066093C4047093C5048093C60447
:10BD70009093C70407C0412C512C8EE4682E83E4B5
:10BD8000782E03C0412C512C3201C301B2012C96F4
:10BD90000FB6F894DEBF0FBECDBFDF91CF91FF90FD
:10BDA000EF90DF90CF90BF90AF909F908F907F905B
:10BDB0006F905F904F9008952F923F924F925F92B5
:10BDC0006F927F928F929F92AF92BF92CF92DF92AB
:10BDD000EF92FF92CF93DF9300D01F92CDB7DEB7E3
:10BDE000609012157090131580908B0990908C09BB
:10BDF000A0908D09B0908E09B301072C000C880B20
:10BE0000990B0F941C02A50194010F947F066B01FE
:10BE10007C016093B4047093B5048093B60490934E
:10BE2000B70420ED3CEC4CE45DE360913B14709171
:10BE30003C1480913D1490913E140F947B021B01A1
:10BE40002C012091B0043091B1044091B204509182
:10BE5000B304C501B4010F947F069B01AC01C2017C
:10BE6000B1010F947B021B012C0123E333E343E771
:10BE70005FE36091AC047091AD048091AE04909149
:10BE8000AF040F947B029B01AC01C201B1010F947E
:10BE9000800669837A838B839C836093AC04709360
:10BEA000AD048093AE049093AF048092B00490925E
:10BEB000B104A092B204B092B3048091B80E88236A
:10BEC00021F081E08093AB04B9C020E030E040E293
:10BED00051E4C701B6010F94A608181624F481E0B6
:10BEE0008093AB04A4C020E030E040E251ECC701F5
:10BEF000B6010F94160287FDE4CF672811F38091F5
:10BF0000AB04882351F01092A7041092A804109259
:10BF1000A9041092AA041092AB042091431430910A
:10BF200044144091451450914614C701B6010F9432
:10BF30007B022B013C016093A3047093A4048093C3
:10BF4000A5049093A6042091A7043091A8044091E1
:10BF5000A9045091AA04C701B6010F9480064B01B1
:10BF60005C016093A7047093A8048093A904909344
:10BF7000AA0420913F1430914014409141145091F3
:10BF800042140F947B029B01AC0160939F04709359
:10BF9000A0048093A1049093A204C301B2010F9462
:10BFA000800629813A814B815C810F947F062B01A9
:10BFB0003C0120E030E04FE753E40F94A60820E076
:10BFC00030E0A9011816ACF4C701B6010F94A60819
:10BFD00018166CF5A7019601C501B4010F947F06F0
:10BFE0006093A7047093A8048093A9049093AA0473
:10BFF0001EC0C301B2010F94160287FF22C020E0C9
:10C0000030E0A901C701B6010F94160287FF16C0E0
:10C01000A7019601C501B4010F947F066093A704A0
:10C020007093A8048093A9049093AA0407C0412C9C
:10C03000512C8FE7682E83E4782E03C0412C512CBD
:10C040003201C301B2010F900F900F900F90DF915A
:10C05000CF91FF90EF90DF90CF90BF90AF909F90E7
:10C060008F907F906F905F904F903F902F900895AA
:10C070004F925F926F927F928F929F92AF92BF92F8
:10C08000CF92DF92EF92FF920F931F93CF93DF93A4
:10C09000CDB7DEB768970FB6F894DEBF0FBECDBF41
:10C0A0008C015B014A01DC01D7966D917D918D91E8
:10C0B0009C91DA970F941A026B017C01F5012081A3
:10C0C0003181428153810F947B020F9446070F9474
:10C0D000C90769877A878B879C87D4012D913D9109
:10C0E0004D915C91C701B6010F947B020F944607F6
:10C0F0000F94C9076D877E878F87988B29853A852E
:10C100004B855C85283731054105510540F488E7AA
:10C1100090E0A0E0B0E089879A87AB87BC872D8547
:10C120003E854F855889283731054105510540F432
:10C1300088E790E0A0E0B0E08D879E87AF87B88B5E
:10C1400098012D5B3F4FD9018D919D910D90BC9130
:10C15000A02D89839A83AB83BC83BC01CD010F944E
:10C160001C022B013C0169857A858B859C850F9487
:10C170001A02698B7A8B8B8B9C8B20E030E0A901B3
:10C18000C301B2010F941602882329F1A701960179
:10C19000C701B6010F947B024B015C0129893A89E2
:10C1A0004B895C89CA01B9010F947B029B01AC01E8
:10C1B000C501B4010F947F064B015C01A3019201FC
:10C1C000C301B2010F9480069B01AC01C501B4010B
:10C1D0000F945C0703C060E070E0CB010F9446074A
:10C1E0000F94C9076D837E838F83988769817A81D5
:10C1F0008B819C8190958095709561957F4F8F4F35
:10C200009F4F0F941C024B015C016D857E858F85CD
:10C2100098890F941A0269837A838B839C8320E028
:10C2200030E0A901C501B4010F941602882349F139
:10C2300029813A814B815C81CA01B9010F947B024B
:10C240006D8B7E8B8F8B988FA7019601C701B601EE
:10C250000F947B029B01AC016D897E898F89988D3B
:10C260000F947F066B017C01A5019401C501B40107
:10C270000F9480069B01AC01C701B6010F945C07C7
:10C2800003C060E070E0CB010F94F507F80185A0D2
:10C2900096A0A7A0B0A4750164012D813E814F81B5
:10C2A0005885C21AD30AE40AF50A0F94C907C61AB8
:10C2B000D70AE80AF90AF7FE73C020E030E0A901C6
:10C2C000C301B2010F941602882309F443C0A301ED
:10C2D0009201C301B2010F9480066B017C01C5017C
:10C2E000B4010F941A029B01AC01C701B6010F946F
:10C2F0007B026B017C0129893A894B895C89CA01DF
:10C30000B9010F947B029B01AC01C701B6010F94E8
:10C310007F066B017C0129813A814B815C81CA01D6
:10C32000B9010F947B029B01AC01C701B6010F94C8
:10C3300080066B017C0120E030E040E850E4C3015E
:10C34000B2010F947B029B01AC01C701B6010F94AF
:10C350005C0703C060E070E0CB010F9446077B01EF
:10C360006C0120E030E0A9010F94A608181624F013
:10C37000E12CF12CC12CD12CB701C6010F94C907B7
:10C380006D837E838F83988786169706A806B906E5
:10C3900020F48D829E82AF82B886C12CD12C76018A
:10C3A0008D819E81AF81B885F80182A793A7A4A74C
:10C3B000B5A7C80ED91EEA1EFB1EC6A6D7A6E0AAC0
:10C3C000F1AA29853A854B855C8523AF34AF45AF0B
:10C3D00056AFFF962D853E854F8558892083318342
:10C3E0004283538368960FB6F894DEBF0FBECDBF6D
:10C3F000DF91CF911F910F91FF90EF90DF90CF9041
:10C40000BF90AF909F908F907F906F905F904F9074
:10C41000089580916F0081FB992790F981FF05C0F5
:10C4200080916F008D7F80936F001092650910924C
:10C4300066091092670910926809992329F0809182
:10C440006F00826080936F0008954F925F926F92A9
:10C450007F928F929F92AF92BF92CF92DF92EF9294
:10C46000FF920F931F93CF93DF933C01B0E2A0E0C4
:10C470006A2F70E0AB014B0F511D559547954A1738
:10C4800011F04B130BC0E6EBF8E165917491072EA8
:10C49000000C880B990B0F941C0262C0CA01019713
:10C4A000880F991F880F991FFC01E85CF74E0591D2
:10C4B00014919A01220F331F220F331FF901E85CF8
:10C4C000F74EC591D4916016710614F4B42FD2CFF3
:10C4D000A42FC615D7050CF4CBCF865C974EFC0174
:10C4E000E590F490F901E65CF74EC590D490B70161
:10C4F0000F2C000C880B990B0F941C024B015C0154
:10C50000B301601B710B072E000C880B990B0F9465
:10C510001C022B013C01B6016E197F09072E000C8D
:10C52000880B990B0F941C029B01AC01C301B20153
:10C530000F947B026B017C01C01BD10BBE01DD0F90
:10C54000880B990B0F941C029B01AC01C701B6012B
:10C550000F945C079B01AC01C501B4010F948006E8
:10C56000DF91CF911F910F91FF90EF90DF90CF90CF
:10C57000BF90AF909F908F907F906F905F904F9003
:10C5800008950F930FB70F9300916E000B7F0093E8
:10C590006E0078940F930BB70F930CB70F921F9206
:10C5A0002F933F934F935F936F937F938F939F93BB
:10C5B000AF93BF93EF93FF9311240DD2FF91EF91AF
:10C5C000BF91AF919F918F917F916F915F914F91AB
:10C5D0003F912F911F900F900CBF0F910BBF0F91A8
:10C5E0000460F89400936E000F910FBF0F9118959F
:10C5F000CF92DF92EF92FF92C0900205D090030598
:10C60000E0900405F09005058091060590910705DE
:10C610000897BC01990F880B990B0F941C029B0182
:10C62000AC01C701B6010F94160287FF1FC020E0BE
:10C6300030E040E050E4C701B6010F9480060F944B
:10C64000C9077093E9046093E8040E94F6B2DC0124
:10C65000CB01805A9541AF4FBF4F8093E404909334
:10C66000E504A093E604B093E70408C01092E40444
:10C670001092E5041092E6041092E704FF90EF9008
:10C68000DF90CF900895CF92DF92EF92FF92C0900B
:10C690008B09D0908C09E0908D09F0908E098091E3
:10C6A0001215909113154597BC01990F880B990BA2
:10C6B0000F941C029B01AC01C701B6010F94160236
:10C6C00087FF1FC020E030E040E251E4C701B6011F
:10C6D0000F9480060F94C9077093E3046093E204FB
:10C6E0000E94F6B2DC01CB01805C9346AF4FBF4F96
:10C6F0008093DE049093DF04A093E004B093E10400
:10C7000008C01092DE041092DF041092E004109230
:10C71000E104FF90EF90DF90CF90089510921315F1
:10C720001092121580E0AFDF1092070510920605F7
:10C730005FDF0E94C099109213151092121580E0CD
:10C74000A2DF1092FF0480910201807480930001A7
:10C75000109207051092060510920005759808952D
:10C760004F925F926F927F928F929F92AF92BF9201
:10C77000CF92DF92EF92FF920F931F93CF93DF93AD
:10C780003C01BAE3A0E06A2F70E0AB014B0F511DF2
:10C79000559547954A1711F04B130BC0EDE0FAE1A0
:10C7A00065917491072E000C880B990B0F941C0255
:10C7B00062C0CA010197880F991F880F991FFC0159
:10C7C000E95DF64E059114919A01220F331F220F55
:10C7D000331FF901E95DF64EC591D49160167106DB
:10C7E00014F4B42FD2CFA42FC615D7050CF4CBCF99
:10C7F000875D964EFC01E590F490F901E75DF64EF9
:10C80000C590D490B7010F2C000C880B990B0F9496
:10C810001C024B015C01B301601B710B072E000C65
:10C82000880B990B0F941C022B013C01B6016E1969
:10C830007F09072E000C880B990B0F941C029B019B
:10C84000AC01C301B2010F947B026B017C01C01BE0
:10C85000D10BBE01DD0F880B990B0F941C029B01BD
:10C86000AC01C701B6010F945C079B01AC01C50187
:10C87000B4010F948006DF91CF911F910F91FF902B
:10C88000EF90DF90CF90BF90AF909F908F907F9070
:10C890006F905F904F90089560E08091EC049091CC
:10C8A000ED04D3DD60938B0970938C0980938D091F
:10C8B00090938E098091EA049091EB0451DF60938C
:10C8C0000205709303058093040590930505A895D0
:10C8D0001092EE040895CF92DF92FF920F931F9370
:10C8E000CF93DF931F921F92CDB7DEB7F82E8A0148
:10C8F00080911E02882309F444C0E4E4F9E48491A1
:10C900006F019FEFC91AD90A882341F069837A839E
:10C910000E94F0F6F60169817A81F1CFFB018491E2
:10C920006F019FEFC91AD90A882321F00E94F0F6FF
:10C93000F601F5CFEDEBF8E184916F019FEFC91A95
:10C94000D90A882321F00E94F0F6F601F5CFF7FC12
:10C950000BC06F2DFF0C770B880B990B0E94A9F76A
:10C960008AE00E94F0F60DC0E8EBF8E184916F01D7
:10C970009FEFC91AD90A882321F00E94F0F6F60128
:10C98000F5CF80919E04811108C010921E0281E0B3
:10C9900080939E04C8010E9448500F900F90DF9131
:10C9A000CF911F910F91FF90DF90CF90B7CE8F3F27
:10C9B00019F042E45AE102C042E55AE163E67AE145
:10C9C0008ACF8F3F19F04FE05AE102C04FE15AE1A0
:10C9D00060E37AE180CF0F931F93CF93DF93809131
:10C9E00023028F37A0F08F572091FF042093FE047D
:10C9F0009091020121119095907490930001909173
:10CA000000059093FD04992379F0759A0EC09091DA
:10CA1000FE04891728F09091020190749093000110
:10CA20009091FD04891708F075988F5F8093230219
:10CA30009091FC0481E089278093FC0481110E947D
:10CA4000FC9080912202853018F4C1E0C80F01C02B
:10CA5000C0E0823009F4ACC048F48823F9F081309A
:10CA600009F0DAC010927B0080E4B8C0843009F489
:10CA7000BDC008F4B0C0853009F0CEC09091FB0471
:10CA8000911102C08093FB048091FB04815080933C
:10CA9000FB04882309F4C0C0C5E0BEC08091210218
:10CAA0008F5F80311CF480932102B6C01092210266
:10CAB0008091EE04811113C08091F1049091F204F1
:10CAC0009093ED048093EC048091EF049091F00436
:10CAD0009093EB048093EA0481E08093EE048AE073
:10CAE000E1EFF4E0DF011D928A95E9F71092F0047E
:10CAF0001092EF040091EC041091ED041195019552
:10CB00001109D1E08091FF04811101C0D0E0809132
:10CB1000A3059091A405919581959109801791079E
:10CB200044F4DD2331F04FE05AE160E37AE180E044
:10CB3000D2DE8091260290912702919581959109EC
:10CB40000817190744F4DD2331F042E45AE163E6A3
:10CB50007AE180E0C0DE11E080910005811101C022
:10CB600010E02091EA043091EB048091A1059091AE
:10CB7000A2058217930744F0112331F04FE15AE1E7
:10CB800060E37AE18FEFA7DE209124023091250245
:10CB90008091EA049091EB0482179307ECF1112342
:10CBA000D9F142E55AE163E67AE18FEF94DE34C0D1
:10CBB00080917A0086FD2DC0809178009091790057
:10CBC0002091F1043091F204820F931F9093F204AC
:10CBD0008093F10421C010927B0082E480937C005A
:10CBE00080917A00806480937A0016C080917A00E8
:10CBF00086FD11C080917800909179002091EF041A
:10CC00003091F004820F931F9093F0048093EF040F
:10CC100003C0C2E001C0C4E0C09322020E94999800
:10CC20008091900E9091910E009799F001979093BA
:10CC3000910E8093900E892B61F485E79AE1909391
:10CC4000080980930709DF91CF911F910F910C94F0
:10CC50005E8FDF91CF911F910F9108958F929F92D8
:10CC6000AF92BF92CF92DF92EF92FF920F93CF934A
:10CC7000DF9300D01F92CDB7DEB780916814811189
:10CC80001CC18091EE04811110C00F900F900F9085
:10CC90000F90DF91CF910F91FF90EF90DF90CF90A9
:10CCA000BF90AF909F908F900895F6DD0E94F6B2EE
:10CCB0004B015C0180911F02909120021816190609
:10CCC0000CF01CC101979093200280931F02809169
:10CCD000B80E811117C08091DA049091DB04A09105
:10CCE000DC04B091DD040097A105B10559F0A50160
:10CCF0009401281B390B4A0B5B0B57FD03C081E0E5
:10CD00008093B80E6091121570911315072E000CC8
:10CD1000880B990B0F941C0269837A838B839C8305
:10CD20003EE1E32EF12C00E09E012F5F3F4F4BE8E8
:10CD300059E066ED74E085ED94E00E946ABDC09014
:10CD40008B09D0908C09E0908D09F0908E0980912C
:10CD5000A5059091A605BC01990F880B990B0F941E
:10CD60001C029B01AC01C701B6010F94A60818165E
:10CD70000CF4A7C060E06093FF048091DE04909102
:10CD8000DF04A091E004B091E1040097A105B10592
:10CD900021F1A5019401281B390B4A0B5B0B57FDB0
:10CDA0001CC06091E2047091E30480E090E00F9475
:10CDB0001A029B01AC0160918B0970918C098091E2
:10CDC0008D0990918E090F94160287FFBFC04DEF19
:10CDD00058E16FE079E180E07EDD8091E40490919C
:10CDE000E504A091E604B091E7040097A105B10520
:10CDF00011F1881A990AAA0ABB0AB7FC1CC06091F3
:10CE0000E8047091E90480E090E00F941A029B011D
:10CE1000AC01609102057091030580910405909129
:10CE200005050F94160287FF88C04BED58E16EEEA2
:10CE300078E18FEF50DD6091060570910705072EB0
:10CE4000000C880B990B0F941C0269837A838B83E7
:10CE50009C839AE0E92EF12C0FEF9E012F5F3F4F4C
:10CE600042E055E060ED74E084ED94E00E946ABD1C
:10CE70008091B70E81113FC0C0900205D09003058C
:10CE8000E0900405F090050520E030E040EA50E431
:10CE9000C701B6010F94A60887FD0BC020E030E063
:10CEA00046E153E4C701B6010F94160218160CF0C0
:10CEB00046C060E060930005E8CE8EE199E10E94F3
:10CEC00048506091280270912902072E000C880BAF
:10CED000990B0F941C029B01AC01C701B6010F9482
:10CEE000160287FF47CF80E00E94DC5E0F94C407E4
:10CEF0007595679540CF10920005C7CEC0908B09FD
:10CF0000D0908C09E0908D09F0908E0920E030E8F7
:10CF100048E953E4C701B6010F94A6081816CCF0EF
:10CF200020E030E040EA50E4C701B6010F94160259
:10CF300087FFCDCE80E03BDDCACE5ADB7CCF0E949E
:10CF40009F5D0F94C40775956795B4CF80E09BDB18
:10CF500044CF80E036DDC0908B09D0908C09E09002
:10CF60008D09F0908E09DCCFCF92DF92EF92FF9285
:10CF7000CF93DF936A017B01FC018491EF0121963D
:10CF8000882321F00E94F0F6FE01F7CF4AE0C701A6
:10CF9000B601DF91CF91FF90EF90DF90CF900C948E
:10CFA00043F7CF92DF92EF92FF92CF93DF936A0124
:10CFB0007B01FC018491EF012196882321F00E94DE
:10CFC000F0F6FE01F7CF42E0C701B601DF91CF9145
:10CFD000FF90EF90DF90CF900C94C3F7EF92FF9209
:10CFE0000F931F93CF93DF931F92CDB7DEB78C01C2
:10CFF0007B0180E249830E94F0F649814F3F11F0A6
:10D0000084E501C082E40E94F0F68AE30E94F0F613
:10D01000F801608171818281938142E00E94C3F7AF
:10D02000F701408151816281738181E89AE1B9DF22
:10D0300062E070E080E090E00F90DF91CF911F916F
:10D040000F91FF90EF900C94BEB20F931F93CF936C
:10D05000DF93CDB7DEB728970FB6F894DEBF0FBECB
:10D06000CDBF6091121570911315072E000C880B1F
:10D07000990B0F941C026D837E838F839887809118
:10D080008B0990918C09A0918D09B0918E098983AB
:10D090009A83AB83BC834DEFBE016B5F7F4FCE01A4
:10D0A00001969CDF6091060570910705072E000C24
:10D0B000880B990B0F941C026D837E838F83988756
:10D0C0008091020590910305A0910405B09105059A
:10D0D00089839A83AB83BC834FEFBE016B5F7F4F25
:10D0E000CE0101967BDFE9E8FAE184918F010F5FC1
:10D0F0001F4F882321F00E94F0F6F801F6CFE0914F
:10D100000105F0E0E150FB4F608170E080E090E0CD
:10D110000E94A9F7E4E8FAE184918F010F5F1F4FA5
:10D12000882321F00E94F0F6F801F6CF6091000507
:10D1300070E080E090E00E94A9F728960FB6F8947E
:10D14000DEBF0FBECDBFDF91CF911F910F9108952C
:10D150000F931F93CF93DF9300D01F92CDB7DEB70D
:10D16000FC0184918F010F5F1F4F882361F0498379
:10D170005A836B837C830E94F0F6F80149815A81BF
:10D180006B817C81EECFCB01BA010F900F900F9095
:10D190000F90DF91CF911F910F910C94A9F70F93EE
:10D1A0001F93CF93DF938B01FC018491EF012196B4
:10D1B000882321F00E94F0F6FE01F7CFB801110F8D
:10D1C000880B990BDF91CF911F910F910C94A9F7C8
:10D1D0000F931F93CF93DF931F921F92CDB7DEB7AC
:10D1E000FC0184918F010F5F1F4F811102C08B01E1
:10D1F00008C069837A830E94F0F6F80169817A8118
:10D20000F0CFF80181918F01882319F00E94F0F688
:10D21000F8CF0F900F90DF91CF911F910F9108954C
:10D220008F929F92AF92BF92CF92DF92EF92FF9236
:10D230000F93CF93DF931F92CDB7DEB77C015B01D5
:10D240006A01490180910A128823F1F0F7014081B7
:10D250005181C40ED51ED182C08223C001111EC0CF
:10D26000BE016F5F7F4FC4010E94C4ABF7014081D4
:10D2700051814F5F5F4F51834083FFEFAF1ABF0A69
:10D2800081E0C81AD10869F0F701808191810F947B
:10D29000DC058983909126149111E0CFF5018083FC
:10D2A000DFCF0F90DF91CF910F91FF90EF90DF9044
:10D2B000CF90BF90AF909F908F9008958F929F9244
:10D2C000AF92BF92CF92DF92EF92FF920F931F9394
:10D2D000CF93DF931F921F92CDB7DEB7E0910A1272
:10D2E000E11107C069017C015B018B01040F151F6F
:10D2F00022C0FC0120813181420F531F51834083A2
:10D3000042C0F70180809180F50161915F016983DE
:10D31000C4016A830F94DC056A81681310C0BE01E2
:10D320006F5F7F4FC6010E94C4ABF701808191817E
:10D33000019691838083A016B10619F724C0C40119
:10D340000F940506C4010F94DC059981891739F300
:10D35000ECE4F2E484918F010F5F1F4F882321F0EA
:10D360000E94F0F6F801F6CFE9ECFAE184918F0122
:10D370000F5F1F4F882321F00E94F0F6F801F6CFCF
:10D3800081E080930A120F900F90DF91CF911F914F
:10D390000F91FF90EF90DF90CF90BF90AF909F9054
:10D3A0008F900895CF93DF93CDB7DEB72C970FB64C
:10D3B000F894DEBF0FBECDBF8091D4059091D50506
:10D3C000A091D605B091D70589839A83AB83BC839E
:10D3D0008091D8059091D905A091DA05B091DB052F
:10D3E0008D839E83AF83B8878091DC059091DD05A6
:10D3F000A091DE05B091DF0589879A87AB87BC874E
:10D400000E940D4B0E94204D80E00E948C7B81E0A9
:10D410000E948C7B82E00E948C7B0E94B94C4CE085
:10D4200050E064ED75E0CE0101960F947B09892BE5
:10D4300051F02C960FB6F894DEBF0FBECDBFDF9132
:10D44000CF910C9452B52C960FB6F894DEBF0FBE58
:10D45000CDBFDF91CF91089561E0FC0180810C94F4
:10D46000C8B18EBD0DB407FEFDCF08958FEF8EBD00
:10D470000DB407FEFDCF8EB508950F931F93CF9384
:10D48000DF938B010E94F6B2EB01F0DF8F3F49F092
:10D490000E94F6B26C1B7D0B60177107B0F380E041
:10D4A00001C081E0DF91CF911F910F910895CF923C
:10D4B000DF92EF92FF921F93CF93DF9300D01F92E2
:10D4C000CDB7DEB76C01162FFC019281892F806ADF
:10D4D00086958CBD90FD03C081E0963009F480E014
:10D4E0008DBD60E0F601808129833A834B835C83A4
:10D4F0000E94C8B16CE271E0C601BFDF812F806479
:10D50000B0DF88E1E82EF12C5C814B813A812981E2
:10D51000DA01C9010E2C04C0B695A7959795879599
:10D520000A94D2F729833A834B835C839ADFF8E02D
:10D53000EF1AF10829813A814B815C8188EFE81666
:10D540008FEFF80629F7112321F0183021F08FEF23
:10D5500003C085E901C087E884DF1C3009F486DF59
:10D5600010E084DFF601838387FF04C01F3F11F0C2
:10D570001F5FF7CF0F900F900F900F90DF91CF911B
:10D580001F91FF90EF90DF90CF9008950F931F931E
:10D59000CF93DF93EC0189018C81833039F089E0EE
:10D5A000440F551F661F771F8A95D1F79A01AB016B
:10D5B00068E1CE017CDF882311F086E02FC08EEF7A
:10D5C0008EBD80E090E00DB407FEFDCFF801E80FBE
:10D5D000F91F20812EBD0DB407FEFDCF21812EBD88
:10D5E0000296811522E0920771F70DB407FEFDCF78
:10D5F0008FEF37DF8FEF35DF39DF8B838F7185302A
:10D6000029F083E18983CE0127DF09C068E572E054
:10D61000CE0133DF182F811106C087E18983CE0147
:10D620001BDF10E00FC020E030E0A9016DE0CE016B
:10D630003EDF811103C01ADF882311F086E1EECFAF
:10D64000CE010ADF812FDF91CF911F910F910895B5
:10D65000EF92FF920F931F93CF93DF93EC01790129
:10D660008C81833039F089E0440F551F661F771F86
:10D670008A95D1F79A01AB0161E1CE0118DF8823C9
:10D6800029F084E08983CE01E7DE35C00E94F6B23E
:10D690008B01ECDE8B838F3F49F40E94F6B2601B56
:10D6A000710B6D327140A8F381E103C08E3F39F0F8
:10D6B0008FE08983CE01D0DE8FEFD3DE1CC08FEFE9
:10D6C0008EBDF701D701A150BE4F0DB407FEFDCFAF
:10D6D0009EB591938EBDEA17FB07B9F70DB407FE0F
:10D6E000FDCF8EB58C93C2DEC1DECE01B5DE8FEFED
:10D6F000B8DE81E001C080E0DF91CF911F910F91F2
:10D70000FF90EF9008958F929F92AF92BF92CF9229
:10D71000DF92EF92FF92CF93FC01C080D180E28034
:10D72000F38020E030E0A901C701B6010F94160292
:10D7300087FF08C0C701B601905820E030E04AE7F3
:10D7400054E406C020E030E04AE754E4C701B601E3
:10D750000F947B0220E030E040EA50E40F94800612
:10D7600020E030E040E251E40F945C070F94C407DE
:10D770006B017C01603AF6E87F07F1E08F079105C5
:10D7800084F020EA36E841E050E00F944406CA01F4
:10D79000B9012AE030E040E050E00F944406605DBB
:10D7A00001C060E260932B0580E1C81687E2D806CD
:10D7B000E104F10494F0C701B60120E137E240E052
:10D7C00050E00F944406CA01B9012AE030E040E07D
:10D7D00050E00F944406605D01C060E260932C0548
:10D7E000E8EECE16E3E0DE06E104F10494F0C701B2
:10D7F000B60128EE33E040E050E00F944406CA0141
:10D80000B9012AE030E040E050E00F944406605D4A
:10D8100001C060E260932D05C701B60124E630E047
:10D8200040E050E00F9444068AE0882E912CA12C11
:10D83000B12CCA01B901A50194010F944406605DA1
:10D8400060932E058EE280932F05C701B601A501D6
:10D8500094010F944406C62FCA01B901A501940191
:10D860000F944406605D60933005C05DC093310540
:10D870008BE295E0CF91FF90EF90DF90CF90BF903B
:10D88000AF909F908F9008958F929F92AF92BF928A
:10D89000CF92DF92EF92FF92CF93FC01C080D180B4
:10D8A000E280F38020E030E04AE754E4C701B601AB
:10D8B0000F947B024B015C0120E030E0A901C7011D
:10D8C000B6010F94160287FD05C020E030E040EA63
:10D8D00050E404C020E030E040EA50ECC501B4015F
:10D8E0000F94800620E030E040E251E40F945C07A2
:10D8F0000F94C4076B017C0197FF0AC0F094E09479
:10D90000D094C094C11CD11CE11CF11C8DE201C05B
:10D910008BE280932B05C701B60120E137E240E09E
:10D9200050E00F9444068AE0882E912CA12CB12C53
:10D93000CA01B901A50194010F944406605D60938A
:10D940002C05C701B60128EE33E040E050E00F940B
:10D950004406CA01B901A50194010F944406605D13
:10D9600060932D05C701B60124E630E040E050E0A9
:10D970000F944406CA01B901A50194010F9444060D
:10D98000605D60932E058EE280932F05C701B6017E
:10D99000A50194010F944406C62FCA01B901A5013F
:10D9A00094010F944406605D60933005C05DC093A0
:10D9B00031058BE295E0CF91FF90EF90DF90CF9013
:10D9C000BF90AF909F908F9008958F929F92AF924B
:10D9D000BF92CF92DF92EF92FF92FC01C080D18084
:10D9E000E280F38020E030E0A901C701B6010F9486
:10D9F000160287FF08C0C701B601905820E030E04A
:10DA000040E251E406C020E030E040E251E4C701CA
:10DA1000B6010F947B0220E030E040EA50E40F941E
:10DA2000800620E030E040E251E40F945C070F9460
:10DA3000C4076B017C016031F7E27F078105910526
:10DA400084F020E137E240E050E00F944406CA0140
:10DA5000B9012AE030E040E050E00F944406605DF8
:10DA600001C060E260932D0588EEC81683E0D806F9
:10DA7000E104F10494F0C701B60128EE33E040E080
:10DA800050E00F944406CA01B9012AE030E040E0BA
:10DA900050E00F944406605D01C060E260932E0583
:10DAA000E4E6CE16D104E104F10494F0C701B60116
:10DAB00024E630E040E050E00F944406CA01B9018A
:10DAC0002AE030E040E050E00F944406605D01C081
:10DAD00060E260932F05FAE0CF16D104E104F1046F
:10DAE0009CF08AE0882E912CA12CB12CC701B601A4
:10DAF000A50194010F944406CA01B901A50194013E
:10DB00000F944406605D01C060E260933005C70178
:10DB1000B6012AE030E040E050E00F944406605D3A
:10DB2000609331058DE295E0FF90EF90DF90CF900C
:10DB3000BF90AF909F908F9008958F929F92AF92D9
:10DB4000BF92CF92DF92EF92FF92FC01C080D18012
:10DB5000E280F38020E030E048EC52E4C701B601F7
:10DB60000F947B024B015C0120E030E0A901C7016A
:10DB7000B6010F94160287FD05C020E030E040EAB0
:10DB800050E404C020E030E040EA50ECC501B401AC
:10DB90000F94800620E030E040E251E40F945C07EF
:10DBA0000F94C4079B0177FF06C022273327261B4B
:10DBB000370B8DE201C08BE280932C05C90168EE22
:10DBC00073E00F945809CB01EAE0F0E0BF010F9435
:10DBD0005809805D80932D05C90164E670E00F94BB
:10DBE0005809CB01BF010F945809805D80932E0521
:10DBF000C901BF010F945809282FCB01BF010F9411
:10DC00005809805D80932F058EE280933005205D5A
:10DC1000209331058CE295E0FF90EF90DF90CF905C
:10DC2000BF90AF909F908F900895AC01952F991F52
:10DC30009927991F29F022273327241B350B01C070
:10DC40009A01483E5340ACF0C90168EE73E00F946E
:10DC50005809CB01EAE0F0E0BF010F945809805D5C
:10DC600080932E05C90164E670E00F945809CB013A
:10DC700012C024363105B4F0911102C080E201C017
:10DC80008DE280932E05C90164E670E00F94580977
:10DC9000CB01EAE0F0E0BF010F945809805D80936A
:10DCA0002F050EC080E280932E0580932F052A3029
:10DCB000310584F091118DE280932F05EAE0F0E0C8
:10DCC000C901BF010F945809CB01BF010F94580936
:10DCD000805D05C0911102C080E201C08DE2809399
:10DCE0003005C9016AE070E00F945809805D8093A7
:10DCF00031058EE295E008959C01EAE0F0E0BF0175
:10DD00000F94580990E3980F909331052A3031050C
:10DD1000CCF0CB01BF010F945809805D8093300592
:10DD20002436310594F0C90164E670E00F94580977
:10DD3000CB01BF010F945809805D80932F058FE2BE
:10DD400095E0089581E395E0089580E395E00895D6
:10DD50009C0197FD0EC08436910584F064E670E066
:10DD60000F945809CB016AE070E00F945809805D68
:10DD700006C03195219531098DE201C080E2809382
:10DD80002F052A30310564F0EAE0F0E0C901BF0157
:10DD90000F945809CB01BF010F945809805D01C051
:10DDA00080E280933005C9016AE070E00F94580961
:10DDB000805D809331058FE295E00895CF92DF92E8
:10DDC000EF92FF926B017C0183E3C816D104E1045A
:10DDD000F10470F082E3C81AD108E108F10862E3A7
:10DDE00070E080E090E00E94BEB20E942E66ECCF10
:10DDF000C701B6010E94BEB2FF90EF90DF90CF90B6
:10DE00000C942E664F925F926F927F928F929F92A8
:10DE1000AF92BF92CF92DF92EF92FF920F931F9338
:10DE2000CF9310922705109226052FE320932A0501
:10DE300010922905109228051092220510922305B0
:10DE400010922405109225059C01F90190812F5F05
:10DE50003F4F9032D1F3DF019E34B1F4818190EDD8
:10DE6000980F9A3020F08D3211F08B3269F432968F
:10DE7000DF0131962C9120532A30D0F3CD01DC0103
:10DE800001962C912032D9F3B0931015A0930F1561
:10DE90008D010F5F1F4FCC916AE270E0C8010F94B3
:10DEA000AF09009731F0FC01319780818032E1F3B6
:10DEB0001182CD3429F0C43519F0C73409F005C1F9
:10DEC000F80180810F5F1F4F8032D1F380538A3079
:10DED00008F0FBC0C0932A0510922905109228056E
:10DEE0006AE08091280590912905689FA001699FAB
:10DEF000500D112450932905409328053196DF01D8
:10DF000011978C91282F30E020533109240F351FB1
:10DF10003093290520932805808180538A3008F3A7
:10DF2000DF0131968C918032D9F3CD34D1F42E318A
:10DF3000310591F03CF42731310571F02C31310578
:10DF400081F40AC02537310564F02737310524F004
:10DF5000203A83E0380729F4B0932705A0932605DB
:10DF6000B4C0109227051092260560910F15C12CA0
:10DF7000D12C7601C394CD0101964C91442309F430
:10DF8000A4C0413299F4CD3489F42032310571F4C2
:10DF9000909327058093260563E270E00F94AF0904
:10DFA000009709F492C0FC0110828FC041544A319D
:10DFB00008F04DC0DC01FD015D915032E1F3CF016D
:10DFC00070ED750F7A30D0F05E3229F451815053E4
:10DFD0005A30A0F006C05D3209F465C05B3209F426
:10DFE00062C0A0912605B0912705AB2B09F06AC04D
:10DFF0003197F0932705E093260564C0FC01A42F18
:10E00000B0E04601570104C0880C991CAA1CBB1C37
:10E010004A95D2F740902205509023056090240540
:10E020007090250584289528A628B7288092220577
:10E0300090922305A0922405B0922505309711F007
:10E04000E61B01C0E0E0A85FBA4FEC930AC0409124
:10E05000260550912705452B21F4B0932705A09361
:10E060002605FC01408141544A3130F4DC0183CF64
:10E0700040ED490F4A3040F48E2F7F2F919191113E
:10E08000F7CF482F572F07C043ED490F4230A0F379
:10E090009B3291F3F6CFCA014F5F5F4FFC01708155
:10E0A0007032C9F3E3CF518170ED750F7A3008F407
:10E0B000A6CF5E3209F095CF528150535A3008F402
:10E0C0009ECF8FCFE0E0F0E09ACFCF911F910F91DC
:10E0D000FF90EF90DF90CF90BF90AF909F908F9088
:10E0E0007F906F905F904F900895CF93DF93EBEB0D
:10E0F000FAE18491EF012196882321F00E94F0F645
:10E10000FE01F7CFE7EBFAE18491EF012196882336
:10E1100021F00E94F0F6FE01F7CF62B366956170C0
:10E1200070E080E090E00E94A9F762B3617070E057
:10E1300080E090E00E94A9F78AE00E94F0F6E3EB0D
:10E14000FAE18491EF012196882321F00E94F0F6F4
:10E15000FE01F7CF60910601862F660F990BAA0B7F
:10E16000BB0BBC01CD01662797FD639577278827F8
:10E1700099270E94A9F762B362FB662760F970E0F5
:10E1800080E090E00E94A9F78AE00E94F0F6EFEAB2
:10E19000FAE18491EF012196882321F00E94F0F6A4
:10E1A000FE01F7CF6091060166FB662760F970E01B
:10E1B00080E090E00E94A9F76091060165FB662768
:10E1C00060F970E080E090E00E94A9F78AE00E9488
:10E1D000F0F6EAEAFAE18491EF012196882321F032
:10E1E0000E94F0F6FE01F7CF6091060163FB6627FF
:10E1F00060F970E080E090E00E94A9F7609106016C
:10E200006295617070E080E090E00E94A9F78AE07A
:10E210000E94F0F6E5EAFAE18491EF012196882365
:10E2200021F00E94F0F6FE01F7CF6091060166959D
:10E23000617070E080E090E00E94A9F760910601B3
:10E2400062FB662760F970E080E090E00E94A9F729
:10E250008AE0DF91CF910C94F0F6CF93DF93643096
:10E2600021F128F46130E9F06230E9F004C068304F
:10E27000F9F06031E9F0E4E4F9E48491EF012196EA
:10E28000882321F00E94F0F6FE01F7CFEDE8FAE1D5
:10E290008491EF012196882389F00E94F0F6FE0117
:10E2A000F7CF40E003C040E004C041E060E002C0BE
:10E2B00041E061E0DF91CF910C94E042DF91CF919A
:10E2C0000895CF92DF92EF920F931F93CF93DF9336
:10E2D00000D01F92CDB7DEB7E090111519821A82D7
:10E2E0001B821C82CE0101966C0100E012E020EE40
:10E2F00035E04CED55E068ED75E084ED95E00E9469
:10E300009C9B0F900F900F900F90DF91CF911F91DA
:10E310000F91EF90DF90CF9008954F925F926F92A0
:10E320007F928F929F92AF92BF92CF92DF92EF92A5
:10E33000FF920F931F93CF93DF93CDB7DEB72C9748
:10E340000FB6F894DEBF0FBECDBF6D837E838F8383
:10E35000988729873A874B875C87470158013601A0
:10E360008091000290910102A0910202B0910302FB
:10E3700089839A83AB83BC83D601CD90DD90ED90E9
:10E38000FC9020E030E0A901C701B6010F9416020D
:10E39000811106C0E8E0F0E1C590D590E590F490D9
:10E3A000A50194016091DC057091DD058091DE0589
:10E3B0009091DF050F94160287FF11C0C0920002F2
:10E3C000D0920102E0920202F09203028092DC05F8
:10E3D0009092DD05A092DE05B092DF0572DFF301B9
:10E3E000408051806280738020E030E0A901C30149
:10E3F000B2010F941602811106C0412C512C88ECF9
:10E40000682E82E4782E40920002509201026092BF
:10E410000202709203028D819E81AF81B885809344
:10E42000D4059093D505A093D605B093D7058985DB
:10E430009A85AB85BC858093D8059093D905A09328
:10E44000DA05B093DB053DDFA50194016091DC05A1
:10E450007091DD058091DE059091DF050F94A6088F
:10E4600018168CF4C0920002D0920102E0920202CF
:10E47000F09203028092DC059092DD05A092DE0509
:10E48000B092DF051EDF0E94D54B89819A81AB8156
:10E49000BC818093000290930102A0930202B0938A
:10E4A00003022C960FB6F894DEBF0FBECDBFDF91EE
:10E4B000CF911F910F91FF90EF90DF90CF90BF9081
:10E4C000AF909F908F907F906F905F904F90089546
:10E4D000CF92DF92EF92FF926B017C010E94F6B225
:10E4E000C60ED71EE81EF91E0E94F6B2DC01CB0153
:10E4F0008C199D09AE09BF09B7FF04C080E00E94D6
:10E50000A850F2CFFF90EF90DF90CF900895AF9298
:10E51000BF92CF92DF92EF92FF920F931F93CF9310
:10E52000DF938DEEA82E82E0B82E99E4E92E94E0D8
:10E53000F92E04ED15E025E8C22E23E0D22EC0E02E
:10E54000D0E0F50181915F010E943A90882321F18A
:10E550000E940790FE01E356FC4F2081211104C068
:10E560002091A103222341F0F801208131814281D1
:10E5700053810F9480060AC0C330D10539F0F601EB
:10E5800020813181428153810F947F06F70160839E
:10E590007183828393830AC0F80180819181A28173
:10E5A000B381F70180839183A283B3832196F4E042
:10E5B000EF0EF11C0C5F1F4F84E0C80ED11CC4305D
:10E5C000D10509F0BECF86E40E9481908823C9F06E
:10E5D0000E94079020E030E0A9010F94A6081816C9
:10E5E00084F40E94079020E030E040E752E40F946A
:10E5F0005C07609300027093010280930202909383
:10E60000030280917F0E83FD2AC0609155047091B2
:10E61000560480915704909158042091E005309160
:10E62000E1054091E2055091E305E091B405EE2348
:10E63000B1F00F947F069B01AC016091C105709110
:10E64000C2058091C3059091C4050F948006609324
:10E65000C1057093C2058093C3059093C405DF91F3
:10E66000CF911F910F91FF90EF90DF90CF90BF90CF
:10E67000AF9008952F923F924F925F926F927F9248
:10E680008F929F92AF92BF92CF92DF92EF92FF92C2
:10E690000F931F93CF93DF93CDB7DEB7C455D10946
:10E6A0000FB6F894DEBF0FBECDBF90911E02992326
:10E6B00009F408C5382E2BDF82E50E94819088235B
:10E6C00009F430C10E9407906B017C014090D40591
:10E6D0005090D5056090D6057090D7052091D8054B
:10E6E0003091D9054091DA055091DB052D8F3E8F91
:10E6F0004F8F58A38091490490914A04A0914B04F4
:10E70000B0914C0489A39AA3ABA3BCA320914D0460
:10E7100030914E0440914F045091500429A73AA7DC
:10E720004BA75CA720E030E0A901C701B6010F9418
:10E730001602882309F4AEC4A301920169A17AA14B
:10E740008BA19CA10F94160281110DC02D8D3E8DC1
:10E750004F8D58A169A57AA58BA59CA50F9416028B
:10E76000882309F497C4A32CB12C01E010E020E029
:10E7700030E0A901C701B6010F94160287FD02C05F
:10E7800000E010E0A016B10649F480E090E0A0E8B7
:10E79000BFE38DAB9EABAFABB8AF08C020E030E0BD
:10E7A00040E85FEB2DAB3EAB4FAB58AFA3019201FE
:10E7B00069A17AA18BA19CA10F947F066DA77EA76A
:10E7C0008FA798AB2D8D3E8D4F8D58A169A57AA549
:10E7D0008BA59CA50F947F0669AB7AAB8BAB9CABEA
:10E7E0002DA53EA54FA558A9CA01B9010F947B02DA
:10E7F0004B015C0129A93AA94BA95CA9CA01B9013D
:10E800000F947B029B01AC01C501B4010F948006FB
:10E810000F94EB086DA37EA38FA398A720E030E0B0
:10E8200040E05FE30F947B024B015C01A70196017E
:10E83000C701B6010F947B026B017C01A501940115
:10E84000C501B4010F947B029B01AC01C701B60165
:10E850000F947F060F94EB089B01AC016DA97EA974
:10E860008FA998AD0F947B024B015C0129A13AA1BD
:10E870004BA15CA1C301B2010F94800620E030E0FF
:10E8800040E05FE30F947B026B017C0169A97AA9E8
:10E890008BA99CA990582DA13EA14FA158A50F94DA
:10E8A0005C079B01AC01C501B4010F947B029B0185
:10E8B000AC01C701B6010F948006A30192010F9429
:10E8C0007F066B017C0129A53AA54BA55CA56D8D42
:10E8D0007E8D8F8D98A10F94800620E030E040E07F
:10E8E0005FE30F947B022B013C012DA13EA14FA1C0
:10E8F00058A56DA57EA58FA598A90F945C079B01CF
:10E90000AC01C501B4010F947B029B01AC01C301B2
:10E91000B2010F9480062D8D3E8D4F8D58A10F941E
:10E920007F0614C089E40E948190882329F00E9408
:10E9300007906B017C0103C0C12CD12C76018AE4C5
:10E940000E9481908823D9F00E94079069A77AA736
:10E950008BA79CA720E030E0A901C701B6010F9466
:10E96000160281111AC020E030E0A90169A57AA53C
:10E970008BA59CA50F94160281110FC08BC320E0BC
:10E9800030E0A901C701B6010F941602882309F4EB
:10E9900081C319A61AA61BA61CA6D701C601B0588A
:10E9A0008D8F9E8FAF8FB8A329A53AA54BA55CA5E7
:10E9B000505829A33AA34BA35CA39C01AD01BC0111
:10E9C000CD010F947B024B015C0129A13AA14BA11F
:10E9D0005CA1CA01B9010F947B029B01AC01C50186
:10E9E000B4010F9480060F94EB0825966CAF7DAFB1
:10E9F0008EAF9FAF25978091D4059091D505A091BA
:10EA0000D605B091D7058DA39EA3AFA3B8A7A70144
:10EA10009601BC01CD010F9480066DAB7EAB8FAB30
:10EA200098AF2091D8053091D9054091DA055091E1
:10EA3000DB052DA73EA74FA758AB29A53AA54BA5A7
:10EA40005CA56DA57EA58FA598A90F9480066196FB
:10EA50006CAF7DAF8EAF9FAF61978091490490916D
:10EA60004A04A0914B04B0914C0489AB9AABABAB78
:10EA7000BCAB2DA93EA94FA958ADBC01CD010F9447
:10EA80007F066B017C0120914D0430914E04409132
:10EA90004F045091500429AF3AAF4BAF5CAF619631
:10EAA0002CAD3DAD4EAD5FAD619769AD7AAD8BAD2F
:10EAB0009CAD0F947F064B015C018091DC05909129
:10EAC000DD05A091DE05B091DF0521968CAF9DAFED
:10EAD000AEAFBFAF21979C01AD0160915104709121
:10EAE000520480915304909154040F947F062B019B
:10EAF0003C012091550430915604409157045091A7
:10EB0000580429962CAF3DAF4EAF5FAF2997809147
:10EB1000E0059091E105A091E205B091E3056596CD
:10EB20008CAF9DAFAEAFBFAF6597A70196016D8D5E
:10EB30007E8D8F8D98A10F947B022D966CAF7DAF4B
:10EB40008EAF9FAF2D97A501940169A17AA18BA1EA
:10EB50009CA10F947B029B01AC012D966CAD7DAD09
:10EB60008EAD9FAD2D970F9480062D966CAF7DAF27
:10EB70008EAF9FAF2D97A50194016D8D7E8D8F8DEA
:10EB800098A10F947B024B015C01A701960169A13A
:10EB90007AA18BA19CA10F947B029B01AC01C501C2
:10EBA000B4010F947F062D962CAD3DAD4EAD5FADFB
:10EBB0002D970F94F3066B017C0120E030E0A90152
:10EBC0000F94160287FF0AC02BED3FE049EC50E49A
:10EBD000C701B6010F9480066B017C01332051F010
:10EBE0002BED3FE049EC50E4C701B6010F947F06DE
:10EBF0006B017C0120E030E0A901C701B6010F9450
:10EC00001602811120C029A93AA94BA95CA96DA1BE
:10EC10007EA18FA198A50F941602811114C029AD71
:10EC20003AAD4BAD5CAD6DA57EA58FA598A90F94AF
:10EC30001602811108C09BEDC92E9FE0D92E99ECD8
:10EC4000E92E90E4F92EA701960125966CAD7DADD5
:10EC50008EAD9FAD25970F947B024B015C0120E0A8
:10EC600030E0A901C301B2010F9416028823C9F054
:10EC7000A5019401C501B4010F947B024B015C0115
:10EC8000A3019201C301B2010F947B029B01AC016D
:10EC9000C501B4010F9480060F94EB084B015C0191
:10ECA0000DC020E030E0A901C501B4010F94A60811
:10ECB00087FF04C0B7FAB094B7F8B0942FE632E1FA
:10ECC00043E85AE3C501B4010F94160287FDFAC167
:10ECD000C501B4010F94F5070F94C9071B01672BF9
:10ECE00019F422242394312CB10180E090E00F9498
:10ECF0001A024B015C019B01AC01C701B6010F94E4
:10ED00005C076DA37EA38FA398A7A5019401C301FF
:10ED1000B2010F945C0725966CAF7DAF8EAF9FAFAD
:10ED2000259765962CAD3DAD4EAD5FAD65972996A7
:10ED30006CAD7DAD8EAD9FAD29970F947F06A5017B
:10ED400094010F945C0729966CAF7DAF8EAF9FAF97
:10ED500029972DA13EA14FA158A5CA01B9010F9431
:10ED60007B0220E030E040E05FE30F947B029B01F8
:10ED7000AC0160E070E080E89FE30F947F0669AF2C
:10ED80007AAF8BAF9CAF21962CAD3DAD4EAD5FAD54
:10ED9000219729873A874B875C8765968CAD9DAD17
:10EDA000AEADBFAD65978D879E87AF87B88B6091FD
:10EDB000040270910502072E000C880B990B0F942A
:10EDC0001C022091000230910102409102025091F8
:10EDD00003020F947B022AE037ED43E25CE30F94D9
:10EDE0007B02698F7A8F8B8F9C8F0E94F6B29B017A
:10EDF000AC0128533F4F4F4F5F4F21962CAF3DAF93
:10EE00004EAF5FAF21974D8C5E8C6F8C78A041E048
:10EE100050E05AAB49AB59E15DA749A95AA942153F
:10EE2000530509F410C10E942E660E94F6B2DC015F
:10EE3000CB0121962CAD3DAD4EAD5FAD2197821B30
:10EE4000930BA40BB50BB7FD11C00E94F6B29B014A
:10EE5000AC0128533F4F4F4F5F4F21962CAF3DAF32
:10EE60004EAF5FAF219780E00E94A8503DA5315082
:10EE70003DA73323E9F129AD3AAD4BAD5CAD69A1B6
:10EE80007AA18BA19CA10F947B026B017C012DA127
:10EE90003EA14FA158A5B201C3010F947B02A70167
:10EEA00096010F9480067B018C0129AD3AAD4BADE4
:10EEB0005CADB201C3010F947B024B015C012DA13B
:10EEC0003EA14FA158A569A17AA18BA19CA10F9445
:10EED0007B029B01AC01C501B4010F947F062B019D
:10EEE0003C01C701D80189A39AA3ABA3BCA351C01D
:10EEF00049A95AA9BA0180E090E00F941A022DA105
:10EF00003EA14FA158A50F947B024B015C010F94C9
:10EF100059076B017C01C501B4010F94E1084B0155
:10EF20005C01A70196016D8D7E8D8F8D98A10F9448
:10EF30007B022B013C01A501940169A57AA58BA553
:10EF40009CA50F947B029B01AC01C301B2010F94FD
:10EF500080062B013C01A50194016D8D7E8D8F8D66
:10EF600098A10F947B024B015C01A701960169A552
:10EF70007AA58BA59CA50F947B029B01AC01C501D2
:10EF8000B4010F947F0669A37AA38BA39CA359E1D4
:10EF90005DA79201A3016DA97EA98FA998AD0F94D9
:10EFA000800669837A838B839C8329A13AA14BA134
:10EFB0005CA161966CAD7DAD8EAD9FAD61970F94F8
:10EFC00080066D837E838F83988725962CAD3DAD1B
:10EFD0004EAD5FAD259769857A858B859C850F94AD
:10EFE000800669877A878B879C8729962CAD3DADF3
:10EFF0004EAD5FAD29976D857E858F8598890F947D
:10F0000080066D877E878F87988BCE0101960E9440
:10F010000F55E0901115198A1A8A1B8A1C8ACE0195
:10F0200041966C018E01075E1F4F9E01235F3F4F8B
:10F03000AE01475F5F4FBE016B5F7F4F40970E94FD
:10F040009C9B811120C0E09011151D8A1E8A1F8A89
:10F05000188EDE0155966D018E01075E1F4F25E566
:10F0600034E041E554E06DE474E089E494E00E940A
:10F070009C9B80E1E9E4F4E0A4EDB5E001900D9201
:10F080008A95E1F71FC029A93AA92F5F3F4F3AABF4
:10F0900029ABC3CEE4E4F9E484918F010F5F1F4FE5
:10F0A000882321F00E94F0F6F801F6CFE1E6FCE1BA
:10F0B00084918F010F5F1F4F882321F00E94F0F68B
:10F0C000F801F6CFCC5ADF4F0FB6F894DEBF0FBE73
:10F0D000CDBFDF91CF911F910F91FF90EF90DF9007
:10F0E000CF90BF90AF909F908F907F906F905F90E8
:10F0F0004F903F902F9008952F923F924F925F92A2
:10F100006F927F929F92AF92BF92CF92DF92EF92D7
:10F11000FF920F931F93CF93DF93CDB7DEB728975E
:10F120000FB6F894DEBF0FBECDBF2A013B01902E73
:10F13000A12E6901082F10E0F801E35BFF4EE49176
:10F14000BB24B3941E160CF4B12CFF24F39420E0DE
:10F1500030E0A901C301B2010F94A60818160CF003
:10F16000F12C000F111F000F111FC8018C529A4F74
:10F170001C01FC0110821182128213820E94BD8F39
:10F18000F1014082518262827382E090111520E089
:10F1900030E0A901692D7A2DC6010F941602811164
:10F1A00008C0F801E050F04F85919591A591B49178
:10F1B00003C0892D9A2DD6018D839E83AF83B88796
:10F1C00019821A821B821C82CE0101966C018E016B
:10F1D0000B5F1F4F20EE35E04CED55E068ED75E01C
:10F1E00084ED95E00E949C9B0E94D54BBF100E942D
:10F1F0000F9928960FB6F894DEBF0FBECDBFDF91F2
:10F20000CF911F910F91FF90EF90DF90CF90BF9023
:10F21000AF909F907F906F905F904F903F902F9016
:10F220000895CF92DF92EF92FF920F931F936A019E
:10F23000E090DC05F090DD050091DE051091DF0522
:10F24000FB012081318142815381FC016081718108
:10F250008281938162D81F910F91FF90EF90DF9090
:10F26000CF900895CF92DF92EF92FF920F931F936A
:10F270006B01FC01E080F18002811381E4EDF5E097
:10F28000248135814681578160817181828193819A
:10F2900044D81F910F91FF90EF90DF90CF90089589
:10F2A0002F923F924F925F926F927F928F929F9296
:10F2B000AF92BF92CF92DF92EF92FF920F931F9384
:10F2C000CF93DF93CDB7DEB768970FB6F894DEBF64
:10F2D0000FBECDBF182F909124159770973069F409
:10F2E0008FE40E948190882319F00E94F88F03C058
:10F2F0008FE40E943A908111F6C10E94D54B809113
:10F30000000290910102A0910202B0910302809349
:10F310009C0590939D05A0939E05B0939F058091B9
:10F3200004029091050290939B0580939A0584E6D0
:10F3300090E0909305028093040281E08093C705DA
:10F34000111119C088E50E943A90382E89E50E9473
:10F350003A90182F8AE50E943A90282E311006C064
:10F36000111110C081110EC0312E0AC0112351F0AD
:10F37000312E082F08C03324339411E02224239423
:10F3800001E001C000E00E94939082E50E9481901C
:10F39000882361F00E9407906B017C0120E030E03F
:10F3A000A9010F941602882371F106C0C12CD12C3B
:10F3B00080EAE82E80E4F82E011105C0311003C068
:10F3C000112309F40EC1C0925104D0925204E0926C
:10F3D0005304F09254042091DC053091DD054091F6
:10F3E000DE055091DF05C701B6010F94A608181677
:10F3F00054F419821A821B821C82BE016F5F7F4FF8
:10F4000081E594E02FDF01110DC0311003C011110F
:10F41000E3C0E7C0111106C080E00E940C4F00233A
:10F42000B1F3DAC01092D8051092D9051092DA051E
:10F430001092DB051092D4051092D5051092D605D6
:10F440001092D7050E94BD8FEDE4F0E12491288F42
:10F45000E1E4F0E185909590A590B490E5E4F0E1C9
:10F460004590559065907490A3019201C501B40137
:10F470000F94A60818162CF4A5019401C301B2013B
:10F4800004C0A3019201C501B4010F945C076B0194
:10F490007C01E4E0F0E185919591A591B4918D878F
:10F4A0009E87AF87B88BE0E0F0E185919591A591BB
:10F4B000B491898B9A8BAB8BBC8B2D853E854F8508
:10F4C0005889BC01CD010F94160287FD09C09D85A6
:10F4D0009D8BAE85AE8BBF85BF8B28892D8708C0DD
:10F4E00089898D8B9A899E8BAB89AF8BBC89BD87AF
:10F4F000A7019601C701B6010F947B0220E030E01E
:10F5000040E85FE30F9480060F94EB089B01AC0189
:10F510006D897E898F899D850F947B0269877A87A3
:10F520008B879C87EEE4F0E1F49020E030E040EC43
:10F530005FE3C301B2010F947B022B013C016F2DED
:10F54000FF0C770B880B990B0F941C029B01AC01ED
:10F55000C301B2010F947B0269837A838B839C83FE
:10F5600020E030E040EC5FE3C501B4010F947B0282
:10F570006B017C01288D622F220F770B880B990B72
:10F580000F941C029B01AC01C701B6010F947B02D2
:10F590006D837E838F839887AE01475F5F4FBE0187
:10F5A0006F5F7F4FCE0105963CDE0E940F9910924F
:10F5B000D8051092D9051092DA051092DB05109249
:10F5C000D4051092D5051092D6051092D7050111D9
:10F5D00023CF311021CF1BCF81E00E940C4F0111AE
:10F5E00003C0222009F457C0809124158370833012
:10F5F000E9F060E086E89CE10E945391ECE4F2E4DB
:10F6000084918F010F5F1F4F882321F00E94F0F635
:10F61000F801F6CFE7E7FCE184918F010F5F1F4F00
:10F620008823C9F10E94F0F6F801F6CF0E94BD8F41
:10F6300080E090E0A0E2B1E48093490490934A0412
:10F64000A0934B04B0934C0480934D0490934E04CC
:10F65000A0934F04B09350048091DC059091DD0598
:10F66000A091DE05B091DF05809351049093520480
:10F67000A0935304B093540419821A821B821C82F3
:10F68000AE014F5F5F4F6DE474E089E494E0C9DD43
:10F6900082E00E940C4F0E94BD8F60E084E99CE1F3
:10F6A0000E9453918091C5058093C70580919C0568
:10F6B00090919D05A0919E05B0919F0580930002B9
:10F6C00090930102A0930202B093030280919A05E5
:10F6D00090919B05909305028093040283E08093B0
:10F6E00051020E9452B568960FB6F894DEBF0FBE65
:10F6F000CDBFDF91CF911F910F91FF90EF90DF90E1
:10F70000CF90BF90AF909F908F907F906F905F90C1
:10F710004F903F902F9008950F931F93CF93DF93B7
:10F7200094E0899FE00111248E010B571C4FFE01CC
:10F73000E853FA4FDE01A45CBB4F2D913D914D91F2
:10F740005C9160817181828193810F948006F801C0
:10F750006083718382839383FE01E75BF34E85911F
:10F760009591A591B491FE01EF56FC4F8083918352
:10F77000A283B383FE01EB5AF34E85919591A59137
:10F78000B491C35FDD4F88839983AA83BB83DF91E4
:10F79000CF911F910F910895EF92FF920F931F93B6
:10F7A000CF93DF937C0184E50E948190D82F88233A
:10F7B00049F10E94E78FC82F181604F5ECE4F2E433
:10F7C00084918F010F5F1F4F882321F00E94F0F674
:10F7D000F801F6CF8DE40E94F0F6B70180E090E0EA
:10F7E0004AE00E9443F76C2FCC0F770B86E39CE135
:10F7F0000E94CF688AE00E94F0F608C0809301055D
:10F80000D0E004C080911115809301058D2FDF9108
:10F81000CF911F910F91FF90EF9008954F925F92BB
:10F820006F927F929F92AF92BF92CF92DF92EF92B0
:10F83000FF920F931F93CF93DF931F92CDB7DEB745
:10F840000E945E8F811151C28091CE07853028F4CD
:10F850000E9434F8AC0197FF3DC18091210F8823AD
:10F8600009F443C28091CE07811102C0109299051C
:10F87000EE24E3944091C1115091C2116091C311E3
:10F880007091C4118091BD119091BE11A091BF11D2
:10F89000B091C011481759076A077B0708F4E12C9B
:10F8A00000E010E0BB24B39480E6A82E9FE0C92EB0
:10F8B0009CE1D92E2DE8922E8091CE07853008F05C
:10F8C00014C2E11012C28091990581110EC280917B
:10F8D000181190911911A0911A11B0911B118093D8
:10F8E000C1119093C211A093C311B093C41141E010
:10F8F00050E0BE016F5F7F4F80E191E10E94B9D07F
:10F90000019719F4898190E002C08FEF9FEFF82EE4
:10F91000EE24E3944090C1115090C2116090C31145
:10F920007090C4114091BD115091BE116091BF11F2
:10F930007091C0114416550666067706C8F4E12C8E
:10F940008F3FFFEF9F0709F46EC02AE0821709F48A
:10F950008FC08DE0F81609F48BC093E2F91619F008
:10F96000EAE3FE129DC080919805811199C075C08F
:10F970000E94D54B80E191E10E94E3D480912B114C
:10F98000882359F1815080932B11989EC001112436
:10F9900041E061E0805D9E4E0E9475ECE0912B118C
:10F9A00024E0E29FF0011124E45DFE4E408151818C
:10F9B000628173814093C1115093C2116093C3114E
:10F9C0007093C41180E191E10E94A4CE8091220F36
:10F9D0008823C1F0B092210F15C01092210F0E9410
:10F9E000E34C0E94C0990E941A996D3371058105FC
:10F9F000910530F0D0920809C09207090E945E8FED
:10FA0000109284038091210F81112BC0E2E2FCE16E
:10FA100084913F019FEF691A790A8823F1F00E94CF
:10FA2000F0F6F301F5CFE4E4F9E484913F012FEF20
:10FA3000621A720A882321F00E94F0F6F301F5CFD2
:10FA4000E3E1FCE184913F019FEF691A790A882381
:10FA500021F00E94F0F6F301F5CFE3E2FE1208C0B8
:10FA600005C023E2F2123EC100E010E0B092990519
:10FA7000109298050115110519F40E942E660DC00B
:10FA80008091E905A89E000D111D1124F801E35194
:10FA9000FA4F108280E00E942D8F00E010E00CCF22
:10FAA0000F35110508F008CFFBE3FF1202C0B0923A
:10FAB0009805809198058111FFCE8091E905F801A4
:10FAC000A89EE00DF11D1124E351FA4FF0820F5F63
:10FAD0001F4FF2CE982F20912014309121148A309C
:10FAE00019F09D3009F0CCC0109297052115310511
:10FAF00019F40E942E66A8CEF901E95CFA4F108233
:10FB0000109221141092201427E335E08901F901A5
:10FB100080812F5F3F4F8032C9F378018E3409F026
:10FB20007CC00115110509F478C06AE07CE1C801C8
:10FB30000F949501DD24D394892B11F4D12C09C0A5
:10FB40006EE470E0C80104960F94AF09009709F0C5
:10FB50008C014AE050E060E070E0C80101960E942C
:10FB6000F6FE6093330570933405809335059093CA
:10FB70003605009122141091231420912414309101
:10FB800025140F5F1F4F2F4F3F4F601771078207DC
:10FB9000930729F0D11003C087ED9BE12AC06AE2E8
:10FBA00070E0C7010F94DE099C01009701F1982FC6
:10FBB0009E1910E0992339F09150F701E90FF11DDA
:10FBC00080811827F7CF4AE050E060E070E0C9017B
:10FBD00001960E94F6FE012F10E020E030E0601751
:10FBE00071078207930741F088EB9BE102C08EE822
:10FBF0009BE10E9427EE31CE809133059091340530
:10FC0000A0913505B091360580932214909323146A
:10FC1000A0932414B093251407C080911F0F88234C
:10FC200019F083EE9AE1E5CF80911E02811122C086
:10FC300067E470E0C7010F94AF090097D9F04AE07C
:10FC400050E060E070E001960E94F6FE64307105BD
:10FC500088F4E7E1FBE184918F010F5F1F4F882358
:10FC600021F00E94F0F6F801F6CF60E08DE09BE114
:10FC70000E94539161E087E395E00E94428FE4CDBA
:10FC80002F3531050CF0E0CD9C35C1F40E9434F8DD
:10FC900097FDDACD209197052111D6CD2091201422
:10FCA00030912114A9014F5F5F4F5093211440936D
:10FCB0002014F901E95CFA4F8083C6CD9B3319F417
:10FCC00081E080939705809197058111BDCDC90191
:10FCD00001969093211480932014F901E95CFA4F66
:10FCE0004083B2CD10929805C8CE0F90DF91CF918E
:10FCF0001F910F91FF90EF90DF90CF90BF90AF904A
:10FD00009F907F906F905F904F900895CF93DF9377
:10FD1000EC0160E0CE010E94428F811104C080E0BE
:10FD20000E94A850F6CFCE010E94EE4F8823B9F36F
:10FD3000DF91CF910895CF93DF93CDB7DEB7AB9727
:10FD40000FB6F894DEBF0FBECDBF789484B5826045
:10FD500084BD84B5816084BD85B5826085BD85B56F
:10FD6000816085BD80916E00816080936E001092ED
:10FD70008100809181008260809381008091810068
:10FD800081608093810080918000816080938000F9
:10FD90008091B10084608093B1008091B000816057
:10FDA0008093B00080919100826080939100809157
:10FDB0009100816080939100809190008160809398
:10FDC00090008091A10082608093A1008091A100A9
:10FDD00081608093A1008091A00081608093A00049
:10FDE00080912101826080932101809121018160B5
:10FDF0008093210180912001816080932001809176
:10FE00007A00846080937A0080917A008260809387
:10FE10007A0080917A00816080937A0080917A00E4
:10FE2000806880937A001092C10082E08093C000C5
:10FE30001092C50087E08093C4008091C10080616A
:10FE40008093C1008091C10088608093C10080913F
:10FE5000C10080688093C1008091C1008F7D809334
:10FE6000C1001092A005E0E1FEE184918F010F5FD7
:10FE70001F4F882321F00E94F0F6F801F6CFECE442
:10FE8000F2E484918F010F5F1F4F882321F00E94BD
:10FE9000F0F6F801F6CF14B710FF0DC0E7E0FEE171
:10FEA00084917F012FEFE21AF20A882321F00E9449
:10FEB000F0F6F701F5CF11FF0DC0E6EFFDE18491FB
:10FEC0007F013FEFE31AF30A882321F00E94F0F646
:10FED000F701F5CF12FF0DC0E4EEFDE184917F0143
:10FEE0009FEFE91AF90A882321F00E94F0F6F70142
:10FEF000F5CF13FF0DC0E3EDFDE184917F01AFEF7E
:10FF0000EA1AFA0A882321F00E94F0F6F701F5CFE9
:10FF100015FF0CC0E2ECFDE184918F010F5F1F4FD4
:10FF2000882321F00E94F0F6F801F6CF14BEEBEB27
:10FF3000FDE184918F010F5F1F4F882321F00E9404
:10FF4000F0F6F801F6CF80E20E94F0F6E4EBFDE176
:10FF500084918F010F5F1F4F882321F00E94F0F6DC
:10FF6000F801F6CF8AE00E94F0F6ECE4F2E4849126
:10FF70008F010F5F1F4F882321F00E94F0F6F801D8
:10FF8000F6CFE4EAFDE184918F010F5F1F4F8823D4
:10FF900021F00E94F0F6F801F6CFE0E9FDE184914E
:10FFA0008F010F5F1F4F882321F00E94F0F6F801A8
:10FFB000F6CFE7E5FDE184918F010F5F1F4F8823A6
:10FFC00021F00E94F0F6F801F6CFECE4F2E484911F
:10FFD0008F010F5F1F4F882321F00E94F0F6F80178
:10FFE000F6CFE0E4FDE184918F010F5F1F4F88237E
:10FFF00021F00E94F0F6F801F6CFECE4F2E48491EF
:020000021000EC
:100000008F010F5F1F4F882321F00E94F0F6F80147
:10001000F6CF8091251590912615FE0131967F012E
:10002000BF01009719F0681B790B02C06B52754134
:1000300081E39DE10E94CF6860EF74E08AE19DE179
:100040000E94CF688AE00E94F0F681E08093E40588
:100050008093E5058093E6058093E7058093E805A6
:100060000E9436F58CE0E8ECF5E0A4EDB5E00190F7
:100070000D928A95E1F70E94BD8F80910101806405
:100080008093010180910101806180930101809141
:1000900001018860809301016D9A80910101806265
:1000A0008093010188E00E9499FC809101018860A1
:1000B0008093010186E00E9499FC6C9A82E00E9484
:1000C00099FC87ED80937A0010927E0010927D005B
:1000D00080917E00816080937E0080917E008460AC
:1000E00080937E0080E888BD80916E00846080935C
:1000F0006E006AEF70E080E090E00E94BEB285E0A2
:1001000090E09093A6058093A50560E0809126027B
:10011000909127020E94256220E030E040EA50E4FE
:100120000F94160287FF0AC0809126029091270241
:1001300040979093270280932602E7CF81E391E0D6
:10014000909329028093280260E08091A30590910A
:10015000A4050E94256220E030E848E953E40F94AA
:10016000A608181654F48091A3059091A405409612
:100170009093A4058093A305E7CF809124029091EA
:1001800025020E94B06320E030E040EA50E40F9482
:10019000160287FF0AC080912402909125024097A1
:1001A0009093250280932402E8CF8091A10590913D
:1001B000A2050E94B06320E030E046E153E40F94D2
:1001C000A608181654F48091A1059091A2054096B6
:1001D0009093A2058093A105E8CF1092B3051092E9
:1001E000AF051092B0051092B1051092B2051092B1
:1001F000AB051092AC051092AD051092AE051092B1
:10020000A7051092A8051092A9051092AA0582E3ED
:1002100090E00F94DC05863119F00E942D9A08C0F9
:1002200040E150E063E370E085EB95E00F94CC058E
:1002300081E08093B40526982E9A25982D9A2498CB
:100240002C9A1092C7051092C5051FB7F89480919B
:10025000C605811124C0E2EFF2E48491E8E3F3E4FF
:100260009491E82FF0E0EE0FFF1FED55FD4BA591A7
:10027000B491EC91E92321F461E085E30E94C8B1D7
:1002800085E30E9487BB8CB580618CBD8CB5806492
:100290008CBD84E30E9487BB83E30E9487BB80916F
:1002A000C6058F5F8093C6051FBF579AFBE0CF2E10
:1002B000F3E0DF2E10E0D6016D916D0170E0812F2B
:1002C0000E945E431F5F1530B1F7999A989A80910A
:1002D00007018068809307019A9A809107018064E2
:1002E00080930701809107018062809307018091CC
:1002F00007018860809307018091070180618093E6
:1003000007018091070182608093070180910701B6
:10031000846080930701E0E1CE2EE3E0DE2E10E062
:10032000F60161916F01812F0E942D711F5F1530C1
:10033000B9F780910A01826080930A0180910A01D5
:10034000816080930A0180910A01846080930A0190
:1003500080910A01806480930A0180910A0180687B
:1003600080930A010F9A179A0E9A169A0D9A159A67
:100370000C9A149A0B9A139A389A4098179A80916B
:1003800024158E7F80932415399A4198169A80916E
:1003900024158D7F809324153A9A4298159A80915E
:1003A00024158B7F809324153B9A4398149A80914F
:1003B00080008C7F8093800080918100877E8860A0
:1003C00080938100809180008F7380938000809162
:1003D0008100887F82608093810080E090E4909328
:1003E000890080938800109285001092840080918B
:1003F0006F00826080936F0081E08093C7057894DE
:100400000E9418446C9A0E9414950E9439F90E9427
:100410009F970091D0112091D11110E06801F8E36D
:10042000CF1AD108D7FE04C0680137E3C31AD10838
:10043000D594C7942BA70E9412BDC8014E979695DC
:100440008795B82E0257110916950795D02E2BA522
:100450006EEE962E920E7AEFA72EA20E05E91CE103
:1004600023E147E06CE08C2D0E94E0BB84E00E9419
:10047000E59741EF52E0692D8B2D0E9460BC47EF5C
:1004800052E06A2D8D2D0E9460BC0E94A6BB811196
:10049000E5CF64EC79E080E090E00E94DE6E98E2C7
:1004A00088E10FB6F894A895809360000FBE9093F2
:1004B00060005E0181E2A80EB11C8091730F87FD80
:1004C00043C08091210F81113FC08091220F811183
:1004D00002C00E9466EE8091220F882391F18091E4
:1004E000730F282F082E000C330B3F938F93A7E137
:1004F000BEE1BF93AF93BF92AF920F94AF0140E0C4
:1005000050E0BA0188E79FE00E94A4CE0F900F90C0
:100510000F900F900F900F9080917B0F823088F09A
:100520008091800F9091810FA091820FB091830FE5
:100530008F719927AA27BB27892B8A2B8B2B09F42C
:1005400092C18FEF8093730F8091CF07882309F4B6
:1005500062C01092CF070E94CBC11092CE071092BA
:10056000E9051092CD070E9490B30E94C0990E94A5
:100570008E63109287091092860910928909109251
:1005800088091092540240900F15509010150EE7F4
:100590001EE1F80184918823D9F12DB63EB66AE0B8
:1005A00070E0C8010F945A013C01009721F06C01E2
:1005B000C01AD10A04C0C8010F9465016C01C601BC
:1005C00001962DB73EB7281B390B0FB6F8943EBFE6
:1005D0000FBE2DBF8DB79EB701964C01A601B80185
:1005E0000F948601F401EC0DFD1D10820C0D1D1DF4
:1005F000672811F00F5F1F4FC4010E94026F80E057
:100600000E9403270FB6F8943EBE0FBE2DBEC1CF89
:10061000C2010E94026F8091CE07853008F4FED897
:100620008091CE07882309F49DC080911F0F8823F5
:1006300009F485C00091CD07F0E60F9F80011124D9
:1006400003511A4F6AE77EE1C8010F949501892B87
:10065000F9F080E191E10E9463CE80E191E10E9496
:10066000E3D41092200F10921F0FE7E6FEE1849171
:100670008F010F5F1F4F882341F00E94F0F6F801B1
:10068000F6CF8091200F81115AC00E94645559C045
:10069000F80101900020E9F731976F01C01AD10AE3
:1006A000109210116EE470E0C8010F94AF094C0174
:1006B000009739F421E0C21AD108F801EC0DFD1DB4
:1006C0000EC060E270E00F94AF098C010F5F1F4F06
:1006D0006AE270E0C4010F94AF09FC0131978DE02C
:1006E00081838AE082831382F80101900020E9F778
:1006F0003197AF01401B510BB80180E191E10E949D
:1007000039CF80911011882309F4BBCFE4E4F9E4D8
:1007100084918F010F5F1F4F882321F00E94F0F614
:10072000F801F6CFE0E2FEE184918F010F5F1F4FE9
:10073000882309F4A6CF0E94F0F6F801F5CF0E94B5
:100740005FFD8091CE07882369F081508093CE07AA
:100750008091CD078F5F853018F48093CD0702C05C
:100760001092CD078091EC05882309F46DC090911B
:10077000EC058091EB05981709F466C0ECE4F2E40F
:1007800084918F010F5F1F4F882321F00E94F0F6A4
:10079000F801F6CFE8E5FEE184918F010F5F1F4F6E
:1007A000882321F00E94F0F6F801F6CF8091EC0545
:1007B00080FD8EC08091EC0584FD8AC090E2D92E28
:1007C0008091EC0581FD90C08091EC0585FD8CC089
:1007D00000E28091EC0582FD92C08091EC0586FDDF
:1007E0008EC010E28AE00E94F0F61F9280E28F93A2
:1007F0001F921F931F920F931F92DF92A7E3BEE1F8
:10080000BF93AF931F920E94FAA82DB73EB7255F02
:100810003F4F0FB6F8943EBF0FBE2DBF8091EA0543
:10082000882391F01092210F80E191E10E9463CE24
:1008300080E191E10E94E3D41092200F10921F0FEB
:100840000E9490B30E948E638091EC058093EB052B
:1008500080E00E94A85080E090E0892B09F42DCE22
:100860000E9400002ACE40E050E0B70188E79FE0F8
:100870000E94DBD118160CF064CEF7010190002025
:10088000E9F731971E2F1E19115068F06701C10E4C
:10089000D11C17FDDA94D6018C9190E00F94730966
:1008A000F6018083F1CF8A858E3709F435CE45E095
:1008B00050E0B501CE0101960F94C109892B09F0D2
:1008C0002BCEC5010E946AAB8091730F8F5F3ACE29
:1008D00080E00E94F34CAB01BC0184E59EE10E94E4
:1008E000D16788E5D82E6CCF81E00E94F34CAB0134
:1008F000BC0180E59EE10E94D16709E56ACF82E0F4
:100900000E94F34CAB01BC018CE49EE10E94D167D4
:100910001AE568CF80911F09813041F0823019F4C7
:1009200080E89FE1089583E79FE1089580E99FE1D2
:100930000895CF92DF92EF92FF920F931F93CF9380
:100940008091BD0E9091BE0EA091BF0EB091C00ED1
:10095000B7FF08C01092BD0E1092BE0E1092BF0ECF
:100960001092C00E80910E0990910F09A09110096C
:10097000B09111094091BD0E5091BE0E6091BF0E15
:100980007091C00E84179507A607B70744F48093AB
:10099000BD0E9093BE0EA093BF0EB093C00E80917B
:1009A00051028823E1F14091BD0E5091BE0E60913D
:1009B000BF0E7091C00E8091120990911309A09101
:1009C0001409B09115098A019B01080F191F2A1FEC
:1009D0003B1FC901B8010F941C026B017C0120E090
:1009E00030E0A9010F94160287FD05C020E030E039
:1009F00040E05FE304C020E030E040E05FEBC7018F
:100A0000B6010F9480060F94C407CB010E94A86E14
:100A1000BC0180911809909119090E94DF5BC09177
:100A2000EF07C11108C080911A098823C9F180918C
:100A300051028823A9F14091BD0E5091BE0E6091E4
:100A4000BF0E7091C00E8091120990911309A09170
:100A50001409B09115098A019B01080F191F2A1F5B
:100A60003B1FC901B8010F941C02E0911609F091D7
:100A70001709309721F06083718382839383E0911B
:100A80001B09F0911C09309731F080911A098111EE
:100A900001C0C11119958091EF0781110E94CD5BB2
:100AA0001092EF07CF911F910F91FF90EF90DF9081
:100AB000CF9008958091BD0E9091BE0EA091BF0E73
:100AC000B091C00EB7FF08C01092BD0E1092BE0EBE
:100AD0001092BF0E1092C00E80910E0990910F09D6
:100AE000A0911009B09111094091BD0E5091BE0E18
:100AF0006091BF0E7091C00E84179507A607B707C7
:100B000044F48093BD0E9093BE0EA093BF0EB0939D
:100B1000C00E80915102882399F0209112093091E2
:100B200013098091BD0E9091BE0E820F931F0E94FB
:100B3000A86EBC0180911809909119090E94DF5B91
:100B40002091EF07211108C080911A09882339F1FB
:100B500080915102882319F1409112095091130993
:100B60008091BD0E9091BE0E840F951FE0911609E5
:100B7000F0911709309711F091838083E0911B0960
:100B8000F0911C09309731F080911A09811101C050
:100B9000211119958091EF0781110E94CD5B109270
:100BA000EF0708950F931F93CF93DF9360E085E0E5
:100BB0000E94485BD091D407C0E0D1110BC0809156
:100BC0005102882319F1A6DE00E010E021E041E0A7
:100BD000BC0119C0D13059F4809151028823B1F081
:100BE00000E010E020E041E06BEF70E20CC0D2309A
:100BF00069F480915102882349F000E010E020E080
:100C000041E06EEE70E28C2F0E94345DCF5FDF5FBB
:100C1000C53099F683E08093D307DF91CF911F9180
:100C20000F910895FF920F931F93CF93DF9360E08E
:100C300085E00E94485BD091D407C0E082E0F82EA6
:100C4000D1110CC080915102882309F447C062DEA3
:100C500000E010E021E041E0BC0119C0D13059F4BE
:100C6000809151028823D1F100E010E020E041E0C2
:100C700065EE70E20CC0D23071F48091510288238D
:100C800069F100E010E020E041E066ED70E28C2FB9
:100C90000E94345D23C0D33059F4809151028823DF
:100CA000E9F000E010E020E041E064ED70E2EFCF19
:100CB000D430A1F480915102882371F000E010E05B
:100CC00021E040E069EC70E28C2F0E94345D60917D
:100CD0001E098C2F0E944198F0925102CF5FDF5F76
:100CE000C53009F0ADCFC093D307DF91CF911F91ED
:100CF0000F91FF900895FF920F931F93CF93DF936F
:100D000060E085E00E94485BD091D407C0E082E0BB
:100D1000F82ED1110CC080915102882309F447C0EC
:100D2000F9DD00E010E021E041E0BC0119C0D13064
:100D300059F4809151028823D1F100E010E020E0C5
:100D400041E060EC70E20CC0D23071F4809151024D
:100D5000882369F100E010E020E041E062EB70E2FE
:100D60008C2F0E94345D23C0D33059F480915102FE
:100D70008823E9F000E010E020E041E060EB70E261
:100D8000EFCFD430A1F480915102882371F000E0BC
:100D900010E021E040E065EA70E28C2F0E94345DB3
:100DA00060911E098C2F0E944198F0925102CF5FF2
:100DB000DF5FC53009F0ADCFC093D307DF91CF918E
:100DC0001F910F91FF900895FF920F931F93CF9360
:100DD000DF9360E085E00E94485BD091D407C0E0DB
:100DE00082E0F82ED1110CC080915102882309F4C1
:100DF00047C090DD00E010E021E041E0BC0119C0F7
:100E0000D13059F4809151028823D1F100E010E0F3
:100E100020E041E065E970E20CC0D23071F48091CD
:100E20005102882369F100E010E020E041E064E82D
:100E300070E28C2F0E94345D23C0D33059F480912E
:100E400051028823E9F000E010E020E041E065E78E
:100E500070E2EFCFD430A1F480915102882371F079
:100E600000E010E021E040E06AE670E28C2F0E9492
:100E7000345D60911E098C2F0E944198F0925102BE
:100E8000CF5FDF5FC53009F0ADCFC093D307DF91EF
:100E9000CF911F910F91FF900895FF920F931F9391
:100EA000CF93DF9360E085E00E94485BD091D40748
:100EB000C0E082E0F82ED1110CC08091510288234D
:100EC00009F447C027DD00E010E021E041E0BC016B
:100ED00019C0D13059F4809151028823D1F100E03A
:100EE00010E020E041E06AE570E20CC0D23071F41D
:100EF00080915102882369F100E010E020E041E098
:100F00006DE470E28C2F0E94345D23C0D33059F41D
:100F1000809151028823E9F000E010E020E041E0F8
:100F20006BE470E2EFCFD430A1F4809151028823BA
:100F300071F000E010E021E040E060E470E28C2F0E
:100F40000E94345D60911E098C2F0E944198F0929E
:100F50005102CF5FDF5FC53009F0ADCFC093D3073B
:100F6000DF91CF911F910F91FF900895FF920F9302
:100F70001F93CF93DF9360E085E00E94485BD091A0
:100F8000D407C0E082E0F82ED1110CC0809151024C
:100F9000882309F447C0BEDC00E010E021E041E016
:100FA000BC0119C0D13059F4809151028823D1F18C
:100FB00000E010E020E041E061E370E20CC0D230DC
:100FC00071F480915102882369F100E010E020E083
:100FD00041E062E270E28C2F0E94345D23C0D33086
:100FE00059F4809151028823E9F000E010E020E0FC
:100FF00041E060E270E2EFCFD430A1F48091510281
:10100000882371F000E010E021E040E065E170E24B
:101010008C2F0E94345D60911E098C2F0E94419894
:10102000F0925102CF5FDF5FC53009F0ADCFC093C2
:10103000D307DF91CF911F910F91FF900895FF92F9
:101040000F931F93CF93DF9360E085E00E94485B8E
:10105000D091D407C0E082E0F82ED1110CC080916D
:101060005102882309F447C055DC00E010E021E07C
:1010700041E0BC0119C0D13059F48091510288235C
:10108000D1F100E010E020E041E06CE070E20CC043
:10109000D23071F480915102882369F100E010E0B0
:1010A00020E041E06CEF7FE18C2F0E94345D23C093
:1010B000D33059F4809151028823E9F000E010E028
:1010C00020E041E06AEF7FE1EFCFD430A1F48091DE
:1010D0005102882371F000E010E021E040E06FEE63
:1010E0007FE18C2F0E94345D60911E098C2F0E943D
:1010F0004198F0925102CF5FDF5FC53009F0ADCF6C
:10110000C093D307DF91CF911F910F91FF90089566
:10111000FF920F931F93CF93DF9360E085E00E94CF
:10112000485BD091D407C0E082E0F82ED1110CC00A
:1011300080915102882309F447C0ECDB00E010E005
:1011400021E041E0BC0119C0D13059F48091510235
:101150008823D1F100E010E020E041E060EE7FE183
:101160000CC0D23071F480915102882369F100E003
:1011700010E020E041E060ED7FE18C2F0E94345DC3
:1011800023C0D33059F4809151028823E9F000E064
:1011900010E020E041E069EC7FE1EFCFD430A1F432
:1011A00080915102882371F000E010E021E040E0DE
:1011B0006EEB7FE18C2F0E94345D60911E098C2FB5
:1011C0000E944198F0925102CF5FDF5FC53009F075
:1011D000ADCFC093D307DF91CF911F910F91FF90B7
:1011E0000895EF92FF920F931F93CF93DF9361E0E7
:1011F00081E00E94485BD091D407C0E081E0FF24E9
:10120000F39492E0E92ED1112CC08823D9F080917B
:10121000D2071816BCF04091BD0E5091BE0E6091E1
:10122000BF0E7091C00E4F5F5F4F6F4F7F4F409367
:10123000BD0E5093BE0E6093BF0E7093C00E8F5FB5
:101240008093D20780915102882309F44BC000E0BB
:1012500010E020E041E06DEB7FE18C2F0E94345DD7
:1012600041C0D130F1F49091D207913029F08091B2
:1012700051028823B9F10DC08091EF078823B9F39B
:101280001092EF07E0921D098091BA0E882379F33E
:1012900032C081E0913009F080E020E249EA5FE16C
:1012A0001FC0D230F9F49091D207923029F080918A
:1012B00051028823B9F00DC08091EF078823B9F35C
:1012C0001092EF07F0921D098091BA0E882379F3EE
:1012D00012C081E0923009F080E020E24EE95FE147
:1012E0006C2F45D7CF5FDF5F80E0C53009F08BCF33
:1012F00083E08093D307DF91CF911F910F91FF90EF
:10130000EF900895EF92FF920F931F93CF93DF9387
:101310001092D1071092D00761E081E00E94485BF3
:10132000D091D407C0E081E0FF24F394D1112CC008
:101330008823D9F08091D2071816BCF04091BD0ED9
:101340005091BE0E6091BF0E7091C00E4F5F5F4F07
:101350006F4F7F4F4093BD0E5093BE0E6093BF0EF4
:101360007093C00E8F5F8093D207809151028823C3
:1013700009F4BAC000E010E021E041E068E27FE15A
:101380008C2F0E94345DB0C0D130F9F41091D20797
:10139000113031F080915102882309F4A5C00DC0AD
:1013A0008091EF078823B1F31092EF070E94CD5B85
:1013B0008091BA0E882371F39FC081E0113009F04B
:1013C00080E024E04EE65FE145C0D23009F510919F
:1013D000D207123031F080915102882309F484C081
:1013E0000FC08091EF078823B1F31092EF0788EDCB
:1013F0009AE80E9438958091BA0E882361F37CC0E8
:1014000081E0123009F080E023E042E65FE122C093
:10141000D33019F51091D207133031F08091510279
:10142000882309F461C00FC08091EF078823B1F3CE
:101430001092EF078BED9AE80E9438958091BA0ED2
:10144000882361F359C081E0133009F080E023E084
:1014500046E55FE16C2F8BD647C0D43009F044C01D
:10146000E090D20784E0E81629F0809151028823A9
:10147000D9F125C08091EF078823B9F31092EF07C7
:10148000F092E9071092E5071092E6071092E7073D
:101490001092E8076091D007660F770B6E5E7A4E68
:1014A0000EED1AE822E231E048E750E087E49FE1E0
:1014B0000E9447A98091BA0E8823B9F21DC0E0911D
:1014C000D007EE0FFF0BEE5EFA4E808191810E94F5
:1014D000A86E9C0181E094E0E91280E000E048E31E
:1014E0005FE16C2F0E94975CCF5FDF5F80E0C530CB
:1014F00009F01CCFC093D307DF91CF911F910F91BB
:10150000FF90EF900895EF92FF920F931F93CF9368
:10151000DF93CDB7DEB72B970FB6F894DEBF0FBEC3
:10152000CDBF7C019091D007492F092E000C550B9F
:101530002091D107213051F0223019F021E03FE114
:101540000AC097FF06C026E13FE105C02DE03FE15C
:1015500002C02FE13FE15F939F933F932F938E0152
:101560000F5F1F4F1F930F930F94AF01F09213154E
:10157000E092121580E00E94436381E08093F007BF
:10158000C8010E94867E1092F0070F900F900F9076
:101590000F900F900F902B960FB6F894DEBF0FBEF2
:1015A000CDBFDF91CF911F910F91FF90EF900895E4
:1015B00088EC90E0A8CF80EF90E0A5CFE091D00735
:1015C000EE0FFF0BEE5EFA4E808191819CCF2F9241
:1015D0003F924F925F926F927F928F929F92AF92C3
:1015E000BF92CF92DF92EF92FF920F931F93CF9310
:1015F000DF93CDB7DEB76F970FB6F894DEBF0FBE9F
:10160000CDBF8091EF071092EF07882319F00E9459
:10161000CD5BF3C02090B5053090B6058091B7053D
:101620009091B8059F8F8E8F8091B9059091BA05E2
:10163000A091BB05B091BC058A8F9B8FAC8FBD8FED
:101640004090BD055090BE056090BF057090C005EC
:101650008090C1059090C205A090C305B090C405CC
:1016600060E085E00E94485BE090D407F12CDE0149
:1016700011966D01E1100DC0809151028823E1F0B7
:10168000C1010E947C6E8C0120E040E063EF7EE1AE
:1016900010C0B1E0EB1210C080915102882361F0BC
:1016A0008E8D9F8D0E947C6E8C0120E040E067EE65
:1016B0007EE18F2D0E94345D8A8D9B8DAC8DBD8D1A
:1016C0008E8B9F8BA88FB98FB601CE0146960E9454
:1016D0003D9A92E0E9120BC0809151028823B1F04B
:1016E00000E010E020E040E064ED7EE10CC0A3E00B
:1016F000EA120CC080915102882341F0860120E05B
:1017000040E063ED7EE18F2D0E94345D4E8A5F8A5A
:10171000688E798EB601CE0146960E943D9AB4E05D
:10172000EB120BC0809151028823B1F000E010E071
:1017300020E040E060EC7EE10CC085E0E8120CC0E7
:1017400080915102882341F0860120E040E06FEB58
:101750007EE18F2D0E94345D20E030E048EC52E4C1
:10176000C501B4010F945C070F94C407CB016AE074
:1017700070E00F9458099F938F9320E030E04AE780
:1017800054E4C501B4010F945C070F94C4079F9300
:101790008F937F936F93A7EBBEE1BF93AF93DF92DD
:1017A000CF920F94AF010FB6F894DEBF0FBECDBF3E
:1017B000B6E0EB120BC0809151028823B1F000E03B
:1017C00010E020E040E066EA7EE10CC087E0E8122D
:1017D0000CC080915102882341F0860120E040E056
:1017E00065EA7EE18F2D0E94345DF394E39495E0E9
:1017F000F91240CF88E08093D3076F960FB6F89424
:10180000DEBF0FBECDBFDF91CF911F910F91FF9033
:10181000EF90DF90CF90BF90AF909F908F907F9090
:101820006F905F904F903F902F900895CF92DF92EE
:10183000EF92FF920F931F93CF93DF9300D01F92ED
:10184000CDB7DEB78091BD0E9091BE0EA091BF0EB8
:10185000B091C00EB7FF08C01092BD0E1092BE0E20
:101860001092BF0E1092C00E80910E0990910F0938
:10187000A0911009B09111094091BD0E5091BE0E7A
:101880006091BF0E7091C00E84179507A607B70729
:1018900044F48093BD0E9093BE0EA093BF0EB09300
:1018A000C00E80915102882379F14091BD0E509174
:1018B000BE0E6091BF0E7091C00E80911209909182
:1018C0001309A0911409B09115096A017B01C80E92
:1018D000D91EEA1EFB1EC701B6010F941A0220E0B2
:1018E00030E048EC52E40F947B0269837A838B8367
:1018F0009C83CE0101960E94E56CBC018091180981
:10190000909119090E94DF5B1091EF0711110AC035
:1019100080911A09882309F442C0809151028823DA
:1019200009F43DC04091BD0E5091BE0E6091BF0EB6
:101930007091C00E8091120990911309A091140921
:10194000B09115096A017B01C80ED91EEA1EFB1E63
:10195000C701B6010F941A0220E030E048EC52E4CF
:101960000F947B020F94C907E0911609F0911709B3
:10197000309721F06083718382839383E0911B0908
:10198000F0911C09309731F080911A09811101C042
:10199000111119958091EF0781110E94CD5B109272
:1019A000EF070F900F900F900F90DF91CF911F9145
:1019B0000F91FF90EF90DF90CF900895CF92DF923C
:1019C000EF92FF920F931F93CF93DF9300D01F925C
:1019D000CDB7DEB78091BD0E9091BE0EA091BF0E27
:1019E000B091C00EB7FF08C01092BD0E1092BE0E8F
:1019F0001092BF0E1092C00E80910E0990910F09A7
:101A0000A0911009B09111094091BD0E5091BE0EE8
:101A10006091BF0E7091C00E84179507A607B70797
:101A200044F48093BD0E9093BE0EA093BF0EB0936E
:101A3000C00E80915102882379F14091BD0E5091E2
:101A4000BE0E6091BF0E7091C00E809112099091F0
:101A50001309A0911409B09115096A017B01C80E00
:101A6000D91EEA1EFB1EC701B6010F941C0220E01E
:101A700030E048EC52E40F947B0269837A838B83D5
:101A80009C83CE0101960E94E56CBC0180911809EF
:101A9000909119090E94DF5B1091EF07111109C0A5
:101AA00080911A09882309F43FC08091510288234C
:101AB000D9F14091BD0E5091BE0E6091BF0E709154
:101AC000C00E8091120990911309A0911409B09150
:101AD00015096A017B01C80ED91EEA1EFB1EC7014B
:101AE000B6010F941C0220E030E048EC52E40F9461
:101AF0007B02E0911609F0911709309721F060837D
:101B0000718382839383E0911B09F0911C093097C4
:101B100031F080911A09811101C01111199580913C
:101B2000EF0781110E94CD5B1092EF070F900F908D
:101B30000F900F90DF91CF911F910F91FF90EF9039
:101B4000DF90CF900895CF92DF92EF92FF920F93A4
:101B50001F93CF93DF9300D01F92CDB7DEB7809154
:101B6000BD0E9091BE0EA091BF0EB091C00EB7FFFA
:101B700008C01092BD0E1092BE0E1092BF0E1092B1
:101B8000C00E80910E0990910F09A0911009B0919B
:101B900011094091BD0E5091BE0E6091BF0E709123
:101BA000C00E84179507A607B70744F48093BD0EAF
:101BB0009093BE0EA093BF0EB093C00E80915102C1
:101BC000882379F14091BD0E5091BE0E6091BF0EF9
:101BD0007091C00E8091120990911309A09114097F
:101BE000B09115096A017B01C80ED91EEA1EFB1EC1
:101BF000C701B6010F941C022AE037ED43E25CE313
:101C00000F947B0269837A838B839C83CE01019638
